:1000000000800020BD010000B5E100006DE10000AE
:100010006DE100006DE100006DE100006DE10000A8
:100020006DE100006DE100006DE10000B5E1000050
:10003000B5E100006DE10000AD0B0100B10B010066
:10004000B5E10000B5E10000B5E10000B5E1000058
:10005000B5E10000B5E10000B5E10000B5E1000048
:10006000B5E10000B5E10000B5E10000B5E1000038
:10007000B5E10000B5E10000B5E10000B5E1000028
:10008000B5E10000B5E10000B5E10000B5E1000018
:10009000B5E10000B5E10000B5E10000B5E1000008
:1000A00045B8000051B80000B5E10000B5E100001E
:1000B000B5E10000B5E10000B5E10000B5E10000E8
:1000C000B5E10000B5E10000B5E10000B5E10000D8
:1000D000B5E10000B5E10000B5E10000B5E10000C8
:1000E000B5E10000B5E10000B5E10000B5E10000B8
:1000F000B5E10000B5E10000B5E10000FDEF000052
:10010000B5E1000081F50000B5E10000B5E10000B7
:10011000B5E10000B5E10000B5E10000B5E1000087
:10012000B5E10000B5E10000B5E10000B5E1000077
:10013000B5E10000B5E10000B5E10000B5E1000067
:10014000B5E10000B5E10000B5E10000B5E1000057
:100150005D0F0100710F0100850F0100990F010073
:10016000B5E100009DF80000B5E10000B5E1000038
:10017000B5E10000B5E10000B5E10000B5E1000027
:10018000B5E10000B5E10000B5E10000B5E1000017
:10019000B5E10000B5E10000B5E10000B5E1000007
:1001A000B5E10000B5E10000B5E10000B5E10000F7
:1001B000B5E10000B5E10000B5E10000564B4CF29E
:1001C000205210B51A804DF628121A8000BF00BFC9
:1001D0000DF0F4FF514B4FF010621A60504A9A60D4
:1001E000504ADA60504A136813F4807304D14F49BF
:1001F0000B604FF4A85313604D4B1A78110703D5C9
:100200001A7842F008021A704A4B4B492A221A7097
:100210004A4A4B4B8B4204D252F8040F43F8040B6A
:10022000F8E7484B484900228B4202D243F8042B9E
:10023000FAE74649464A002352F8230041F82300D2
:1002400001336F2BF8D1434B434A802103F8011B44
:100250009342FBD1414B3D4A1A60414B8A221A70AE
:10026000A3F5805324225A70A0221A709A7992071B
:10027000FCD59A79D406FCD43A4A937903F00C035E
:10028000082B384BF9D103221A7140225A719A79FE
:100290009006FCD5334A9179324B4906FBD5324A58
:1002A000324911600221516020221A709A7902F0BD
:1002B0000C020C2AFAD12E4B2E4A1A602E4B2F4AD2
:1002C0001A6000225A60072243F8042C2C4AC3F813
:1002D0000C2D62B60EF0FCFA144B1B68DA0705D53C
:1002E00028480EF0C9F8284B284A1A60284B1B787A
:1002F0005B0609D5244C254B22689A4204D121483B
:100300000EF0BAF80023236012F0B6F90DF05CFF8E
:1003100010F0BAFEFEE700BF0E200540308004401A
:10032000823F04000100002B10D0034014D0034092
:1003300002D0074000E00740949CFF1F7C6401004E
:100340004088FF1F949CFF1F44A4FF1F0082FF1FD3
:100350000000000000E400E05FE400E008ED00E0E1
:100360000050064000400640448004400000030165
:1003700004800440C010050014E000E0FF76010096
:1003800000002020DE217E631CE00340A5C3945AB8
:1003900000F00740FFFFFFFFFFFFFFFFFFFFFFFF32
:1003A000FFFFFFFFFFFFFFFFFFFFFFFFFFFFFFFF5D
:1003B000FFFFFFFFFFFFFFFFFFFFFFFFFFFFFFFF4D
:1003C000FFFFFFFFFFFFFFFFFFFFFFFFFFFFFFFF3D
:1003D000FFFFFFFFFFFFFFFFFFFFFFFFFFFFFFFF2D
:1003E000FFFFFFFFFFFFFFFFFFFFFFFFFFFFFFFF1D
:1003F000FFFFFFFFFFFFFFFFFFFFFFFFFFFFFFFF0D
:10040000FFFFFFFFFFFFFFFFFFFFFFFFDEF9FFFF23
:1004100010B5054C237833B9044B13B10448AFF33E
:1004200000800123237010BD949CFF1F000000007A
:1004300078640100084B10B51BB108490848AFF3B8
:1004400000800848036803B910BD074B002BFBD0A0
:10045000BDE81040184700BF00000000989CFF1F37
:1004600078640100949CFF1F0000000038B504462A
:10047000104621700A491D4611F0E6FE01464FF074
:100480007E5011F095FF074911F0DEFEE5606060D7
:10049000256165610EF0ACF9E061204638BD00BF12
:1004A000DB0FC9400024744938B50446104621705A
:1004B00009491D4611F0C8FE01464FF07E5011F06B
:1004C00077FF064911F0C0FEE56060602561656157
:1004D0000EF08EF9E06138BDDB0FC940002474498D
:1004E00038B503780446032B20D8DFE803F01A1848
:1004F0001002C168406911F09DFD0D490546606814
:1005000011F056FF0146284611F052FF38BD084948
:10051000406811F04DFFE16811F096FE38BDC068EB
:1005200038BDC168406911F085FD38BD002038BD77
:100530000024744970B504460E460EF059F905467C
:10054000E069281A11F02CFEE3682361E561666119
:10055000A0610146606811F02BFF0146A0601048C1
:1005600011F026FF11F0FCF910F096FE11F00EFDCF
:10057000054601464FF07E5011F05CFD616911F0B7
:1005800063FE21690646284611F05EFE01463046AC
:1005900011F052FDE0602046BDE87040FFF7A0BFBB
:1005A000000080BF08B50E200DF0BAFC114B1B886F
:1005B000012B19D0104B1B88984213DB40F6FF71BA
:1005C0008842D4BFC3EB0001C3EB0101C1EB013191
:1005D000C3F57F630F33282091FBF3F1BDE808409A
:1005E0000DF05CBF0021F3E70146BDE80840142090
:1005F0000DF054BFF89EFF1F8C9DFF1F10B50446E1
:1006000010F08AFC204610BD70B44C88A04220D95E
:1006100001230133DBB21CB2660031F8144084427E
:100620001D46F6D3A04211D005F10045013D965B71
:1006300031F8151032F81530401AF21A00FB02F0AA
:10064000641A90FBF4F4E01870BC7047905B70BCC7
:10065000704702260125E5E700280CDA064A4342E6
:1006600082FB0320DA17C2EB600000EB4000A3EB33
:100670008000C0F10C007047ABAAAA2A38B5234B02
:100680001B78002B2CD015200DF04AFC204B186055
:10069000204B1B88984203DA1F4C237863BB38BD7C
:1006A0001E4A1488A042A4EB0302A8BF20467F2A5A
:1006B0001CDDC01AC001541C90FBF4F4002CEBD0DC
:1006C000154B1A780AB901221A70154D2B689C42F5
:1006D00004D0144BE1B2187809F030F92C6038BD21
:1006E00011200EF0B9FF0A4B1860D1E7C01AC0EB19
:1006F000C01090FBF2F4E1E70A4B0021187809F0F2
:100700001DF90023064A2370136038BDAC9EFF1FFD
:10071000C09CFF1F3C9DFF1F849FFF1F249FFF1F46
:100720007C9FFF1F149DFF1F38B50F200EF094FF14
:100730001B4A1C4B12881860C0F53B600830904281
:1007400020DB194B1B889842A3EB0204A8BF184674
:10075000801A7F2CC6BFC0010134C0EBC01090FBD3
:10076000F4F47CB1114B1A780AB901221A70104DB9
:100770002B689C4204D00F4BE1B2187809F0DEF8E8
:100780002C6038BD094C237803B938BD094B0021D2
:10079000187809F0D3F80023054A2370136038BD98
:1007A000909DFF1FD89CFF1F109FFF1F349FFF1FAE
:1007B000489DFF1F329DFF1FF0B40E8886420DD268
:1007C00003F10043013B31F81350854202D9F0BCDC
:1007D000FFF71ABF32F81300F0BC70471088F0BC66
:1007E000704700BF094B1B880C2B09D8084A80B200
:1007F00052F8232028B143F6FE73984203D9108C97
:100800007047108870470349FFF7FEBEEE9CFF1F3C
:10081000A43C0100403E01004B4B4C4A2DE9F047FF
:100820001E8814684A4BB442B3F80080494B33DB4E
:100830004445A8BF4446A6421C60C8BF00202DDD29
:10084000C6EB0807B7F5804F33DB80037B1C90FBBA
:10085000F3F0FFF7C7FF404A404B15881B88C0F3F1
:10086000C61909FB05F57F2D8246A8BF7F252BB34E
:10087000A64253DC4445D4BFC6EB0404C6EB0804CF
:100880009F42CCBF03FB04445C43354BC8BF0137D8
:1008900094FBF7F71F6013E034461E60C6EB0807B1
:1008A000A045D4BFC6EB0800C6EB0400B7F5804FE7
:1008B000CBDAC0EB803090FBF7F0CAE7284A136030
:1008C000284C2368994508D0274B1B88002B34D12E
:1008D000264B1B886BBBC4F80090254C23689A45B7
:1008E00006D0214B1B885A1F032A19D9C4F800A02F
:1008F000204C23689D420FD01F4B188848B11A4BDB
:100900001E4A1B88D35C834203D0C0B2E9B209F00F
:1009100015F82560BDE8F087BDE8F0870024AFE753
:10092000164AD05C2030C0B20AF07F0109F006F808
:10093000DCE7484609F0A2F8CDE7104A4946D05C0A
:1009400008F0FCFFC4E700BF8C9DFF1FF49EFF1F53
:10095000569FFF1FB89CFF1FC89CFF1FCA9CFF1F0C
:100960005C9FFF1F2C9DFF1FDA9EFF1F829DFF1FB4
:10097000E89CFF1F849DFF1FEA9EFF1FB889FF1F91
:100980002DE9F04F17208BB00EF066FEDFF850B364
:10099000CBF8000016200EF05FFEB34BB34A1B8865
:1009A00010600C2B00F00582B14A00211F2B117042
:1009B00037D0B04FB04B3A88B04E53F82250002396
:1009C0003370AF4BAF4A1B88AF491288013B012AF5
:1009D00031F91330059300F00682AC4B0193AC4B18
:1009E0000293DFF80083DFF8009300230093A94B04
:1009F0001B88012B00F04D82DFF8F0A2A64B039379
:100A0000DAF80040A54B04930023A54A1288013A66
:100A1000032A00F28682DFE812F00101DC001100F7
:100A20007101A04B934F1B783988934A934E52F82B
:100A30002150003318BF01233370C2E720460593CD
:100A400011F0AEFB984911F0FFFB059B04461846D8
:100A500011F0A6FB954911F0F7FB0146204611F075
:100A6000EBFA11F0B7FD0446CAF80040D8F80000D0
:100A700011F096FB8C4911F0E7FB8246009811F0CB
:100A80008FFB8A4911F0E0FB0146504611F0D4FA81
:100A900011F0A0FDC8F80000854A864BB2F800E0CE
:100AA0001988854BDBF800201B88DFF844C2CEEBA9
:100AB000040804EB0E0AC1EB000E08440499039CE1
:100AC000C1F800A00199C4F80080C1F800E00299C3
:100AD0009A420860BCF8001080F25281C3EB010C0E
:100AE000624865454FF0000E006880F256816C1C2C
:100AF00083420CF1010C0EFB04FE9EFBFCFE00F396
:100B000092838142A8BF0146C91A04FB01F191FBFF
:100B1000FCF19A4200F317818342C0F21481DFF89E
:100B2000D4A1DAF8000011F03BFB644911F08CFB12
:100B3000634911F081FA11F04DFDA0F5FF531C3B04
:100B4000082B98BF4FF40050D9F80040DFF8A88177
:100B5000044443F6FF77BC42A8BF3C4624EAE47451
:100B60002046CAF8004011F01BFB8146307805FB97
:100B700000F011F015FB4FF07A5111F065FB0146C2
:100B8000484611F057FA11F025FD4E4BB842A8BF68
:100B900038461B7820EAE070C8F80000002B00F00F
:100BA000E380B4F5005F00F0DF8005F06BFE464B9C
:100BB000D8F8000001221A70444C2368834205D003
:100BC00080B208F08BFED8F8003023600BB0BDE88F
:100BD000F08F2046059311F0E3FA3D4911F034FB04
:100BE000059B0446184611F0DBFA3A4911F02CFB3C
:100BF0000146204611F020FA11F0ECFC0446CAF838
:100C00000040D8F8000011F0CBFA314911F01CFB7C
:100C10008246009811F0C4FA2E4933E72046059326
:100C200011F0BEFA2C4911F00FFB059B0446184643
:100C300011F0B6FA294911F007FB0146204611F0E0
:100C4000FBF911F0C7FC0446CAF80040D8F80000D0
:100C500011F0A6FA204911F0F7FA8246009811F037
:100C60009FFA1E490EE700BF269FFF1FE49CFF1F4F
:100C7000BE9CFF1F209DFF1F7489FF1F0A9FFF1F3F
:100C80003689FF1FFA9EFF1FE4400100809FFF1F6F
:100C9000589DFF1F889EFF1F189FFF1F8C9EFF1FE0
:100CA0004889FF1FD89EFF1FCDCC4C3FCDCC4C3E7A
:100CB000C489FF1F4089FF1FF09EFF1F9A99193FAB
:100CC000CDCC4C4542A0FF1F809DFF1F3889FF1FE0
:100CD0006666663FCDCCCC3D3333733FCDCC4C3DC7
:100CE0001C9DFF1FB09CFF1F309FFF1F149FFF1F05
:100CF000009DFF1FAC89FF1F4489FF1F20460593FD
:100D000011F04EFAC54911F09FFA059B04461846AA
:100D100011F046FAC24911F097FA0146204611F047
:100D20008BF911F057FC0446CAF80040D8F80000CF
:100D300011F036FAB94911F087FA8246009811F09D
:100D40002FFAB7499EE63B88002B3FF4E8AEC1EB93
:100D50000E03002BB8BF5B42092B00F3E5804FF474
:100D60000050DFF808A3EFE6AE4C2378002B3FF4E9
:100D700023AF05F083FD0023D8F8000023701BE7A4
:100D8000C3EB010CA8488A42D4BFC3EB020EC3EBED
:100D9000010E65450068FFF6AAAE83420EFB05FE14
:100DA000C8BF00249EFBFCFE40F3348294FBFCF1A0
:100DB000AFE69E4B1B78002B00F0D5809C4F9D4BDF
:100DC00039889D4A53F821009C4E0121002311705F
:100DD000337011F0E5F94FF07C5111F035FA11F054
:100DE000F9FB0546EDE5964B964A1B889649127825
:100DF000013B31F91340002A40F0B08011200EF081
:100E00002BFC0090914B0193D3F80090009B9945E7
:100E100040F3AC808E4BDFF858821B888D4A012B43
:100E2000D8F80030B2F800A08B4A02922846A3EB13
:100E3000040400F0CE8011F0B3F9029A52F82A109F
:100E400011F002FA0146002011F0F4F811F0C2FB93
:100E5000009BC9EB04029C42B8BF1C469042C9EB00
:100E6000040480F2CA8000FB0444013294FBF2F4D3
:100E70007A4BDFF800920293D9F80030234403EB59
:100E8000D3735B10C9F80030754B1B88012B7FF4BE
:100E9000B3AD744B03931C460F200EF0DDFB2268AC
:100EA00004929042034680F2E980694A1288012A3E
:100EB00000F02E81674A07901288674C06922846F8
:100EC00011F06EF9069ADFF8B0A154F82210DAF8A2
:100ED000004011F0B9F90146002011F0ABF8059B74
:100EE000E21A059211F076FB059A079B04999A4243
:100EF000C1EB020EB8BF1A46704580F23381521A18
:100F000000FB02220EF1010192FBF1F2D9F8001070
:100F1000554804900A4402EBD2725210C9F80020DE
:100F200073E5D8F80000B7E50EF500500130401A1F
:100F300011F036F93A49DFF834A111F085F9044689
:100F4000DAF8000011F02CF9344911F07DF901466E
:100F5000204611F071F811F03DFBF5E515200CF07D
:100F6000DFFF00904EE7344A137022E53B4B0293BB
:100F7000D3F80090009B994544DA354BDFF8F080B8
:100F80001B88344A012BD8F80030B2F800A0324A4E
:100F9000039228461C4400F0EC8011F001F9039AFA
:100FA00052F82A1011F050F911F014FB009B9C42EA
:100FB000C9EB0402A8BF1C46C9EB04049042BABFA7
:100FC00000FB04440132444394FBF2F4DFF8A490A4
:100FD00052E711F0E5F8029A52F82A1011F034F9AC
:100FE00011F0F8FA009BC9EB04029C42B8BF1C4602
:100FF0008242C9EB04043FF736AF00FB04F494FBD4
:10100000F2F435E7DFF86C90DFF86480D9F800304F
:1010100003EBD3735B10C9F80030E8E49A99193FE9
:10102000CDCCCC3E809DFF1FE49CFF1FD89EFF1FB0
:10103000209DFF1F7489FF1FBE9CFF1F0A9FFF1F7B
:10104000C889FF1FAC9EFF1FF83D0100809FFF1F56
:101050005E9DFF1F089DFF1FFC400100589DFF1F64
:10106000889EFF1F189FFF1F8C9EFF1FAC89FF1FCC
:10107000B09CFF1F309FFF1F149FFF1F6B4A0492FD
:1010800012680692904237DD694A1288012A00F000
:101090008E80684A09901188674A0891284607920D
:1010A00011F07EF8079A0899DFF890A152F8211004
:1010B000DAF8004011F0C8F8059B2344059311F0BD
:1010C00089FA0599099B069A9942C2EB010EA8BFBD
:1010D0001946704580F29080891A00FB01110EF1CB
:1010E000010291FBF2F2D9F800100A4402EBD2722D
:1010F0005210C9F8002088E4D9F80020DFF83CA19C
:1011000002EBD2725210DAF80040C9F800207CE4F9
:10111000484A08901188484A07912846069211F0DB
:101120003FF8069A0799DFF814A152F82110DAF86F
:10113000004011F089F8059BE11A059111F04AFA77
:101140000599089B049A9942C2EB010EB8BF194653
:10115000704558DA891A00FB01110EF1010291FB6A
:10116000F2F2D3E60499521A00FB02F292FBFEF26D
:10117000CCE611F015F8039A52F82A1011F064F831
:101180000146002010F056FF11F024FA009A944214
:10119000C9EB0403A8BF1446C9EB04049842BABFC4
:1011A00000FB04440133444394FBF3F40EE721496C
:1011B000214A089028460C88079210F0F1FF079A00
:1011C000DFF878A052F82410DAF8004011F03CF86B
:1011D0000146002010F02EFF059B2344059311F0DB
:1011E000F9F90599089B069A9942C2EB010EA8BF2E
:1011F00019467045FFF670AF069A891A00FB01F197
:1012000091FBFEF26FE7049A891A00FB01F191FB52
:10121000FEF27BE68842D4BFC3EB0004C3EB0104BB
:1012200005FB04F4C2E519466EE400BF8C9EFF1F67
:101230005E9DFF1F089DFF1FFC400100149FFF1FC4
:1012400008B5244B1B88FBB1234B1B78FBB1234B08
:101250001B78E3B1224B1B78CBB1224B1B78B3B187
:10126000214B22481A78C2B9214A224900881288A3
:1012700009680244B1EB620F09DD01221A70642093
:10128000BDE8084005F012BB174A117801B908BD46
:101290001370BDE8084008F0C5BB154A1649008820
:1012A000128809680244B1EB620FF0DD00221A7067
:1012B00008F0B8FB642005F0F9FA642005F0F6FAAE
:1012C000642005F0F3FA4FF41670BDE808400DF005
:1012D000B1BA00BF9E9EFF1F889FFF1F509FFF1F38
:1012E000519FFF1F529FFF1FEC9CFF1F009DFF1F80
:1012F000F09EFF1F1C9DFF1FE49CFF1F38B5114C83
:10130000232025780CF00CFE0F4A42F82500131F0D
:1013100002F1C400002253F8041F83420A44FAD1A8
:1013200023780A4907480A4C0133DBB2322B81FB90
:10133000025108BF0023D217C2EB211203702260B2
:1013400038BD00BFCC9CFF1F9C9DFF1F1F85EB512C
:10135000EC9EFF1F2DE9F04FB74DB84E2868B84CF2
:1013600083B010F01DFFB74910F06EFF0746102044
:101370000EF072F910F014FFB34910F065FF394612
:1013800010F05AFE11F026F931882860884223882F
:101390007EDA1F4600225B1ADFF8D482DFF8D4E23F
:1013A0007F2BCABFD201C2EBC212013392FBF3F30F
:1013B000B8F80020CEF80030192A00F0DF801A2A91
:1013C00000F02B811E2A00F05B814FF00108C1461E
:1013D0009E4B1B88002B66D09D4A1288032A00F280
:1013E00009818842C0F25F81B842D4BFC1EB0000DE
:1013F000C1EB0700791A8B42B4BF03FB00005843CE
:10140000944F954BB8BF013190FBF1F018603888CC
:1014100000284FD03188D5F800E0884ADFF818A2BC
:10142000714500F38280DFF83CC29CF80030002B4D
:101430004CD14FF0010B04288CF800B046D1B8F124
:10144000000F40F0CB81854B1888F0B1B9F1000F47
:101450001BD02B68318822888B4280F29C8100232C
:10146000541A7E2C7E4DD5BFC3EB8313C3EBC3133D
:101470005B00013493FBF4F42B680134A34203D0E6
:10148000C0B2E1B208F05AFA2C6003B0BDE8F08FA8
:101490009842D4BFC1EB0002C1EB03021F467AE7BA
:1014A00099464FF001081E2A00F0D281694F388812
:1014B0000028AFD1694B1B88002BABD1694A11784A
:1014C0000029E2D0137003B0BDE8F08F012800F0CE
:1014D0001281022800F003810328B4D1624B1B88DB
:1014E000092BB0D0B8F1000FADD02B683788228817
:1014F000BB4280F295810023D71B7E2FDFF86CB1B1
:10150000D5BFC3EB8313C3EBC3135B00013793FB5E
:10151000F7F7DBF800300137BB4203D0F9B24A20BD
:1015200008F00CFACBF800708DE74E4B1A78002AC1
:10153000ABD0002401281C7000F0C280022840F0CB
:101540003181B8F1000F00F0C280484D2B68002BAC
:1015500000F0BD800420214608F0F0F93F4B2C60DC
:101560001888002891D0B9F1000F8ED0C0B20021A8
:1015700008F0E4F93A4B00221A6086E7DFF8F8A099
:10158000DFF8F8909AF80030BBB1DFF8D0E0BEF891
:1015900000E0BEF1000F10D099F800C09C4500F0AB
:1015A00099805FFA8EF07F2108F0C8F99AF8003030
:1015B000B8F8002089F800300FE099F800E09E4567
:1015C00000F08880254B0021187808F0B7F99AF8C8
:1015D0000030B8F8002089F800301C4B1B88002B25
:1015E0003FF45EAF1E2A40F02B814FF001084FF010
:1015F000000951E0884258DBB842A1EB0701A8BFBF
:1016000038468B42A0EB070055DA03FB00004B1C69
:1016100090FBF3F3104A136048E7DFF85CA09AF8F8
:101620000030002B0BBF4FF001084FF000084FF0C7
:1016300000094FF00109CBE6109DFF1FA49EFF1F7C
:10164000A09EFF1F9A99193FCDCCCC3E609FFF1FF3
:101650001C9FFF1F189DFF1F949DFF1F389FFF1F9A
:10166000F49CFF1F2D9FFF1FDA9EFF1F989DFF1FF9
:10167000269FFF1F0C9FFF1FD89EFF1FD29CFF1F9E
:10168000DFF8E8A1744B9AF800801B88B8FA88F854
:101690004FEA58184FF000099AF8002042B3286822
:1016A0003188278898E60020A4E60846C91B8B42AB
:1016B000A0EB0700A9DB03FB00F393FBF1F3A9E721
:1016C000B8F1000F03D0654D2B68002B7FD1644B20
:1016D000188846E74FF001084FF0000978E6B8F1A6
:1016E000000F3FF4B0AEDFF874B1DBF8003030E04B
:1016F0005C4B1A60DAE6B8F1000F3FF4A4AEB4F820
:1017000000A0F245D4BFC1EB0A03C1EB0E03C1EB4D
:101710000A0ABAF17E0FDFF844B1D5BFC3EB8313D9
:10172000C3EBC3135B000AF1010A93FBFAFADBF87F
:1017300000300AF1010A534504D05FFA8AF1012012
:1017400008F0FCF83888CBF800A002287FF4C4AE7B
:1017500053462A68B6F800A02188524559DA00227B
:10176000CAEB010ABAF17E0FD3BFC2EB8212C2EB01
:10177000C2120AF1010A520092FBFAFA0AF1010AB6
:101780009A4504D05FFA8AF1042008F0D7F8388827
:10179000CBF800A0A0E69342D4BFC1EB0303C1EB9A
:1017A00002035DE6032828D12F4B1B88092B8ED01E
:1017B000B8F1000F8BD0294D2B68002B87D04A2021
:1017C000214608F0BBF8264B2C601888C9E6214654
:1017D00008F0B4F8224B2C601888C2E640207F2124
:1017E0008DE80C0008F0AAF8388858459DE80C00F0
:1017F0001DD002287FF470AE75E704287FF467AF30
:10180000B8F1000F3FF463AF2146402008F096F88E
:101810005DE78A42D4BFCAEB0202CAEB01029FE72E
:101820009342D4BFC7EB0303C7EB020364E6DAF8C5
:1018300000E01188B4F800A08E45FFF668AF60E7BD
:101840002868318827884FF001084FF00009C3E568
:101850000023DFF818A01FE7609FFF1F989DFF1F60
:10186000389FFF1F949DFF1FDA9EFF1FD89EFF1F0A
:1018700008B5114B1B88022B09D0052B07D0032B71
:1018800015D0042B0BD00D4B01221A7008BD7F21FF
:10189000412008F053F8094B01221A7008BD7F213E
:1018A000092008F04BF8054B01221A7008BD4021B1
:1018B000092008F043F8E6E7929DFF1F3E9DFF1FB9
:1018C00038B5074B074D1B88052B044606D02B68FF
:1018D000834203D0C1B2052008F030F82C6038BD37
:1018E000929DFF1F3C9FFF1F38B5124D124C2B8855
:1018F000052B12D022684AB9022B0ED0033B012BD4
:1019000013D90E4A00231370236038BD002105202F
:1019100008F014F82B88022B04D10021412008F094
:101920000DF8EEE7052BE9D1F7E70021092008F0D3
:1019300005F8E6E7929DFF1F3C9FFF1F3E9DFF1F9E
:10194000464B1B881D2B70B541D0454D0024454B9F
:101950001B88022B16D0444B1B88022B54D028889E
:10196000424B002C1B780ADB8442A8BF044634B1EA
:10197000002B3AD02046BDE87040FFF7A1BF002BF6
:101980002FD170BD3A4B1B78002B37D015200CF0AF
:10199000C7FA384B1860384A1288002ADBD0374A19
:1019A000186811888142D6DC354B2A881B8883420F
:1019B000A3EB0106A8BF03465B1AB242BABF02FB03
:1019C00003330136534393FBF6F31C44C3E72A4B1E
:1019D0001C888CB12B4B224D1C78002CB7D02C8846
:1019E000B5E7BDE87040FFF77FBFFFF741FF204636
:1019F000BDE87040FFF764BF194DA8E711200DF056
:101A00002BFE1C4B1860C6E70F200DF025FE1A4B6D
:101A10001D4A1B881060002BA1D01C4AC0F53B63F7
:101A2000118808338B429ADB194A2888128893421E
:101A3000A2EB0105A8BF1346A842A3EB010306DAF7
:101A400000FB0333013593FBF5F31C4488E700FBEF
:101A500003F292FBF5F31C4482E700BF269FFF1FB1
:101A60002A9FFF1FFA9EFF1F889EFF1F3E9DFF1F9C
:101A7000AC9EFF1FC09CFF1F929DFF1F3C9DFF1F40
:101A8000249FFF1FD89EFF1FD89CFF1F909DFF1F04
:101A9000109FFF1F38B510200DF0DEFDC830B0F5E7
:101AA000FA7FC0F2EE80B0F57A6F0146A8BF4FF41E
:101AB0007A6101F51673B3F57A6FA8BF4FF47A63B4
:101AC0009BB289B28E4A8F4C11802220238008F06D
:101AD000B7F821888C4D8D4C242008F0B1F80E20E9
:101AE0000CF01EFA40F6FF71C8308842A8BF0846C5
:101AF00020EAE07000F2DC5283B28A42A8BF0A46B4
:101B00000220194622802B8008F09AF821880420B0
:101B100008F096F817200DF09FFD044616200DF0F2
:101B20009BFDA042B8BF204600F1C801B1F5FA7F85
:101B3000C0F2A280B1F57A6FA8BF4FF47A6101F5C7
:101B40004873B3F57A6FA8BF4FF47A639BB289B23A
:101B50006F4A704C11800A20238008F071F82188A8
:101B60000C2008F06DF80F200DF076FDC0F53F61F8
:101B70000431B1F5AF6F7CDBB1F5FA6FA8BF4FF45C
:101B8000FA6189B2644BC0F54360B0F5AF6F19805C
:101B90006CDBB0F5FA6FA8BF4FF4FA6083B25F4C0C
:101BA000A420238008F04CF8A620218808F048F8EB
:101BB0000B200CF009FE002868D011200DF04CFD20
:101BC00000F1C801B1F52F7F6EDA40F214534FF4E3
:101BD0002F71534A1180534C0620238008F030F8AF
:101BE0002188082008F02CF800244FF4AF75E1B2EA
:101BF0004D4809F05DFE01348542A8BF05460C2C16
:101C0000F5D101200DF028FD044600200DF024FD43
:101C1000323CA0F1320345496FF4957000FB03F3A9
:101C200000FB04F081FB034281FB0041DB17C0177E
:101C3000C3EB6223C0EB612003F5AF7200F5AF7315
:101C40009342A8BF13469D42A8BF1D46A5F11401AB
:101C5000312938DC40F26C7332213548354A018035
:101C600013602A20BDE8384007F0EABF4FF4AF63A5
:101C700095E74FF4AF6185E740F214534FF4FA71E2
:101C800066E740F24C434FF4FA711BE715200CF065
:101C900047F900F59671B1F52F7F96DB41F25C2391
:101CA00099421FDD194694E741F25C239942F9DC21
:101CB0001B4A00F5487089B2B0F52F7F118019DA00
:101CC0004FF42F7387E740F23A72A5F5B9751A4BB6
:101CD00002FB05F583FB0523ED17A5EB631389B222
:101CE0003233BAE70E4A00F5617089B2B0F52F7F42
:101CF0001180E5DB8342A8BF03469BB26BE700BFC0
:101D0000A49EFF1FA09EFF1F8C9DFF1F569FFF1FBD
:101D1000F09EFF1F009DFF1F909DFF1F109FFF1F44
:101D20003C9DFF1F249FFF1F7C9DFF1F67BBCF466D
:101D30004E9FFF1FB489FF1FB5814E1B2DE9F04F49
:101D40000C2083B00CF0B8F80C200CF0A5FCC149B5
:101D5000DFF888A314200CF0AFFCBF49BF4809F09E
:101D600077FA022103200CF03DFD022104200CF043
:101D700039FD022105200CF035FD022106200CF072
:101D800031FD01210A200CF02DFD012109200CF06C
:101D900029FD01210D200CF025FD012128200CF04A
:101DA00021FD012114200CF01DFD02210B200CF05F
:101DB00019FD01210C200CF015FD00210C200CF068
:101DC000FDFC012121200CF00DFD02211C200CF056
:101DD00009FD01211B200CF005FD00211B200CF04A
:101DE000EDFC1C200CF0F0FCB0FA80F35B091A202B
:101DF0008AF800300CF036FF1F2000210CF0F8FEAE
:101E000004200CF0E1FC002800F0F08005200CF02C
:101E1000DBFC002800F068810023914C0620237031
:101E20000CF0D2FCB0FA80F35B094FF0000B8D4A46
:101E3000137006F051FA2378002B40F0D2805846F8
:101E400007F028FF884B894A1B88148888498948ED
:101E5000894DA3F5AF7240F23A7303FB02F381FBA5
:101E60000321DB17A3EB61113231062300937B4A78
:101E700001600C235A2181482C7009F081FD002853
:101E800000F039817E4A7F481268DFF854920023BF
:101E90000121FEF709FB0B200CF096FC011E0CBF84
:101EA0000123002389F8003000F0B980764F774D88
:101EB000774EDFF8308200233B602B6033600424D0
:101EC0000F200DF0C9FB336803440E2033600CF083
:101ED00027F83B6899F8002018443860002A79D028
:101EE00015200CF01DF82B681844286004F0010040
:101EF00080F0010004F0CAFCB8F80030002B14BFD9
:101F00004B20DC200CF096FC013CD9D133683968B9
:101F10005D4A28685F4F002BB8BF03330029B8BF64
:101F20000331891011605C495C4A098814889B1050
:101F300000283360B8BF0330594E8210581A194434
:101F40002A6031603860574D57485849161B224463
:101F50002E6002600B60BBF1000F64D1B8F8003056
:101F6000002B4FD0524B012404201C600CF02CFCA1
:101F700018B9504B404A1C7010704F4B1B881C2BDB
:101F800058D04E4C04F1C80523200BF0C9FF44F88B
:101F9000040F01200CF04EFCAC42F5D19AF8003051
:101FA0001BB1474B1B78002B4ED1002121200CF098
:101FB00005FC444A444B1078187007F007FE04F003
:101FC0005DFC4249424845F6BF5203B0BDE8F04FC0
:101FD0000EF058BF11200DF03FFB2B68184428600D
:101FE00084E703B0BDE8F04F09F046B806200CF0D6
:101FF000EBFB00287FF40AAF194C034620704FF02A
:10200000010B14E74FF4FA7004F050FC04F03AFCB2
:1020100006F0BCFC4FF4AF600CF00CFCA2E7112002
:102020000CF0E0FB42E7FFF735FDB8F80030002B7D
:1020300098D1E7E7274B18880028A2D0264BC0B2DA
:10204000197807F07BFC9CE7012121200CF0B6FBFE
:10205000AFE700BF001B374640420F007091FF1FE3
:10206000F29CFF1F909EFF1F4E9FFF1F289FFF1F88
:10207000B5814E1BB489FF1F549DFF1F7C9DFF1F20
:102080003C89FF1FB89EFF1FC49CFF1FB09CFF1F11
:10209000149FFF1F189FFF1FC489FF1F4089FF1F48
:1020A0008C9EFF1F809FFF1F589DFF1F689FFF1F73
:1020B000209FFF1FDD9CFF1F269FFF1F989DFF1F76
:1020C000A69EFF1FA89EFF1F869EFF1FA50500005E
:1020D000449FFF1F5C9DFF1F0C9DFF1F8A9EFF1FDB
:1020E000AC9EFF1FE69EFF1F03200CF06DFBB0FAB5
:1020F00080F35B0991E603200CF066FB0028FAD11F
:1021000004200CF061FB0028F5D105200CF05CFBED
:102110000028F0D106200CF057FB0028EBD10DF081
:10212000BBFB00BF2DE9F04F89B005ADB54F2C4684
:1021300008AE611BC9B2B44809F0BAFB3B888342C0
:1021400094BF0020012004F8010BA642F1D1AF4B4F
:102150009DF814601F889DF81650AD4B9DF818101F
:102160009DF81A001E7073199DF81C20A94CDFF809
:1021700014C3DFF814E325700B440344A64C8CF819
:1021800000101344DFF804C38EF80000012FDFF8BD
:1021900000E38CF80020DBB2237088BF4FF0000C06
:1021A0009E4C98BF4FF0010C8EF800C04FF0000E0F
:1021B00084F800E06AB9002800F07881002900F076
:1021C0008B81042396482370032F00F067822278C6
:1021D00005E0002900F0B580062291482270914B5D
:1021E000DFF8B0A29DF815E09DF81770DFF8A8920F
:1021F000DFF8A8B28C4DDFF8A8828C4E9DF819103C
:10220000027083F800E09DF81B209DF81DE09DF80A
:102210001EC08AF8007001209DF81F70009389F895
:1022200000102A7088F800E08BF800C037700DF0BD
:1022300013FA7F497F4AD1F800E0009B7045CCBF7C
:1022400001210021117040F3AB807B4A1288182ACB
:1022500000F2A68079490F880C3A002F40F0A68042
:10226000774993F800C00B7899F800909AF800101D
:102270009BF8007095F800B02478A3EB4C03A9EB11
:10228000890A5B1A5344C7EB877AC7EB8A07DFF8E2
:10229000B8A11F4498F80030BAF800A007EB4B072C
:1022A00096F800B03B440BFB0A33664F4FF00C0A24
:1022B0001AFB043AC7F800A0B9F1000F0BD033782D
:1022C0004BB1614B1B88042B0CBF0AF1020A0AF1C7
:1022D000040AC7F800A05D4B5D4CDFF8C8B11B884D
:1022E0002488DBF800B05B4F5B4E3F883688033BA9
:1022F000C4EBC4045C4403EB4303DFF8ACB10AEB6A
:1023000083033B44DBF800B0544FC6EBC60657F8D6
:102310002440534F5E440C3B134457F826601A196F
:102320003244BCF1000F12D02B7883B1002940F069
:10233000CF80B9FA89F94B4B4FEA591983F80090CD
:102340000EE0002851D005222270354847E7454B62
:1023500000241C7019B198F80030002B3DD10021E9
:10236000414B70451970C8BF404B4149C8BFC3F8C5
:1023700000A00B689A422CD03E4B3F4C186803904B
:10238000039820601B6804933C4C049B24880A60DB
:102390001B1AA34284BF3A4B1A6009B0BDE8F08F04
:1023A00026490F880022002F3FF45AAF012F00F07A
:1023B000FF80022F00F02981032F00F09080214F31
:1023C0009AF8001093F800C099F80090D7F800A090
:1023D00072E72948274B0068D4E7BCF1000FBED153
:1023E000B9F1000FBBD10121BAE7012FABD9002D04
:1023F00000F03F8116B9012F00F2A680022323705E
:102400000748E1E64E9FFF1F7C9DFF1F729EFF1F46
:10241000509FFF1F519FFF1FF89CFF1F929EFF1FA1
:10242000A29EFF1F859FFF1F899FFF1F2C9FFF1FDD
:10243000B489FF1FD89EFF1F269FFF1FBC9CFF1F54
:10244000C689FF1FE09EFF1F289DFF1FFE9EFF1FE6
:102450001C9FFF1FCE9CFF1F409DFF1F883E010059
:1024600040390100629FFF1F639FFF1F6C9FFF1F8A
:10247000349DFF1F60A0FF1F249DFF1F369FFF1F7D
:10248000749FFF1F529FFF1F539FFF1F549FFF1FEB
:10249000FC9EFF1F869FFF1F879FFF1F889FFF1FB8
:1024A0008A9FFF1F949DFF1F5C9FFF1F00299ED0E6
:1024B000002D00F0DC807D480322974222707FF4DB
:1024C0008EAE0378062B7FF482AE0722227086E65A
:1024D000774B0021197042E7012F88D871E67549C2
:1024E00093F800C00B7899F800909AF800109BF8C8
:1024F000007094F800A02C78A3EB4C03A9EB890B97
:102500005B1A5B444FF0050B1BFB0733009398F8F5
:1025100000300193009BDFF8C4B1C7EBC707BA4492
:102520000533019FBBF800B003EB440334783B4410
:1025300004FB0B33604C614F54F82A400C3303EB1F
:10254000040AC7F800A0B7E658480578012D7FF6C1
:102550003BAE07B125705A4D2D88002D00F09880B4
:10256000002B40F09580574B1B88013B9BB2062BFC
:1025700000F28E80544B1B78002B00F08980534B67
:102580001B68012B7FF420AE514D524B2D68DFF8B4
:1025900050E183FB0536EB17C3EB660303EB430304
:1025A000A5EB8303AEF800304B4B03251D700BE603
:1025B000404993F800C00B7899F800909AF8001001
:1025C0009BF8007095F800A02478A3EB4C03A9EBCE
:1025D000890B5B1A5B44C7EB877BC7EB8B0B3F4FC9
:1025E0005B4498F800B03F8803EB4A0A3378DA443A
:1025F000C4F1060403FB07A3E4B24FF00C0A2F4F0B
:102600001AFB043AC7F800A056E62A4993F800C01E
:102610000B7801932B780093019B9AF8001099F89E
:1026200000909BF800A02478A3EB4C03A9EB890B46
:102630005B1A5B44A3F1020B284BCAEBCA0A544451
:102640001B88DFF8A0A00193BDF800305AF824A041
:1026500098F8004017FB03BB3778019B5C4407FBED
:1026600003431833154F9A44C7F800A024E6012FFE
:1026700006D9002E3FF468AF0C4801232370A3E570
:102680000A480378002B7FF417AF002EF5D19BE5A5
:102690000E4B1B68012B7FF497AD85E700293FF4B3
:1026A00096AD002A7FF493AD0BE700BFA29EFF1FFB
:1026B000629FFF1FC689FF1F44420100E09EFF1F6B
:1026C000089FFF1FAA9EFF1F8E9DFF1F209FFF1FB9
:1026D000749FFF1FABAAAA2AA889FF1F289DFF1F6E
:1026E000E49EFF1FAC4001002DE9F04F3A4B1B78F0
:1026F0008BB0002B6BD10E200BF012FC0FF050FDB5
:1027000001463648364E374DFDF714FF3348FDF786
:10271000E7FE0FF05FFF80F30C003060FFF702FD73
:102720002C68012C7AD0022C00F0CF82032C00F010
:1027300053842D4E2D4C33682D4A2E4E0993099B00
:10274000316812882360591A013A9142274F00F2EA
:10275000B782294E32689A1A092A00F2A082274EBF
:1027600032689A1A0D2A00F29582254E32689A1A1A
:10277000252A1AD9234B1B88002B40F0A481224B19
:102780001B78002B40F09F81FEF7B8FD1F4B1B8884
:102790001B3B9BB2022B04D81D4B1B78002B40F037
:1027A000958104F095F8236833601A4D2A689B1AC6
:1027B000502B00F21482184B1B88012B00F02F8243
:1027C00007F062F806F01CFF0BB0BDE8F08F08F0D0
:1027D000DFFA0BB0BDE8F08FF29CFF1FB89EFF1F21
:1027E000F49EFF1F209FFF1F60A0FF1FB49EFF1FCE
:1027F000B089FF1F889DFF1F6C9DFF1F4C9DFF1F11
:10280000509DFF1F9E9EFF1FEC9CFF1F269FFF1FDA
:10281000D89EFF1F989EFF1FF89EFF1FDFF854935E
:10282000AF4AB9F800001378834204D0C3B2184607
:10283000137007F01BF8DFF84083AA4AB8F800309D
:102840001178994204D0A84F3978002940F0BC870C
:10285000A64A33681288A64E9A42C0F29781A54ACA
:102860001278002A40F09281DFF810A3BAF8003005
:1028700023B9A14B1B88002B00F0AF859F4AA04BCA
:1028800011881B889F4A0B4412685B1093429E4A32
:10289000126880F2288500219342B4BF01230B46C1
:1028A00004910293ACBF4FF0010B8B4605910E20B3
:1028B0000BF036FB954B964A1B6803930133002BB4
:1028C0008446176840F39687802BA8BF8023914ADF
:1028D000914912780191002A00F0628109789142B1
:1028E00000F05E81B8F80010DFF88CE2994201F048
:1028F0006D817D49AEF80030884B4FF0010E81F8B4
:1029000000E01978DFF878E2854B01981B780270B7
:102910008EF80010002B40F04283029B002B40F009
:102920003983A7F252339C4533DA734B1B88002B53
:102930002FD0BBF1000F40F032837A4B1B881BB1C4
:10294000059B002B40F02B83049B13B3764B1A7826
:10295000FAB9DFF8309299F8004001221A70002C81
:1029600040F00885714B1B78002B42F0C884704BF7
:102970001B78002B02F054876E4B1B784BB96E4BC3
:102980001B7833B1B8F8003057490A33A8F8003043
:102990000A700E200BF0C4FA6FF454731F44874280
:1029A00002DC614B00221A7000200CF055FE634AD5
:1029B000634B1168634C1B888842D4BF00220122FC
:1029C0002270002B00F0B9845F4B1C7894426DD0CC
:1029D00088426BDD58490878002800F0B6875B49CB
:1029E00091F800C0BCF1000F40F0AD87584FDFF800
:1029F00098E197F800A0574C574F8EF800C04FF061
:102A0000010E0194039784F800C087F800C081F894
:102A100000E0BAF1000F08D000240C70019F039968
:102A20004FF0010E87F800E00C704049097800294A
:102A300001F06F80494C94F800E0BEF1000F41F0C6
:102A40002081DFF814814FF0010C88F800E084F851
:102A500000C0374C247894B1DFF82CE19EF800C018
:102A6000BCF1000F41F00381DFF8E0904FF0010866
:102A700089F800C08EF80080002901F04F803849A5
:102A8000097899B134480178002941F0F680DFF8DF
:102A9000BCE0344F2F4C8EF800104FF0030E87F837
:102AA00000E02E4F21700124397004701A702E4BF3
:102AB0001B88A3F11B02012A40F274861D2B00F033
:102AC00092862A4C37E6FEF7BBFB5DE6284B1B7867
:102AD000002B3FF466AE2B68012B7FF462AE62E6FA
:102AE000869EFF1F549DFF1FDD9CFF1F8C9DFF1FB7
:102AF00060A0FF1FEC9CFF1F749DFF1F009DFF1F28
:102B0000F09EFF1F1C9DFF1FE49CFF1F6C9FFF1F7B
:102B1000C49CFF1F629FFF1F309DFF1F639FFF1F0D
:102B2000729DFF1FAE9EFF1F919EFF1F859FFF1F7F
:102B3000869FFF1F879FFF1F889FFF1FB489FF1F6E
:102B4000AA9EFF1F069DFF1FB49CFF1FE89EFF1F4C
:102B5000899FFF1F3A9FFF1F8E9DFF1FB59CFF1F80
:102B6000D89EFF1FA889FF1F269FFF1FB49EFF1F2F
:102B70002C9FFF1FA89EFF1F289FFF1F389DFF1F30
:102B8000319DFF1F929EFF1FDC9CFF1F31688E4A04
:102B9000069106988D49106002220B602A6063E658
:102BA0008B49DFF8A0E2097800293FF4ADAE9EF82A
:102BB000000081423FF4A8AE03984B2840F3C98738
:102BC0001833802BB8F80000A8BF802398423FF448
:102BD0009BAE8048038080480123037094E605F093
:102BE000C7FB7E4B1B788BB97D4B1B7873B97D4B34
:102BF0001B785BB97C4B1B7843B97C4B1B782BB99A
:102C00007B4B1B7813B903F039FE01E003F042FE61
:102C100023682B60774B1B88012B7FF4D1AD764B5B
:102C2000764A19681778764EA92303FB01F100292B
:102C3000744BB8BF01F57F511868734BB8BF3F3173
:102C400089132A225439183802FB00111D786FF0BD
:102C5000140202FB071232606C49002D00F04A8119
:102C60000B689A4200F3028480F24481684D287810
:102C7000002840F0EA8767480068D0F17F0048BF2D
:102C80000330801001301B1A9A4200F333810B602D
:102C90001A4630E1FEF754FE2368336065E5FDF720
:102CA0006FFEFEF757FB5C4B1B88032B00F0A585DE
:102CB0005A4B1B88032B00F0A485236833604EE534
:102CC000FDF7AAFD3B68336043E5554A3468128836
:102CD000A24204DB464B1B78002B00F00884514EC7
:102CE000394833680793504B079900681B88091AC5
:102CF000994200F2AD80002B00F0AA804B4B19885E
:102D000000293FF4DEAE314B49481B680088A342DE
:102D1000B8BF23469A4201F3B881464A8342A8BF0E
:102D200003461360DFF8208188F80010354FFDF767
:102D300073FD38687F2840F302863F4B7F3883FB62
:102D40000032C317C3EB620303EB4303A0EB830022
:102D500073303A4B02931B883860002B40F0248775
:102D6000204B01931B78002B00F07084344C2378A7
:102D7000002B00F06B84DFF8D490DFF8BCA04FF09C
:102D8000000B0CE003F17300C0B298F8001006F0DD
:102D900005FE23780BF1010B5B4540F357843B683C
:102DA00059F8040F1844A0F17F038AFB0321DA17B6
:102DB000C2EB610202EB42027F28A3EB8203E1DC5B
:102DC000FDF74AFCE0E700BF449DFF1FB09EFF1FD8
:102DD000639FFF1F289FFF1FDD9CFF1F8E9DFF1F0E
:102DE000E89EFF1F3A9FFF1FB59CFF1FDC9CFF1F43
:102DF000EC9CFF1FF89EFF1FAC89FF1F0A9FFF1F5F
:102E0000649DFF1F749FFF1F3E9DFF1F789DFF1F46
:102E1000409FFF1F3C9FFF1FFA9EFF1F889EFF1FC2
:102E20008C9DFF1F60A0FF1F709DFF1FD49CFF1F84
:102E3000569FFF1FB89CFF1FABAAAA2A169DFF1F13
:102E40007089FF1F319DFF1F609DFF1F4889FF1F75
:102E50008F4B90491B6808888F49A342B8BF23460F
:102E60009A4200F321838D4C09888342A8BF034610
:102E7000236000297FF456AF9A42C8BF0B4640F347
:102E80001A83801AB0F5804FAABF9B03C3EB83332C
:102E9000013093FBF0F0FDF7A5FCC0F3C6100FF076
:102EA0007FF97F4B044618880FF07AF97D49074671
:102EB00020460FF0C9F9014638460FF0C5F9214602
:102EC0000FF0BAF84FF07E5104460FF05BFB00287C
:102ED00041F0D080744920460FF072FB002840F08A
:102EE000C38620460FF09CFBC0B2DFF8108288F842
:102EF00000001BE70A606D4B188858B36C4B2568BF
:102F000053F82040B5FBF4F3772C04FB135300F384
:102F1000C482C3EBC30303EB031393FBF4F36548D1
:102F2000654C50F823002468644BA0F2FF7004FB4A
:102F300000F000F57D3000F5607000EB4004C0EB60
:102F4000C40083FB00430344C017C0EBA3400B380D
:102F500002440A605A495B4B0888198800F27C7069
:102F60004300B3F57C6FA1F164014FEA4100B5BFA6
:102F70005549564903FB02225A4381FB0231114451
:102F8000D317C3EBE123C11881F30C0128200BF008
:102F900085FA15E4BAF80030002B3FF4C2AC4C4B74
:102FA0001B685A1C002A40F3AC81802A00F3A881D8
:102FB000484C494949482488098800682144B0EBB5
:102FC000610FC0F24B86A3F148020F2A3FF6E1AC35
:102FD000473BA9F80030DCE4414BD6F80080198863
:102FE000414540F38F803F4B1B78002B40F08A8097
:102FF000DFF80C9199F800007F2840F31186A3F1C7
:1030000055337F3803F1004383FB0032C317C3EB12
:10301000620303EB4303A0EB83007330324B029354
:103020001B88C0B289F80000002B41F010802F4BA4
:1030300001931B78002B00F09A842D4C2378002BF1
:1030400000F095842B4FDFF8B0804FF0000A0AE0C3
:1030500003F17300C0B206F0C5FC23780AF1010A3F
:10306000534540F3848457F8043F99F8000018440E
:10307000A0F17F0388FB0321DA17C2EB610202EBA8
:1030800042027F28A3EB8203E2DCFDF7E5FAE1E7E9
:10309000B09EFF1F569FFF1FD49CFF1FB89CFF1FB1
:1030A000649FFF1FCDCCCC3D0000FE42D09CFF1F93
:1030B000643E01003C3701000C9FFF1F4D2612812A
:1030C000789FFF1F4C9FFF1F81DFFF8183200882B5
:1030D000E09EFF1FA49EFF1FA09EFF1F109DFF1FCD
:1030E0008C9DFF1FEC9CFF1F169DFF1F3A9FFF1F2B
:1030F0007089FF1F4889FF1FABAAAA2A609DFF1F86
:10310000DC9EFF1FB74F38687F2800F3DB81FDF797
:10311000A3FADFF8489399F80040844200F03B821C
:10312000B14B1B88002B43D1B04AB14812680088CC
:10313000914205DC8242D4BFC1EB0203C1EB000324
:10314000411AB1F5804FA6BF9B030131C3EB833316
:1031500093FBF1F0FDF746FBC0F3C6100FF020F82B
:10316000A44B804618880FF01BF8A34982464046BE
:103170000FF06AF8014650460FF066F841460EF02F
:103180005BFF4FF07E5180460FF0FCF9002840F0C5
:10319000D7869A4940460FF013FA002840F061851F
:1031A00040460FF03DFAC0B2DFF8B48288F8000064
:1031B0007F2C40F3B68392487F3C80FB0430E317BA
:1031C000C3EB600000EB4000A4EB800073308D4B3C
:1031D00001931B78C0B289F80000002B40F01883DF
:1031E000894B04931B78002B40F0FD84874B03939D
:1031F0001B78002B40F04187854B0293039B1B7883
:10320000FBB1844B1B88012B00F0EC85022B00F0F6
:103210009587032B01F0AD81042B01F05E83052B14
:1032200001F04884062B01F09685072B01F02C87CE
:10323000082B02F02980092B02F0F5800A2B02F0FE
:10324000CE82019B1B78002B00F05084029B704CB7
:103250001988002900F0C08438687F2840F3D5829F
:10326000674B7F3883FB0032C317C3EB620303EB6A
:103270004303A0EB830073303860002940F07A8468
:10328000019B1B78002B00F09281634C2378002B6C
:1032900000F08D81DFF8CCA1DFF8C4814FF0000B86
:1032A0000CE003F17300C0B298F8001006F076FB52
:1032B00023780BF1010B5B4540F379813B685AF8A9
:1032C000040F4F4A1844A0F17F0382FB0321DA1751
:1032D000C2EB610202EB42027F28A3EB8203E0DC37
:1032E000FDF7BAF9DFE793424FF0000B80F2F78069
:1032F0000123CDF808B0CDF814B00493FFF7D7BA86
:1033000080244649464B474A09881B8812680B446B
:10331000B2EB630FBFF63DAB434B1B78002B40F085
:10332000A983B8F80030414AA3423FF432AB404B86
:10333000148001221A70FFF72CBB344F3D4C3148EA
:1033400031493D4A3B70237003700B701370FFF7D7
:10335000AEBB3A4B1B78002B7FF41BAB039B384A68
:10336000243B83F34703D9B25B20136006F0E6FAEF
:1033700099F80040032C30D1DFF8EC8098F8003049
:10338000002B42F01B832F4F3B78002B42F0098328
:103390002A4C2378002B42F0F7822B4B1B78002B12
:1033A00042F0E582294A1380294B1B78002B42F01A
:1033B000D1820D4B7F221A8098F800306BB93B7890
:1033C0005BB923784BB9234A7F210720138006F08D
:1033D000B5FA7F210B2006F0B1FA1F4B1F68FFF7EB
:1033E000D8BA00BF749FFF1FD49CFF1FB89CFF1F5B
:1033F000569FFF1F649FFF1FCDCCCC3D0000FE42B7
:10340000ABAAAA2A3A9FFF1FB59CFF1F8E9DFF1FE4
:10341000169DFF1FAA9EFF1F7089FF1FA09EFF1F02
:10342000A49EFF1F109DFF1FD89EFF1F289FFF1FF8
:10343000DD9CFF1FE89EFF1FDC9CFF1F889FFF1F76
:10344000FC9CFF1F879FFF1F869FFF1F829DFF1F02
:10345000899FFF1FDA9EFF1FC49CFF1FDC9EFF1F7A
:10346000609DFF1F4889FF1F859FFF1FB94D28786A
:10347000002840F00E83B8480068D0F17F0048BFB4
:10348000033003EBA0030133B4480B609A42B8BF8A
:103490000260FFF630AD1A462DE5C3EB0313D800EA
:1034A000631C90FBF3F33AE5AD4B09881A600029E1
:1034B0007FF438AC13469842D4BFC2EB0003C2EB92
:1034C0000303DEE4A74B7F3883FB0032C317C3EB53
:1034D000620303EB4303A0EB8300733019E601237F
:1034E000CDF810B0CDF808B00593FFF7E0B901238F
:1034F0002B609D4E9D4CFFF71EB9039B1B78FBB1C3
:103500009B4B1B88012B00F0C283022B00F094869A
:10351000032B00F0B587042B01F0BB81052B01F0D4
:103520005482062B01F00F84072B01F0F984082B3D
:1035300001F06486092B01F0DC870A2B02F002817E
:10354000029B1B88002B00F01E83019B1B783BB95C
:10355000049B1B7823B9039B1B78002B00F0778713
:10356000844B1B78002B00F02D8183490B78082BAE
:1035700000F2288181483A680068814C0133DBB24F
:103580005F1E101A44F827000B707E4BD6F800809F
:10359000198889F800208845734E7FF792AA32680F
:1035A000794B0892089A714C1A60FFF7C4B8049BD3
:1035B0001B78002BA1D03B68A3F10C007F2840F3BF
:1035C0001B8368488B3B80FB0320DA17C2EB60004B
:1035D00000EB4000A3EB800303F17300DFF8BC8134
:1035E000C0B298F8001006F0D9F9019B1B78002BA7
:1035F00083D0614C2378002B3FF47FAFDFF8A0A18C
:103600004FF0000B0CE003F17300C0B298F800100B
:1036100006F0C4F923780BF1010B5B457FF76DAF22
:103620003B685AF8040F4F4A1844A0F18B0382FB01
:103630000321DA17C2EB61020C3802EB42027F2849
:10364000A3EB8203DFDCFDF707F8DEE7494B1B78CD
:10365000002B40F09E824D4B1B78002B45D03B68E1
:10366000A3F10C007F2840F3D8823E4A8B3B82FBBB
:103670000321DA17C2EB610202EB4202A3EB8203E1
:1036800003F17300C0B298F8001006F087F9019BAF
:103690001B7853B3384C23783BB3DFF80491DFF841
:1036A000C4A04FF0000B0BE003F17300C0B298F818
:1036B000001006F073F923780BF1010B5B4514DD64
:1036C0003B6859F8040F1844A0F18B038AFB0321CF
:1036D000DA17C2EB61020C3802EB42027F28A3EB3F
:1036E0008203E1DCFCF7B8FFE0E7294B1B78FBB174
:1036F0001F4B1B88012B00F02684022B00F01D8637
:10370000032B00F0AC87042B01F00C81052B01F09A
:103710003B82062B01F03583072B01F05B83082BDE
:1037200001F00586092B01F09F860A2B01F0B9876D
:10373000029B1B88002B00F04382164B1B78002B4A
:1037400040F03982144B3A681A7003232B60FFF75C
:10375000B8B900BF409FFF1F3C9FFF1F789DFF1F10
:10376000B89CFF1FABAAAA2A60A0FF1FB49EFF1F30
:10377000AA9EFF1FE89EFF1F7089FF1FE09CFF1F8E
:103780004C89FF1F8C9DFF1F20A0FF1FB59CFF1FB2
:103790008E9DFF1FDC9CFF1FDC9EFF1F609DFF1F97
:1037A0004889FF1FDFF8108398F80030002B40F0A5
:1037B000BC80BC4F3B78002B40F06E84BA4C3B7011
:1037C000FEF7B9BF3A68E0E6DBB21846137006F0C0
:1037D00073F9B649B648B74A00230B703B700370C3
:1037E0001370FFF735B8B44AAE4B12781A70AE4C6E
:1037F000FEF7A1BF0123FFF76AB8FCF73FFFFFF711
:1038000057BAFCF791FFFFF758BAFCF725FF33E5ED
:10381000AA4B02931B8863BBA64B0493A84B03934C
:10382000A84C23787BB3DFF8AC82DFF89CA24FF082
:10383000000B09E003F17300C0B206F0D3F823785F
:103840000BF1010B5B451EDD58F8043F99F80000B1
:103850001844A0F17F038AFB0321DA17C2EB61024F
:1038600002EB42027F28A3EB8203E3DCFCF7F4FEC9
:10387000E2E7904B0493924B039306F0B3F8019B5D
:103880001B78002BCCD1049B1B78002B3FF4B6ACEB
:1038900099F80030A3F10C007F2840F3BB818A48DF
:1038A0008B3B80FB0320DA17C2EB600000EB40008B
:1038B000A3EB800303F17300C0B206F093F8019B01
:1038C0001B78002B00F09B817E4C2378002B01F0AD
:1038D0006882DFF80082DFF8F0A14FF0000B0AE009
:1038E00003F17300C0B206F07DF823780BF1010BF1
:1038F0005B457FF783AC58F8043F99F80000184403
:10390000A0F18B038AFB0321DA17C2EB61020C38AA
:1039100002EB42027F28A3EB8203E1DCFCF79CFE72
:10392000E0E72046FCF798FE51E4684A1278002A46
:1039300040F0DA825B4F5C4C3B70FEF7FCBEFCF75C
:103940008BFEFFF706BA00240C70614991F800A0C5
:10395000BAF1000F3FF469A855490191097800298F
:1039600000F07085019C00212170FFF75EB8514B7B
:103970001B78002B42D099F80030A3F10C007F286F
:1039800040F39883504A8B3B82FB0321DA17C2EB4A
:10399000610202EB4202A3EB820303F17300C0B2A7
:1039A00006F020F8019B1B7843B3464C23782BB3D9
:1039B000484FDFF814814FF0000A09E003F173006B
:1039C000C0B206F00FF823780AF1010A534515DD5D
:1039D00057F8043F99F800001844A0F18B0388FBC6
:1039E0000321DA17C2EB61020C3802EB42027F2896
:1039F000A3EB8203E2DCFCF72FFEE1E7304B1B7800
:103A0000FBB1354B1B88012B00F0B686022B00F072
:103A1000B687032B01F01B81042B01F0A581052B38
:103A200001F0D183062B01F0EB84072B01F0988580
:103A3000082B01F00887092B01F069870A2B01F098
:103A40004387029B1B88002B00F00F83174B1B78CA
:103A5000002B40F00583214B1B78002B40F0FB82AC
:103A60001F4B204A1988D6F80080002001231060DF
:103A70002B6090E54B2C40F3D7801834802CB8F89D
:103A80000030194AA8BF8024A3427FF450ACFEF74F
:103A900080BF0130C0B2022836D828701A46FFF71E
:103AA0002ABA00BFD29CFF1FB49EFF1FE89EFF1FD3
:103AB0003A9FFF1FB59CFF1FD89EFF1F169DFF1F3B
:103AC0008E9DFF1F7089FF1FABAAAA2A2C9FFF1F84
:103AD000899FFF1F4889FF1FAA9EFF1FDC9CFF1FB5
:103AE0008C9DFF1FB89CFF1F289FFF1F049B1B7806
:103AF000002B7FF4ABAB039B1B78002B7FF4A6ABB2
:103B0000029B1988FFF7A8BB00222A701A46FFF70C
:103B1000F2B9A24C2478002C7EF49EAF00287EF4EB
:103B2000AEAFBAF1000F7EF4AAAF002C7EF4A7AFBF
:103B30009B49097800297EF4A5AF9A489A490470F8
:103B40000C709A4F9A489B493C7004700C70FEF7B9
:103B5000ADBF243B002BB8F8000040F36D849842C1
:103B60003EF4D2AE9BB29448A8F800300123037013
:103B7000FEF7CABEDFF84482C0B298F8001005F024
:103B80000DFFFFF77DBB8D4B3878197805F006FFE8
:103B9000DBE47F21402005F0D1FE894A894B39685A
:103BA000116000221A7056E5C0B298F8001005F0B6
:103BB000F5FEFFF7D5B87F21422005F0BFFEC1E535
:103BC00098F80010387805F0E9FEB6E57E4BDFF88E
:103BD00008E21978FEF798BE99F8000005F002FF98
:103BE0002188FFF739BB794B02931B88002B41F0EA
:103BF0002A876F4B03934BE6FCF72EFDEEE4039B05
:103C00001B78002B7FF4FDAA049B1B78002B7FF40C
:103C10001DAB75E7FCF720FD4EE6FCF71DFD31E519
:103C2000FCF71AFDFFF7FAB9243C002CB8F8003075
:103C300040F31A86A3423EF4ACAEA4B25E4BA8F8A1
:103C4000004001221A70FEF7A4BE421CD2B2022A22
:103C50003FF65AAF2A701A46FFF74DB91446FFF7E0
:103C60005BBB7F20FFF7A0BA7F20FFF73EB94FF084
:103C7000000C8EF800C0FEF7FFBE00210170FEF7B9
:103C800015BF4FF0000E84F800E0FEF7E2BEDFF84B
:103C90004CA13868BAF800304D4A4E4CC31A82FB2A
:103CA000031ED917C1EB6E0101EB4101A3EB8103A8
:103CB00003EB430354F8233018447F2840F3468530
:103CC0007F3882FB0032C317C3EB620303EB43036D
:103CD000A0EB83007330DFF8E480DFF804B198F8DC
:103CE0000010C0B205F05AFEBBF80030022B7FF680
:103CF00027AC3968BAF80030354ACB1A82FB030E7C
:103D0000D817C0EB6E0000EB4000A3EB800303EB81
:103D1000430304EB8303586808447F2840F330874B
:103D20007F3882FB0032C317C3EB620202EB420210
:103D3000A0EB82007330C0B298F8001005F02EFEA0
:103D4000BBF80030032B7FF6FBAB3968BAF80030C4
:103D50001F4ACB1A82FB030ED817C0EB6E0000EB94
:103D60004000A3EB800303EB430304EB8304A06850
:103D700008447F2840F3A8817F3882FB0032C317B4
:103D8000C3EB620202EB4202A0EB8200733098F8B0
:103D90000010C0B205F002FEFFF7D2BB869FFF1FE6
:103DA000D89EFF1FE89EFF1F3A9FFF1FB59CFF1F75
:103DB0008E9DFF1FDC9CFF1FDD9CFF1F609DFF1F72
:103DC000E09CFF1F7089FF1F639FFF1F169DFF1F51
:103DD000ABAAAA2A683D0100319DFF1FE49EFF1F88
:103DE000F09CFF1FDFF848A399F80000BAF80030F4
:103DF000C54AC64CC31A82FB031ED917C1EB6E011C
:103E000001EB4101A3EB810303EB430354F823309F
:103E100018447F2840F39E847F3882FB0032C3170A
:103E2000C3EB620303EB4303A0EB83007330DFF8C3
:103E300004B3C0B205F0D6FDBBF80030022B7FF60C
:103E400000AA99F80010BAF80030AF4ACB1A82FBEA
:103E5000030ED817C0EB6E0000EB4000A3EB80030D
:103E600003EB430304EB8303586808447F2840F3C3
:103E700083867F3882FB0032C317C3EB620202EBFA
:103E80004202A0EB82007330C0B205F0ABFDBBF87C
:103E90000030032B7FF6D5A999F80010BAF800304E
:103EA000994ACB1A82FB030ED817C0EB6E0000EBC9
:103EB0004000A3EB800303EB430304EB8304A068FF
:103EC00008447F2840F3E5807F3882FB0032C31727
:103ED000C3EB620202EB4202A0EB82007330C0B27D
:103EE00005F080FDFFF7ADB9894F387802F040FD4D
:103EF000884B1B78002B00F0EA803B887E2B00F279
:103F0000E680854CDFF830922268D9F80010521A0A
:103F10000F2A40F2D380814A0133108899B2398048
:103F2000002800F0ED80C9B2C0B205F007FD7C4F5B
:103F3000226898F80030C9F800203B70FEF7FBBB00
:103F40000120FFF731B9DFF8E8A13868BAF800308E
:103F50006D4A6E4CC31A82FB031ED917C1EB6E016A
:103F600001EB4101A3EB810303EB430354F823303E
:103F700018447F2840F3F2837F3882FB0032C31756
:103F8000C3EB620303EB4303A0EB83007330DFF862
:103F9000A4B198F80010C0B205F000FDBBF80030E5
:103FA000022B7FF6C5AB3968BAF80030564ACB1AF7
:103FB00082FB030ED817C0EB6E0000EB4000A3EBB2
:103FC000800303EB430304EB8303586808447F2812
:103FD00040F39F867F3882FB0032C317C3EB620237
:103FE00002EB4202A0EB82007330C0B298F80010DE
:103FF00005F0D4FCBBF80030032B7FF699AB386892
:10400000BAF80030404AC31A82FB031ED917C1EB2D
:104010006E0101EB4101A3EB810303EB430304EBCE
:104020008304A36818447F2841DD7F3882FB003277
:10403000C317C3EB620202EB4202A0EB82007330B3
:10404000C0B298F8001005F0A9FCFFF771BB05F0AD
:10405000C9FCFEF7ECBF0021422005F06FFCFFE435
:104060000021402005F06AFCF5E499F8000005F015
:10407000B9FCEBE40120FEF738BF2A4B02931B8802
:10408000002B3FF4BBA8FFF7F8BB274B1A60FEF7E5
:1040900049BEFCF7E1FA22E71D4B1F4C19886A2044
:1040A00005F0CEFD98F800303B70FEF744BBFCF7FE
:1040B000D3FAC5E7FCF7D0FA71E4174C184F98F81B
:1040C00000303B70FEF737BBFCF7C6FA5FE6174BD4
:1040D0001B78002BF1D03B880D4F002BEDD00E4C00
:1040E000DFF854902268D9F80010521A0F2AE5D947
:1040F0000A4A013B108899B2398000287FF413AF37
:10410000C8B205F0BBFC12E7ABAAAA2A683D0100C1
:104110000C9DFF1F8A9FFF1FB49EFF1F5C9DFF1F0A
:10412000D29CFF1F169DFF1FB89CFF1F899FFF1F7A
:10413000E49EFF1FF09CFF1F709FFF1FDFF834A35A
:1041400099F80000BAF80030C64AC74CC31A82FB7F
:10415000031ED917C1EB6E0101EB4101A3EB8103F3
:1041600003EB430354F8233018447F2840F3FE83C5
:104170007F3882FB0032C317C3EB620303EB4303B8
:10418000A0EB83007330DFF8F0B2C0B205F02AFC78
:10419000BBF80030022B7FF654A899F80010BAF84B
:1041A0000030B04ACB1A82FB030ED817C0EB6E006A
:1041B00000EB4000A3EB800303EB430304EB83031A
:1041C000586808447F2840F3D8857F3882FB003246
:1041D000C317C3EB620303EB4303A0EB830073300D
:1041E000C0B205F0FFFBBBF80030032B7FF629A817
:1041F00099F80010BAF800309A4ACB1A82FB030EE5
:10420000D817C0EB6E0000EB4000A3EB800303EB7C
:10421000430304EB8304A06808447F287FF739AF89
:104220007F3882FB0032C317C3EB620303EB430307
:10423000A0EB8300733052E6DFF838A23868BAF892
:104240000030884A884CC31A82FB031ED917C1EB81
:104250006E0101EB4101A3EB810303EB430354F82F
:10426000233018447F2840F384837F3882FB003258
:10427000C317C3EB620303EB4303A0EB830073306C
:10428000DFF8F881DFF8F0B198F80010C0B205F05F
:1042900085FBBBF80030022B7FF652A93968BAF8CB
:1042A0000030704ACB1A82FB030ED817C0EB6E00A9
:1042B00000EB4000A3EB800303EB430304EB830319
:1042C000586808447F2840F364857F3882FB0032B9
:1042D000C317C3EB620303EB4303A0EB830073300C
:1042E000C0B298F8001005F059FBBBF80030032B62
:1042F0007FF626A93868BAF800305A4AC31A82FBFA
:10430000031ED917C1EB6E0101EB4101A3EB810341
:1043100003EB430304EB8304A36818447F287FF76F
:10432000D3AE7F3882FB0032C317C3EB620303EBCB
:104330004303A0EB8300733029E5DFF838A1386828
:10434000BAF80030474A484CC31A82FB031ED917FB
:10435000C1EB6E0101EB4101A3EB810303EB4303CE
:1043600054F8233018447F2840F306837F3882FBBB
:104370000032C317C3EB620303EB4303A0EB8300DC
:104380007330DFF8F4B098F80010C0B205F006FB07
:10439000BBF80030022B7FF6CBA93968BAF80030A1
:1043A000304ACB1A82FB030ED817C0EB6E0000EB2D
:1043B0004000A3EB800303EB430304EB8303586843
:1043C00008447F2840F3E9847F3882FB0032C3171A
:1043D000C3EB620303EB4303A0EB83007330C0B273
:1043E00098F8001005F0DAFABBF80030032B7FF6DE
:1043F0009FA93868BAF800301A4AC31A82FB031E14
:10440000D917C1EB6E0101EB4101A3EB810303EB73
:10441000430304EB8304A36818447F287FF747AE67
:104420007F3882FB0032C317C3EB620303EB430305
:10443000A0EB8300733003E601283EF465AA012354
:10444000FFF791BB094C0A490394FEF7E5BA4FF414
:104450007A43013BFDD199F8000005F0C3FAFFF75C
:104460007FB800BFABAAAA2A683F01008E9DFF1F3C
:10447000E89EFF1FE49EFF1FF09CFF1F609DFF1F33
:10448000DFF8E8A23868BAF80030B64AB64CC31A6A
:1044900082FB031ED917C1EB6E0101EB4101A3EBB7
:1044A000810303EB430354F8233018447F2840F37F
:1044B000E7817F3882FB0032C317C3EB620202EB55
:1044C0004202A0EB82007330DFF8A482DFF8A4B2CE
:1044D00098F80010C0B205F061FABBF80030022B6A
:1044E0007FF62EA83868BAF800309E4AC31A82FBBD
:1044F0000321DA17C2EB610202EB4202A3EB820353
:1045000003EB430304EB83035B6818447F2840F309
:1045100010847F380C2290FBF2F302FB13007330FF
:10452000C0B298F8001005F039FABBF80030032B40
:104530007FF606A83868BAF800308A4AC31A82FBA8
:104540000321DA17C2EB610202EB4202A3EB820302
:1045500003EB430304EB8304A36818447F287FF72D
:10456000B3AD7F380C2290FBF2F302FB13007330E3
:104570000DE4DFF8F8A199F80000BAF80030794AA4
:10458000794CC31A82FB031ED917C1EB6E0101EBF4
:104590004101A3EB810303EB430354F82330184498
:1045A0007F2840F367817F3882FB0032C317C3EB5B
:1045B000620202EB4202A0EB82007330DFF8B4B17A
:1045C000C0B205F00FFABBF80030022B7EF639AE10
:1045D00099F80000BAF80030624AC31A82FB03213E
:1045E000DA17C2EB610202EB4202A3EB820303EB98
:1045F000430304EB83035B6818447F2840F39083F4
:104600007F380C2290FBF2F302FB13007330C0B230
:1046100005F0E8F9BBF80030032B7EF612AE99F8EE
:104620000000BAF800304F4AC31A82FB0321DA17A0
:10463000C2EB610202EB4202A3EB820303EB4303F2
:1046400004EB8304A36818447F287FF722AD7F38EA
:104650000C2290FBF2F302FB130073303FE4DFF80F
:104660000CA13868BAF800303E4A3F4CC31A82FBAE
:10467000031ED917C1EB6E0101EB4101A3EB8103CE
:1046800003EB430354F8233018447F2840F3F580AC
:104690007F3882FB0032C317C3EB620202EB420297
:1046A000A0EB82007330DFF8CCB098F80010C0B2F5
:1046B00005F074F9BBF80030022B7FF639A8386892
:1046C000BAF80030274AC31A82FB0321DA17C2EB7B
:1046D000610202EB4202A3EB820303EB430304EB10
:1046E00083035B6818447F2840F32A837F380C22B9
:1046F00090FBF2F302FB13007330C0B298F8001085
:1047000005F04CF9BBF80030032B7FF611A8386890
:10471000BAF80030134AC31A82FB0321DA17C2EB3E
:10472000610202EB4202A3EB820303EB430304EBBF
:104730008304A36818447F287FF7B9AC7F380C2224
:1047400090FBF2F302FB1300733079E4FBF784FF74
:10475000FFF7C1BAFBF780FFFFF769BBFBF77CFFF0
:1047600015E400BFABAAAA2AF83F0100E49EFF1F90
:10477000609DFF1FF09CFF1FDFF82CA399F800003D
:10478000BAF80030C34AC44CC31A82FB0317D917C6
:10479000C1EB670101EB4101A3EB810303EB430391
:1047A00054F8233018447F2870DD7F3882FB0032B4
:1047B000C317C3EB620202EB4202A0EB820073302C
:1047C000DFF8E8B2C0B205F00DF9BBF80030022BFB
:1047D0007FF637A999F80000BAF80030AD4AC31A3D
:1047E00082FB0321DA17C2EB610202EB4202A3EB68
:1047F000820303EB430304EB83035B6818447F28C5
:1048000040F39B827F380C2290FBF2F302FB1300F3
:104810007330C0B205F0E6F8BBF80030032B7FF62A
:1048200010A999F80000BAF800309A4AC31A82FB1E
:104830000321DA17C2EB610202EB4202A3EB82030F
:1048400003EB430304EB8304A36818447F281ADDB9
:104850007F380C2290FBF2F302FB13007330C0B2DE
:1048600005F0C0F8FFF7EDB8012B3EF492A8012443
:10487000FFF7E4B9FBF7F0FEA0E6FBF7EDFE12E769
:10488000FBF7EAFE20E6FBF7E7FEE8E7FBF7E4FECE
:1048900096E7DFF814A23868BAF800307D4A7F4CFA
:1048A000C31A82FB031ED917C1EB6E0101EB410154
:1048B000A3EB810303EB430354F8233018447F2810
:1048C000DEDD7F3882FB0032C317C3EB620303EBEC
:1048D0004303A0EB83007330F6E5DFF8CCA199F831
:1048E0000000BAF800306B4A6C4CC31A82FB031EFE
:1048F000D917C1EB6E0101EB4101A3EB810303EB7F
:10490000430354F8233018447F28B3DD7F3882FBFB
:104910000032C317C3EB620303EB4303A0EB830036
:1049200073304BE6DFF880A13868BAF80030594A96
:104930005A4CC31A82FB031ED917C1EB6E0101EB5F
:104940004101A3EB810303EB430354F823301844E4
:104950007F2892DD7F3882FB0032C317C3EB6203EE
:1049600003EB4303A0EB830073309CE6FBF774FE7C
:1049700009E4FBF771FE83E4FBF76EFE01E5DFF867
:1049800028A199F80000BAF80030424A444CC31AF2
:1049900082FB0317D917C1EB670101EB4101A3EBC0
:1049A000810303EB430354F8233018447F287FF737
:1049B0006DAF7F3882FB0032C317C3EB620303EB9A
:1049C0004303A0EB83007330FAE6DFF8DCA038681D
:1049D000BAF800302F4A334CC31A82FB0321DA178E
:1049E000C2EB610202EB4202A3EB820303EB43033F
:1049F00054F8233018447F2840F398817F380C22E4
:104A000090FBF2F302FB13007330DFF8A480DFF8B1
:104A10009CB098F80010C0B204F0C0FFBBF80030A2
:104A2000022B1AD93868BAF800300C22C11A91FB4F
:104A3000F2F302FB131302FB03435B6818447F2865
:104A400040F353847F3890FBF2F302FB1300733082
:104A5000C0B298F8001004F0A1FFBBF80030032B9F
:104A60007EF66EADBAF8003038680C22C11A91FBA0
:104A7000F2F302FB131302FB0344A36818447F28DC
:104A80007FF722AB7F3890FBF2F302FB1300733009
:104A9000FFF77DB9ABAAAA2A683D0100D43901000D
:104AA000683F01007C420100E49EFF1FF09CFF1F55
:104AB000609DFF1FDFF814A399F80000BAF80030DA
:104AC000BD4ABE4CC31A82FB0321DA17C2EB610256
:104AD00002EB4202A3EB820303EB430354F82330BF
:104AE00018447F2840F319817F380C2290FBF2F3A1
:104AF00002FB13007330DFF8D8B2C0B204F072FFCB
:104B0000BBF80030022B19D999F80000BAF8003030
:104B10000C22C11A91FBF2F302FB131302FB0343B5
:104B20005B6818447F2840F3E7837F3890FBF2F3FB
:104B300002FB13007330C0B204F054FFBBF8003026
:104B4000032B7EF67EABBAF8003099F800000C22F9
:104B5000C11A91FBF2F302FB131302FB0344A36897
:104B600018447F287FF795AA7F3890FBF2F302FB69
:104B700013007330FFF7B3B9FBF76EFDFFF784B98D
:104B8000FBF76AFDFFF7D7B8DFF840A23868BAF83C
:104B90000030894A894CC31A82FB0321DA17C2EB21
:104BA000610202EB4202A3EB820303EB430354F8DE
:104BB000233018447F2840F3B6807F380C2290FBC6
:104BC000F2F302FB13007330DFF804B298F8001020
:104BD000C0B204F0E3FEBBF80030022B1AD93868EB
:104BE000BAF800300C22C11A91FBF2F302FB131346
:104BF00002FB03435B6818447F2840F37A837F38C5
:104C000090FBF2F302FB13007330C0B298F800106F
:104C100004F0C4FEBBF80030032B7EF689ADBAF871
:104C2000003038680C22C11A91FBF2F302FB131317
:104C300002FB0344A36818447F287FF738AA7F3813
:104C400090FBF2F302FB13007330FFF7F9B9DFF8C2
:104C50007CA199F80000BAF80030574A584CC31AA2
:104C600082FB0321DA17C2EB610202EB4202A3EBE3
:104C7000820303EB430354F8233018447F2845DDB7
:104C80007F380C2290FBF2F302FB13007330DFF845
:104C900040B1C0B204F0A6FEBBF80030022B18D918
:104CA00099F80000BAF800300C22C11A91FBF2F317
:104CB00002FB131302FB03435B6818447F2877DD74
:104CC0007F3890FBF2F302FB13007330C0B204F0A4
:104CD00089FEBBF80030032B7EF6B3AEBAF8003085
:104CE00099F800000C22C11A91FBF2F302FB131396
:104CF00002FB0344A36818447F287FF7C4AD7F38C4
:104D000090FBF2F302FB13007330A8E5FBF7A4FC61
:104D1000BDE7FBF7A1FCFFF768B9FBF79DFCEAE6EE
:104D2000FBF79AFC73E4FBF797FC4DE7FBF794FC69
:104D30006BE6FBF791FCFFF7F3BBFBF78DFC68E537
:104D4000FBF78AFCD9E4DFF884A03868BAF80030B1
:104D5000194A1C4C40E6DFF874A099F80000BAF834
:104D60000030154A174CADE6DFF860A099F8000056
:104D7000BAF80030104A144C71E7FBF76DFCFFF7EE
:104D80002FBADFF848A03868BAF800300A4A0D4C4C
:104D900001E7FBF761FCFFF7A3BAFBF75DFCFFF748
:104DA0001EBB039B1B78002B7EF42BAAFEF74EBA8A
:104DB000FBF752FC8AE700BFABAAAA2A7C4201009B
:104DC000F83F010024410100D4390100E49EFF1F97
:104DD000F09CFF1FA54C2388002B00F08783A44A7A
:104DE000DFF8A0B21288BBF800100332914228DD30
:104DF000A0493868A04A0988B2F800E0DFF87CC210
:104E0000411A0C2291FBF2F902FB19114FF09009A3
:104E100009FB0EFE02FB01E16FF00B0E5CF80110C6
:104E200001440EFB03107F2840F337847F3890FB4A
:104E3000F2F302FB13007330C0B298F8001004F0D4
:104E4000ADFDBBF8002023881344022B23DD894BE2
:104E5000894A38681B88B2F800C0DFF820E2C31A1C
:104E60000C2193FBF1F201FB1232902303FB0CF3B4
:104E700001FB023373445B6818447F2840F3C38509
:104E80007F3890FBF1F301FB13007330C0B298F848
:104E9000001004F083FDBBF8002023881344032B8B
:104EA00023DD744B744A38681B88B2F800C0DFF801
:104EB000CCE1C31A0C2193FBF1F201FB12329023D7
:104EC00003FB0CF301FB023373449B6818447F28F7
:104ED00040F39D857F3890FBF1F301FB13007330A5
:104EE000C0B298F8001004F059FDBBF800202388E8
:104EF0001344042B7EF71CAC5D4B1B88012B7EF406
:104F000017AC3A68A2F10C007F287FF7D0A88B3A43
:104F10000C2092FBF0F300FB13207330FFF790B8E6
:104F2000524C2388002B40F0D682DFF858B151490B
:104F3000514A0988D7F80080B2F800E04F48C1EB29
:104F4000080C0C229CFBF2F102FB11C14FF0900CFB
:104F50000CFB0EFE02FB01E16FF00B0E405880448B
:104F60000EFB03807F2840F39583A0F17F0393FB22
:104F7000F2F002FB10307330414BC0B2197804F0EC
:104F80000DFDBBF8002023881344022B23DD394A92
:104F9000394B11883868B3F800C0DFF8E0E0411AF7
:104FA0000C2291FBF2F302FB1311902303FB0CF391
:104FB00002FB013373445B6818447F2840F3748418
:104FC0007F3890FBF2F302FB130073302C4BC0B21E
:104FD000197804F0E3FCBBF8002023881344032B6A
:104FE00023DD244A244B11883868B3F800C0DFF869
:104FF0008CE0411A0C2291FBF2F302FB1311902377
:1050000003FB0CF302FB013373449B6818447F28B5
:1050100040F3E3847F3890FBF2F302FB130073301C
:10502000174BC0B2197804F0B9FCBBF800202388F4
:105030001344042B7EF784AA0D4B1B88012B7EF4AE
:105040007FAA3A68A2F10C007F2840F3B7818B3A1F
:105050000C2092FBF0F300FB13207330084BC0B21E
:10506000197804F09BFCFEF76BBA00BF689DFF1F28
:105070000A9DFF1FE49EFF1F949EFF1F643A0100DC
:10508000609DFF1FF09CFF1FCE4C2388002B40F03B
:10509000BF81DFF864B3CC49CC4A098899F8000095
:1050A000B2F800E0DFF85483C1EB000C0C229CFB4B
:1050B000F2F102FB11C14FF0900C0CFB0EFE02FB53
:1050C00001E16FF00B0E58F8011008440EFB0300CD
:1050D0007F2840F36E83A0F17F0393FBF2F002FB85
:1050E00010307330C0B204F07DFCBBF80020238880
:1050F0001344022B22DDB44AB44B118899F8000006
:10510000B3F800C0DFF8F4E2411A0C2291FBF2F38D
:1051100002FB1311902303FB0CF302FB01337344D6
:105120005B6818447F2840F35C847F3890FBF2F37F
:1051300002FB13007330C0B204F054FCBBF8002033
:1051400023881344032B22DD9F4AA04B118899F832
:105150000000B3F800C0DFF8A4E2411A0C2291FB72
:10516000F2F302FB1311902303FB0CF302FB013358
:1051700073449B6818447F2840F39D837F3890FBDD
:10518000F2F302FB13007330C0B204F02BFCBBF847
:10519000002023881344042B7EF753A88C4B1B88D4
:1051A000012B7EF44EA899F80020A2F10C007F2874
:1051B0007EF76FAF8B3A0C2092FBF0F300FB1320CD
:1051C0007330FEF78CBEDFF800A299F80000BAF841
:1051D0000030804CC11A0C2291FBF2F302FB131336
:1051E00002FB03F3E35818447F287FF78FAD7F3825
:1051F00090FBF2F302FB1300733048E5764B1A88FC
:10520000182A13D03B681344A3F118007F2840F3F9
:105210004F830C20973B93FBF0F200FB123303F11A
:1052200073006E4BC0B2197804F0B8FB6C4B6D493B
:105230001A78022A94BF013200221A701A7831F8C3
:105240001200182810D10424022A02F10100C2B26F
:1052500088BF002231F81200182804D1013CF3D194
:105260001A70FEF76DB91A703B680344A3F1180079
:105270007F2840F3A3800C20973B93FBF0F200FBC8
:10528000123303F17300E9E6534B1B88182B12D03D
:1052900099F800201344A3F118007F2840F33483C9
:1052A0000C20973B93FBF0F200FB123303F17300E9
:1052B000C0B204F097FB4A4A4A4B127833F81230D6
:1052C000182B3DF4BEAF99F800201344A3F1180049
:1052D0007F287EF7DEAE0C20973B93FBF0F200FBBD
:1052E000123303F17300FEF7FABDFBF7B5F9FFF7D0
:1052F000AFBBFBF7B1F988E4FBF7AEF91BE43A4B1F
:105300001B78002B00F05882384B1B78002B7DF463
:1053100040AB374B1B78002B3DF43BABB8F800306B
:1053200034490A3BA8F800300A70FDF732BB2A4B1B
:105330001A88182A13D03B681344A3F118007F2859
:1053400040F3BC820C20973B93FBF0F200FB12333E
:1053500003F17300C0B298F8001004F01FFB204B5B
:1053600020491A78022A94BF013200221A701A7852
:1053700031F81200182810D10424022A02F1010089
:10538000C2B288BF002231F81200182804D1013CB3
:10539000F3D11A70FEF7CCB91A703B680344A3F13D
:1053A00018007F287EF783AE0C20973B93FBF0F22A
:1053B00000FB123303F17300FEF742BEFBF74CF91A
:1053C0004CE600BF689DFF1FE49EFF1F949EFF1FD9
:1053D0000A9DFF1F7C420100FA9CFF1F609DFF1F7A
:1053E000A889FF1F009FFF1F869FFF1F879FFF1F2A
:1053F000889FFF1FDD9CFF1FF09CFF1F643A010088
:10540000DFF828A399F80000BAF80030C04CE1E6B4
:10541000C04ADFF82CB31288BBF800100332914267
:105420007FF763AE37E6BC4B1B88182B12D099F878
:1054300000201344A3F118007F2840F342820C207F
:10544000973B93FBF0F200FB123303F17300C0B201
:1054500004F0C8FAB14AB24B127833F81230182B64
:105460007FF431AFFDF7EDBEAB4B1A88182A13D08D
:105470003B681344A3F118007F2840F3AB820C2053
:10548000973B93FBF0F200FB123303F17300C0B2C1
:1054900098F8001004F082FAA04BA1491A78022A69
:1054A00094BF013200221A701A7831F812001828BD
:1054B0007FF473AF0424022A02F1010294BFD2B236
:1054C000002231F8120018287FF466AF013CF2D1B7
:1054D0001A70FEF72DB98F4ADFF864B21288BBF854
:1054E0000010033291427FF74CAD20E5DFF850B257
:1054F0007EE4894B1A88182A13D03B681344A3F121
:1055000018007F2840F323820C20973B93FBF0F296
:1055100000FB123303F17300824BC0B2197804F020
:105520003DFA7E4B7E491A78022A94BF013200224E
:105530001A701A7831F8120018287FF495AE0424F6
:10554000022A02F1010294BFD2B2002231F8120005
:1055500018287FF488AE013CF2D11A70FDF7F0BF35
:10556000714C2388002B40F04382DFF8D4B16F499F
:1055700099F800006E4A09881788DFF8B8E1411AE7
:105580000C2291FBF2FC02FB1C114FF0900C0CFB67
:1055900007F702FB01716FF00B075EF80110014481
:1055A00007FB03107F2840F320827F3890FBF2F343
:1055B00002FB13007330C0B204F014FABBF80020F1
:1055C00023881344022B21DD584B594A99F80000D7
:1055D0001B88B2F800E0574FC31A0C2193FBF1F27D
:1055E00001FB1232902303FB0EF301FB02333B4419
:1055F0005B6818447F2840F314827F3890FBF1F3F6
:1056000001FB13007330C0B204F0ECF9BBF80020CA
:1056100023881344032B21DD444B454A99F80000AD
:105620001B88B2F800E0434FC31A0C2193FBF1F240
:1056300001FB1232902303FB0EF301FB02333B44C8
:105640009B6818447F2840F3E6817F3890FBF1F394
:1056500001FB13007330C0B204F0C4F9BBF80020A2
:1056600023881344042B7EF7ECA92A4B1B88012BBB
:105670007EF4E7A999F80020A2F10C007F287FF7BB
:1056800002A98B3A0C2092FBF0F300FB132073303D
:10569000FFF7E5B8FAF7E0FF6EE4FAF7DDFFFFF792
:1056A000CBBB254B1A88182A13D03B681344A3F1AF
:1056B00018007F2840F3BE810C20973B93FBF0F24B
:1056C00000FB123303F17300C0B298F8001004F02D
:1056D00065F9124B19491A78022A94BF0132002247
:1056E0001A701A7831F8120018287FF456AE042484
:1056F000022A02F1010294BFD2B2002231F8120054
:1057000018287FF449AE013CF2D11A70FEF710B8A8
:10571000244101000A9DFF1F029DFF1FA889FF1F52
:10572000749EFF1F609DFF1F689DFF1FE49EFF1F6B
:10573000949EFF1F643A0100049DFF1F7C9EFF1F83
:10574000F09CFF1FC24B1A88182A13D03B681344E1
:10575000A3F118007F2840F36A810C20973B93FB4C
:10576000F0F200FB123303F17300BA4BC0B21978A8
:1057700004F014F9B84BB9491A78022A94BF0132DF
:1057800000221A701A7831F8120018287FF46CADD4
:105790000424022A02F1010294BFD2B2002231F89D
:1057A000120018287FF45FAD013CF2D11A70FDF7AA
:1057B000C7BEFAF751FF95E4A94B1B78002B7DF487
:1057C000E8A8A84B1B78002B3DF4E3A8B8F80030FC
:1057D000A549013BA8F800300A70FDF7DAB89C4BE8
:1057E0001B88182B12D099F800201344A3F118003D
:1057F0007F2840F313810C20973B93FBF0F200FBD2
:10580000123303F17300C0B204F0ECF8924A934BE8
:10581000127833F81230182B7FF455ADFDF711BD17
:105820008F4B1B78002B7DF494AD8E4B1B78002B97
:105830003DF4AFA8B8F800308B490133A8F8003028
:105840000A70FDF7A6B8894B1B88182B12D099F85F
:1058500000201344A3F118007F2840F3E5800C20BA
:10586000973B93FBF0F200FB123303F17300C0B2DD
:1058700004F0B8F8784A7E4B127833F81230182BBF
:105880003EF4DFA899F800201344A3F118007F2804
:105890007EF7F9AF0C20973B93FBF0F200FB12333D
:1058A00003F17300FEF7DBBFFAF7D6FEFFF78EBBFE
:1058B000FAF7D2FEB5E4FAF7CFFE65E4FAF7CCFECC
:1058C00048E5FAF7C9FEC2E5614B1B88182B12D0D8
:1058D00099F800201344A3F118007F2840F3AD800D
:1058E0000C20973B93FBF0F200FB123303F17300A3
:1058F000C0B204F077F8584A584B127833F8123097
:10590000182BBFD1FEF79DB8FAF7A6FED0E4594B8D
:105910001B88182B12D099F800201344A3F118000B
:105920007F2840F38D800C20973B93FBF0F200FB27
:10593000123303F17300C0B204F054F8464A4E4BE0
:10594000127833F81230182B9CD1FEF77AB8FAF798
:1059500083FEE1E5494B00227F2107201A8003F0F6
:10596000EDFF7F210B2003F0E9FFFDF725BD444B40
:1059700001227F2107201A8003F0E0FF7F210B2006
:1059800003F0DCFFFDF710BD3E4B04227F21072012
:105990001A8003F0D3FF00210B2003F0CFFFFDF7A7
:1059A000FCBC384B02227F2107201A8003F0C6FF7F
:1059B0007F210B2003F0C2FFFDF7EABC314B002131
:1059C00007201C8003F0BAFF7F210B2003F0B6FFF5
:1059D000FDF7D9BCFAF740FE59E5FAF73DFEFFF7AF
:1059E0001FBBFAF739FEFFF7A6BBFAF735FEE2E573
:1059F000254ADFF89CB01288BBF8001003329142B0
:105A00007FF7DCADB3E5FAF727FEFFF73FBAFAF709
:105A100023FEFFF765BAFAF71FFE1CE6FAF71CFE35
:105A2000F1E6FAF719FEEEE5FAF716FE1FE7FAF7C8
:105A300013FE9AE6FAF710FE46E6FAF70DFE57E770
:105A4000FAF70AFE77E7114B0393FDF716BF00BF85
:105A5000049DFF1F609DFF1FA889FF1F7C9EFF1FE5
:105A6000879FFF1F889FFF1FDD9CFF1FFA9CFF1F62
:105A7000009FFF1F029DFF1F749EFF1FD49CFF1FEE
:105A8000829DFF1FDA9EFF1F0A9DFF1F8E9DFF1F35
:105A9000F09CFF1F38B508F0DFFA0B4805F0DEFE7A
:105AA00000234FF07E5201210848FAF7DFFC084B33
:105AB000084A0949802400251C7118461D60BDE86C
:105AC00038400BF0E3BD00BF7C9DFF1FB89EFF1F59
:105AD000449FFF1F1C89FF1FFD05000010B50446F1
:105AE000A4206368198804F0ABF8E368A62019883D
:105AF000BDE8104004F0A4B843682A20198804F0D7
:105B00009FB800BF10B5044622206368198804F0CE
:105B100097F8E36824201988BDE8104004F090B895
:105B200010B504460A206368198804F089F8E36810
:105B30000C201988BDE8104004F082B810B5044666
:105B400006206368198804F07BF8E3680820198848
:105B5000BDE8104004F074B810B504460220636834
:105B6000198804F06DF8E36804201988BDE8104036
:105B700004F066B870B50E4C84B0122504220123DF
:105B800006460390029320468DE82400142310213A
:105B900007F00EFD06220923029303960195204685
:105BA00000921423102107F003FD04B070BD00BF64
:105BB000B89FFF1F70B5AE4CB4F90030032B00F056
:105BC000E880002B4DD0022B6CD0052B00F0988084
:105BD000012B00F0C080042B00D070BD00244FF4D6
:105BE000AF75E1B2A34805F063FE01348542A8BF5A
:105BF00005460C2CF5D1012009F02EFD04460020AD
:105C000009F02AFD323CA0F132039B496FF49570F4
:105C100000FB03F300FB04F081FB034281FB004126
:105C2000DB17C017C3EB6223C0EB612003F5AF7233
:105C300000F5AF739342A8BF13469D42A8BF1D460F
:105C4000A5F11401312900F3E28040F26C73322196
:105C50008A488B4A0180BDE870402A20136003F017
:105C6000EFBF0E2008F05CF940F6FF71C8308842A3
:105C7000A8BF084620EAE07000F2DC5283B28A42F4
:105C8000804D814EA8BF0A460220194633802A80E3
:105C900003F0D6FF2988042003F0D2FFB4F90030C6
:105CA000022B92D1172009F0D7FC0546162009F0E7
:105CB000D3FCA842B8BF284600F1C801B1F5FA7F6D
:105CC000C0F2BF80B1F57A6FA8BF4FF47A6101F5D9
:105CD0004873B3F57A6FA8BF4FF47A639BB289B269
:105CE0006A4A6B4D11800A202B8003F0A9FF298896
:105CF0000C2003F0A5FFB4F90030052B7FF468AF4A
:105D00000F2009F0A9FCC0F53F630433B3F5AF6F72
:105D1000C0F28F80B3F5FA6FA8BF4FF4FA6399B25F
:105D20005C4BC0F54360B0F5AF6F19807EDBB0F51A
:105D3000FA6FA8BF4FF4FA6083B2574DA4202B80AE
:105D400003F07EFF2988A62003F07AFFB4F9003023
:105D5000012B7FF440AF0B2008F036FD00283CD02B
:105D6000112009F079FC00F1C801B1F52F7F3CDB6F
:105D700041F25C23994278DC484A00F5487089B2C8
:105D8000B0F52F7F11806DDB8342A8BF03469BB225
:105D900031E0102009F060FCC830B0F5FA7F4BDB31
:105DA000B0F57A6F0146A8BF4FF47A6101F516731A
:105DB000B3F57A6FA8BF4FF47A639BB289B2384AC1
:105DC000384D118022202B8003F03AFF29882420AF
:105DD00003F036FFB4F90030F3E6152008F0A0F820
:105DE00000F59671B1F52F7F30DA40F214534FF47D
:105DF0002F712A4A11802C4D06202B8003F020FFA2
:105E00002988082003F01CFFB4F90030E3E640F2D3
:105E10003A72A5F5B975254B02FB05F583FB052301
:105E2000ED17A5EB631389B2323311E74FF4AF637B
:105E300083E74FF4AF6173E740F24C434FF4FA71DC
:105E4000BDE740F214534FF4FA7149E741F25C2385
:105E500099420ADC114A00F5617089B2B0F52F7FD2
:105E6000118091DA4FF42F73C5E71946C1E700BFDF
:105E7000949FFF1F7C9DFF1F67BBCF464E9FFF1F58
:105E8000B489FF1F569FFF1F8C9DFF1FF09EFF1FB1
:105E9000009DFF1F909DFF1F109FFF1F3C9DFF1F38
:105EA000A49EFF1FA09EFF1F249FFF1FB5814E1BB6
:105EB0002DE9F041224D82B0012602B284B2009257
:105EC000284601967823192107F0B8FA04F10C024C
:105ED00012B28DE844002846A7197823192104F14D
:105EE000020807F0ABFA3FB20FFA88F819233A46D6
:105EF000284619460196CDF8008007F09FFA7823CE
:105F00003A4628461946CDF80080019604F10A0762
:105F10000B3407F093FA3FB224B278233A4628466E
:105F200019468DE8500007F089FA192300943A4683
:105F300001962846194607F081FA02B0BDE8F081C3
:105F4000B89FFF1F30B583B000230C4605B2009305
:105F500026225B231C210C4806F0C0FF29460123A2
:105F60002622094806F0D6FA002C24B205DB214689
:105F700001232622044806F0CDFA044A044B15807A
:105F80001C8003B030BD00BFB89FFF1FCA89FF1F30
:105F9000CC89FF1F70B5A54C237882B01BB1A44BF0
:105FA0004FF6FF721A80A34BB3F90030C3B9A24A6F
:105FB0009F4B1068B3F9002080F30C005B2303FBB8
:105FC00000F000131C3082424AD04FF0FF31FFF73F
:105FD000B9FF9A4806F0E6FF0023237002B070BDB7
:105FE000012B1BD0022B5AD0032B3FD0042B00F0E7
:105FF0009A80052BF0D10F2009F02EFBC0F53B60F5
:106000000830B0F5AF6F48DBB0F5FA6FA8BF4FF4BA
:10601000FA60A0F5AF625B23894835E0894B1B78B5
:10602000002B70D0152007F07BFF874B1860B0F570
:106030002F7F32DB41F25C239842A8BF1846A0F5BF
:106040002F735B22814802FB03F380FB0320DB17E5
:10605000C3EBA0201C30764BB3F900308342B4D19F
:106060007B4BB3F900300133AFD1B5E7794B1B68F7
:10607000B3F5FA7F11DBB3F57A6FA8BF4FF47A63FB
:106080007548A3F5FA725B2303FB02F380FB032040
:10609000DB17C3EB20201C30DDE71C20DBE76F4B58
:1060A0001B68B3F5FA7F36DBB3F57A6FA8BF4FF400
:1060B0007A63A3F5FA7268485B2303FB02F380FB63
:1060C0000320DB17C3EB20201C30654B1B68B3F5A6
:1060D000FA7F1EDBB3F57A6FA8BF4FF47A63A3F59E
:1060E000FA725D495B2303FB02F381FB0321DB179B
:1060F000C3EB21211C314E4BB3F9003083420CD04D
:10610000FFF720FF65E7112009F0A6FA4E4B186053
:106110008DE71C21EFE71C20D7E74D4BB3F900308A
:106120008B42EDD158E7272200258DE82400762305
:106130001C2142484B4E07F081F916E0B0F5AF7FC5
:10614000A8BF4FF4AF70323803FB00F386FB032186
:10615000DB17C3EB61111C3109B201231D44272257
:10616000364806F0D7F90C2D09D0E9B23E4805F0C3
:106170009FFB31284FF05B03E0DC1C21EDE70120A1
:1061800009F06AFA6FF495733238384A03FB00F06D
:1061900082FB0023C017C0EB632303F5AF73312BE1
:1061A00042DDB3F5AF7FA8BF4FF4AF735B22323B44
:1061B0002C4D02FB03F385FB0325DB17C3EB6515B1
:1061C0001C35002009F048FA6FF495733238274ADD
:1061D00003FB00F082FB0023C017C0EB632303F531
:1061E000AF73312B1EDDB3F5AF7FA8BF4FF4AF7394
:1061F0005B22323B1B4902FB03F381FB0321DB17CC
:10620000C3EB61111C310A4BB3F90030AB4201D032
:10621000284675E70E4BB3F900308B423FF4D9AEF8
:1062200028466DE71C21EEE71C25CAE78E9FFF1F5D
:10623000CA89FF1F949FFF1FF49EFF1FB89FFF1F77
:1062400037800B6DAC9EFF1FC09CFF1FD30585419F
:10625000CC89FF1F109DFF1F011FB8121C9DFF1F3F
:10626000E49CFF1F4B48371B7C9DFF1F67BBCF463D
:106270002DE9F043754C054683B02046D5F80080E3
:10628000EE6806F083FD1120FFF712FE01271923A7
:106290004FF028091946204601972422CDF8009096
:1062A00007F0CCF878231946242201972046CDF830
:1062B000009007F0C3F83946204607F049FC022356
:1062C000192240462382E2810CF09AFF41460246A1
:1062D00020460AF06BFE20460AF07EFE00271423BB
:1062E00003225B4923822046E7810AF05FFE2046B5
:1062F0000AF072FE2323204603225649E7812382B7
:106300000AF054FE20460AF067FE6EB12F20FFF718
:10631000CFFD322303225049E781204623820AF031
:1063200045FE20460AF058FE01234C4A18461370D9
:10633000FFF720FC29896A896B68521A1B885C2A3E
:10634000A3EB010357DD03EB43030132C3EB43131C
:1063500093FBF2F303F11B023C4FDFF80CE113B2A5
:106360001A214FF001088DE802013846AEF80020EE
:106370001946142207F062F8002E4ED0298A6B8A43
:10638000EA685B1A5C2B12883DDC511A5C2202FB26
:1063900001F292FBF3F31B33314A2C4813800126A0
:1063A0001BB2382219468DE84400322207F046F825
:1063B0000022402309218DE806002448194607F0F1
:1063C0000BF83146214807F0C3FB6B681F480222D7
:1063D00044212282E18119880AF04EFE3246214989
:1063E0001A480AF0E3FDEB681848198803B0BDE8C5
:1063F000F0430AF041BE5C2101FB03F393FBF2F38F
:1064000003F11B02A8E7521A02EB4202C2EB42124E
:10641000434492FBF3F31B33BEE74023092132468A
:10642000009138461946019606F0D6FF4146384697
:1064300007F08EFB6B6868210222F9813A82198885
:10644000384603B0BDE8F0430AF016BEB89FFF1F00
:1064500054430100584301005C43010041A0FF1F69
:10646000929FFF1F60430100909FFF1F2DE9F04F97
:106470001F4685B01446002A4ED0052A0646D0F89D
:106480000C8000F0AB800F9B8C4A00EBC305012C05
:10649000B5F80AE029896868C1EB0E0382FB03C2E4
:1064A0001A444FEAE373C3EBA213028851D0042CC1
:1064B00000F08D80824D00220921402328468DE87E
:1064C0000600194606F088FF2846012107F040FB28
:1064D000B8F1000F00F0E8807368022244212A829C
:1064E000E981198828460AF0C7FD76490122284625
:1064F0000AF05CFDF368284619880AF0BDFD724B6E
:10650000022CB3F9001000F0AD80082C00F0C98017
:10651000012005B0BDE8F08F6C4E6D4A33681268FB
:10652000CB1A93420D4655D96A4A3B881178644884
:10653000012918BF012414700E9A06321BB212B240
:106540008DE814001946BDF9382006F077FF356054
:10655000DEE79BB2D31A994203DC9E457146A8BF81
:1065600019460E9A0180B7F90030BDF938A0544899
:1065700002F106094FF0000E0FFA89F9194652464A
:10658000CDF80090CDF804E006F058FF29896A891B
:106590006868521A03885C2AA3EB01037ADD03EBD7
:1065A00043030132C3EB431393FBF2F303F11B02EA
:1065B00013B201203A80194652460190CDF800905E
:1065C0003F4806F03BFF434B00221A7072E712FA75
:1065D00083F3C0E7204605B0BDE8F08F384D4FF09B
:1065E000070A4FF0000B28465A2323228DE8000C9F
:1065F0001A2106F0F1FE2846012107F0A9FA4FF012
:1066000001094FF0350E2323A5F80EE052462B82E8
:106610003149A5F814902846A5F8129003930AF082
:10662000C5FC28460AF0D8FC284606F0BBFC4FF40F
:10663000FA6008F0FFF8FFF7BDFA039B1A211A462B
:1066400028465A238DE8000C06F0C6FE284606F0C0
:10665000A9FC3046FFF70CFE204B83F80090FFF7B3
:1066600099FC27E74A1C12B21A8091423FF450AFBE
:106670000E9AB7F9003012480632012412B2009285
:1066800019460194BDF9382006F0D8FE204605B021
:10669000BDE8F08F5C2101FB03F393FBF2F21B32A8
:1066A00086E700221A80E0E7736868210222E98108
:1066B0002A82198828460AF0DFFC20E7C94216B270
:1066C000B89FFF1F60430100989FFF1F20A0FF1F7E
:1066D0002054010041A0FF1F644301008E9FFF1F53
:1066E0002DE9F04F5A4E5B4DB6F900704C7855F8D5
:1066F000277085B08146984604B10C78DFF874A104
:106700001AB99AF80030002B39D0534D002338467F
:106710002B808AF80030FFF7ABFD504A504BB5F99B
:106720000000012111704FF6FF721A8060B301283A
:106730005ED0012032232246019000934946494B06
:106740003846FFF793FE00240346B5F90020022ADD
:1067500039DD00222A80B6F900203D49002A3BDBC2
:10676000052AC4BF00220A80B8F1000F39D1002CDD
:106770000CBF18464FF0FF3005B0BDE8F08F364D26
:10678000B5F900000028D2D1DFF8ECB0364ADBF8CA
:1067900000301268C3EB0903934227D9334B1A78B0
:1067A000012A18BF01201870FFF7E4F90123CBF884
:1067B0000090012C2AD0042C35D0022C3AD0082C81
:1067C0003ED00024C1E7C6D1FA68002AC1D0B6F98C
:1067D00000201F49002AC3DA05220A80B8F1000F01
:1067E000C5D00393FFF7D6FB039BC0E70346E0E762
:1067F0004FF0000E142322468DE8084049461C4BFA
:1068000038467446FFF732FE03469EE732888AF820
:106810000040013232807A6982B100243846039305
:106820009047039B91E732880121013A32808AF830
:106830000010F0E701222A8000248CE7144684E748
:106840007A69002129804FF0FF34002AE6D182E7DF
:10685000949FFF1FD089FF1F989FFF1F8E9FFF1FD0
:10686000CA89FF1F929FFF1F2054010041A0FF1FF4
:10687000909FFF1F969FFF1F20A0FF1F01210D204B
:1068800007F09CBF00210D2007F098BF01460D20A6
:1068900007F094BF08B50D2007F096FFB0FA80F11D
:1068A00049090D20BDE8084007F088BF10B5002158
:1068B00044080D2007F082FF204607F0BBFF0D20A3
:1068C000012107F07BFF2046BDE8104007F0B2BF72
:1068D000214A224B10881B68984210B535DA204AAD
:1068E0001288141A9A42A8BF1A46B4F5157F22DA04
:1068F000121A40F2532303FB02F393FBF4F1053128
:106900000A2007F0CBFD174B197801B3164B174936
:106910001B6840F2271283F3070302FB03F381FB9A
:1069200003211944DB17C3EBA11105310920BDE890
:10693000104007F0B3BD131A4FF41572611C02FB2F
:1069400003F393FBF1F10531DAE70021D8E70920E1
:10695000BDE8104007F0A2BD8C9DFF1FB89CFF1F33
:10696000569FFF1F3E9DFF1F3C9FFF1F0904028192
:106970007F2838B5A8BF7F200F4C4FF4167202FB5A
:1069800000F284FB02311144D2170546C2EBA1117B
:106990000A2007F083FD7F3D4FF4967303FB05F358
:1069A00084FB03211944DB17A3EBA1110920BDE8E7
:1069B000384007F073BD00BF09040281C368B3F912
:1069C000003030B583EAE374A4EBE374002BA0B28B
:1069D00018DB012300E0134603EB830252009442CC
:1069E000F9DA0A4D90FBF3F285FB03E403FB120096
:1069F000DB173032D3EBA40380B201F8012BF1D1C5
:106A00000B7030BD2D230B700131E2E767666666BF
:106A100038B5094D4624204603F02CF935F8021B01
:106A200000B28842204601D003F00AF90234A4B231
:106A30004E2CF0D138BD00BF009FFF1F024B4420F9
:106A4000198803F0FDB800BFFA9CFF1F38B5094D47
:106A50007824204603F00EF935F8021B00B2884274
:106A6000204601D003F0ECF80234A4B2802CF0D11F
:106A700038BD00BF749EFF1F024B7620198803F0BB
:106A8000DFB800BF029DFF1F38B5094D82242046A4
:106A900003F0F0F835F8021B00B28842204601D01E
:106AA00003F0CEF80234A4B28A2CF0D138BD00BF76
:106AB0007C9EFF1F024B8020198803F0C1B800BFE5
:106AC000049DFF1F024B4E20198803F0B9B800BF88
:106AD000169DFF1F024B9A20198803F0B1B800BF22
:106AE000689DFF1F024B9820198803F0A9B800BFCA
:106AF0000A9DFF1F024B8C20198803F0A1B800BF2C
:106B0000949EFF1F024B9C20198803F099B800BF88
:106B1000F09CFF1F024BA020198803F091B800BF22
:106B2000089FFF1F024B9620198803F089B800BF09
:106B3000E49EFF1F024B8A20198803F081B800BF32
:106B4000AA9EFF1F024B1020198803F079B800BFDE
:106B5000A89EFF1F024B0E20198803F071B800BFDA
:106B6000CE9CFF1F024B2C20198803F069B800BF90
:106B7000EE9CFF1F024B1E20198803F061B800BF76
:106B8000089DFF1F024B2820198803F059B800BF49
:106B9000FE9EFF1F024B6220198803F051B800BF10
:106BA000289DFF1F024B6420198803F049B800BFDD
:106BB000F89EFF1F024BB420198803F041B800BFB4
:106BC0004C9FFF1F024BB620198803F039B800BF55
:106BD000789FFF1F024B5A20198803F031B800BF7D
:106BE000C89CFF1F024B1620198803F029B800BF6C
:106BF000D49CFF1F024B2E20198803F021B800BF40
:106C0000709DFF1F024B3020198803F019B800BF98
:106C1000649FFF1F024B9E20198803F011B800BF2C
:106C2000B089FF1F024BAC20198803F009B800BFE0
:106C3000FA9EFF1F024BAE20198803F001B800BF77
:106C4000149DFF1F024BB020198802F0F9BF00BF4E
:106C5000889EFF1F024BB220198802F0F1BF00BFCF
:106C6000329DFF1F024B1820198802F0E9BF00BFB8
:106C7000929DFF1F024BA220198802F0E1BF00BFC6
:106C80002A9FFF1F024B1A20198802F0D9BF00BFAC
:106C9000209DFF1F024B1C20198802F0D1BF00BFAE
:106CA000189DFF1F024B6620198802F0C9BF00BF64
:106CB000389FFF1F024B7220198802F0C1BF00BF2E
:106CC000609FFF1F024B2020198802F0B9BF00BF50
:106CD000369FFF1F024B3220198802F0B1BF00BF60
:106CE000269FFF1F024B6820198802F0A9BF00BF32
:106CF0005C9DFF1F024B6C20198802F0A1BF00BFF2
:106D0000BC9CFF1F024BBA20198802F099BF00BF3C
:106D1000729EFF1F024B5220198802F091BF00BFE4
:106D20004889FF1F024B5020198802F089BF00BF1D
:106D30003689FF1F024B5420198802F081BF00BF23
:106D4000C489FF1F024B5C20198802F079BF00BF85
:106D5000C889FF1F024B5E20198802F071BF00BF77
:106D60004089FF1F024B5620198802F069BF00BFFF
:106D70005E9DFF1F244B1B880B2B43D8DFE803F0DD
:106D80000B10151A1F24292E33383D0608460422FD
:106D90001E490CF0F3BA084604221D490CF0EEBA65
:106DA000084604221B490CF0E9BA084604221A4995
:106DB0000CF0E4BA0846042218490CF0DFBA084681
:106DC000042217490CF0DABA0846042215490CF0DF
:106DD000D5BA0846042214490CF0D0BA0846042259
:106DE00012490CF0CBBA0846042211490CF0C6BA7D
:106DF000084604220F490CF0C1BA084604220E4985
:106E00000CF0BCBA704700BFE49EFF1F8C5001001D
:106E1000C0510100E04B010078510100E44B01003A
:106E200060510100E84B0100EC4B0100204F0100D4
:106E3000F04B010098500100F44B0100064B074A4B
:106E400010B41C88064B0846002C14BF1146194686
:106E5000042210BC0CF092BA389DFF1FF84B0100C1
:106E6000FC4B0100064B074A10B41C88064B084631
:106E7000002C14BF11461946042210BC0CF07EBA37
:106E8000749DFF1FF84B0100FC4B0100064B074AA5
:106E900010B41C88064B0846002C14BF1146194636
:106EA000042210BC0CF06ABA9E9EFF1FF84B010032
:106EB000FC4B0100064B074A10B41C88064B0846E1
:106EC000002C14BF11461946042210BC0CF056BA0F
:106ED000AE9EFF1FF84B0100FC4B0100064B074A1A
:106EE00010B41C88064B0846002C14BF11461946E6
:106EF000042210BC0CF042BAE69EFF1FF84B0100C2
:106F0000FC4B0100064B074A10B41C88064B084690
:106F1000002C14BF11461946042210BC0CF02EBAE6
:106F2000829DFF1FF84B0100FC4B01001B4B1B888F
:106F30000A2B0AD8DFE803F00A0E12161A1E2226C0
:106F40002A2E0600164B186808607047154B186803
:106F500008607047144B186808607047134B186836
:106F600008607047124B186808607047114B18682A
:106F700008607047104B1868086070470F4B18681E
:106F8000086070470E4B1868086070470D4B186812
:106F9000086070470C4B186808607047AA9EFF1F76
:106FA000244C0100FC4B0100004C0100044C01008A
:106FB000084C01000C4C0100104C0100144C010065
:106FC000184C01001C4C0100204C0100424B1B8856
:106FD000182B0ED8DFE803F07B77726E6964605B74
:106FE00057524E4945413C38332E2A25211C18134F
:106FF0000E0070470846042238490CF0BFB9084615
:10700000042237490CF0BAB9364B1868086070474B
:107010000846042234490CF0B1B9344B18680860B2
:1070200070470846042232490CF0A8B9314B186861
:1070300008607047084604222F490CF09FB90846A3
:1070400004222E490CF09AB92D4B1868086070473D
:10705000084604222B490CF091B92B4B18680860A4
:1070600070472A4B18680860704708460422284970
:107070000CF084B9274B1868086070470846042252
:1070800025490CF07BB9254B186808607047084605
:10709000042223490CF072B9224B1868086070472B
:1070A0000846042220490CF069B9084604221F4909
:1070B0000CF064B91E4B186808607047084604223B
:1070C0001C490CF05BB91C4B1868086070470846F7
:1070D00004221A490CF052B9CE9CFF1F884C0100C3
:1070E000844C0100804C01007C4C0100784C010074
:1070F000744C0100704C01006C4C0100684C0100A4
:10710000644C0100604C01005C4C0100584C0100D3
:10711000544C0100504C01004C4C0100484C010003
:10712000444C0100404C01003C4C0100384C010033
:10713000344C0100304C01002C4C0100284C010063
:10714000F0B52B4E2B4FDFF8C4E005460FCE87B0CD
:107150006C460FC496E803003B68274A274F44F863
:10716000040B40F6CC308342C8BF3A46BEF80060FC
:107170002180012E11889278ADF80D108DF80F2026
:107180002AD032D340F6CA02022E18BF00229A42F9
:1071900026DAA3F698031A491A4AC3EB031381FBB4
:1071A00003011944DB17C3EB6123243382FB032162
:1071B000DA17C2EBA10202EB8201A3EB41033033E9
:1071C00030328DF813308DF811206946284616228A
:1071D0000CF0D4F807B0F0BD40F698029A42D8DB24
:1071E000094B1868CDF81100EFE740F6FC02CEE736
:1071F0009C4C0100EC9EFF1F904C01008C4C010048
:107200003B773B9867666666944C0100849EFF1F3F
:10721000F8B5174C174E2278174D33782F888E46C5
:10722000003218BF012201467046FFF759FA0023C9
:1072300098423370237015DB14BF012000202B8887
:107240009F420ED040F23A72A3F5AF730B490C4C3B
:1072500002FB03F381FB0312DB17A3EB6213323350
:107260002360F8BD0749012218460A702270E6E73C
:10727000308AFF1FAD9FFF1F4E9FFF1FB5814E1B22
:10728000B489FF1FA59FFF1F014B187802F048BC6F
:107290001CA0FF1F014B187802F05CBCAC90FF1FD4
:1072A000134BB3F9003030B583EAE374A4EBE37415
:1072B000002BA0B218DB012300E0134603EB83028E
:1072C00052009442F9DA0B4D90FBF3F285FB03E494
:1072D00003FB1200DB173032D3EBA40380B201F8BA
:1072E000012BF1D10B7030BD2D230B700131E2E782
:1072F000AC90FF1F67666666144BB3F9003070B53B
:1073000083EAE375A5EBE375002BACB21ADB01232E
:1073100000E0034603EB830040008542F9DA0C4E9F
:1073200094FBF3F086FB03E503FB1044DB173030DE
:10733000D3EBA503A4B201F8010BF1D105480B7002
:10734000106070BD2D230B700131E0E7C89CFF1F5A
:1073500067666666B44C0100134BB3F9003030B574
:1073600083EAE374A4EBE374002BA0B218DB0123DF
:1073700000E0134603EB830252009442F9DA0B4D0E
:1073800090FBF3F285FB03E403FB1200DB173032C2
:10739000D3EBA40380B201F8012BF1D10B7030BD07
:1073A0002D230B700131E2E7B089FF1F6766666627
:1073B000134BB3F9003030B583EAE374A4EBE37404
:1073C000002BA0B218DB012300E0134603EB83027D
:1073D00052009442F9DA0B4D90FBF3F285FB03E483
:1073E00003FB1200DB173032D3EBA40380B201F8A9
:1073F000012BF1D10B7030BD2D230B700131E2E771
:10740000149DFF1F67666666134BB3F9003030B5F5
:1074100083EAE374A4EBE374002BA0B218DB01232E
:1074200000E0134603EB830252009442F9DA0B4D5D
:1074300090FBF3F285FB03E403FB1200DB17303211
:10744000D3EBA40380B201F8012BF1D10B7030BD56
:107450002D230B700131E2E7329DFF1F67666666E0
:10746000134BB3F9003030B583EAE374A4EBE37453
:10747000002BA0B218DB012300E0134603EB8302CC
:1074800052009442F9DA0B4D90FBF3F285FB03E4D2
:1074900003FB1200DB173032D3EBA40380B201F8F8
:1074A000012BF1D10B7030BD2D230B700131E2E7C0
:1074B0002A9FFF1F67666666144B1B8801331BB249
:1074C00030B583EAE374A4EBE374002BA0B218DBBD
:1074D000012300E0134603EB830252009442F9DAE1
:1074E0000B4D90FBF3F285FB03E403FB1200DB176B
:1074F0003032D3EBA40380B201F8012BF1D10B7031
:1075000030BD2D230B700131E2E700BF729EFF1FDB
:1075100067666666134BB3F9003030B583EAE374EF
:10752000A4EBE374002BA0B218DB012300E01346A8
:1075300003EB830252009442F9DA0B4D90FBF3F215
:1075400085FB03E403FB1200DB173032D3EBA4030B
:1075500080B201F8012BF1D10B7030BD2D230B70DF
:107560000131E2E74889FF1F67666666134BB3F98E
:10757000003030B583EAE374A4EBE374002BA0B2CF
:1075800018DB012300E0134603EB83025200944210
:10759000F9DA0B4D90FBF3F285FB03E403FB1200D9
:1075A000DB173032D3EBA40380B201F8012BF1D109
:1075B0000B7030BD2D230B700131E2E73689FF1FC0
:1075C00067666666134BB3F9003030B583EAE3743F
:1075D000A4EBE374002BA0B218DB012300E01346F8
:1075E00003EB830252009442F9DA0B4D90FBF3F265
:1075F00085FB03E403FB1200DB173032D3EBA4035B
:1076000080B201F8012BF1D10B7030BD2D230B702E
:107610000131E2E7C489FF1F67666666134BB3F961
:10762000003030B583EAE374A4EBE374002BA0B21E
:1076300018DB012300E0134603EB8302520094425F
:10764000F9DA0B4D90FBF3F285FB03E403FB120028
:10765000DB173032D3EBA40380B201F8012BF1D158
:107660000B7030BD2D230B700131E2E7C889FF1F7D
:1076700067666666134BB3F9003030B583EAE3748E
:10768000A4EBE374002BA0B218DB012300E0134647
:1076900003EB830252009442F9DA0B4D90FBF3F2B4
:1076A00085FB03E403FB1200DB173032D3EBA403AA
:1076B00080B201F8012BF1D10B7030BD2D230B707E
:1076C0000131E2E74089FF1F6766666608B5B820AA
:1076D00002F0D0FA044B1988884204D0B820BDE8E3
:1076E000084002F0ADBA08BDD09CFF1F08B570205D
:1076F00002F0C0FA044B1988884204D07020BDE81B
:10770000084002F09DBA08BD849EFF1F08B5742092
:1077100002F0B0FA044B1988884204D07420BDE806
:10772000084002F08DBA08BD1C9FFF1F054B1B8847
:107730000846042213B904490BF020BE03490BF09C
:107740001DBE00BF169DFF1FBC4C0100B84C0100C0
:107750000E4B1B88032B17D8DFE803F0110C070230
:10776000084604220A490BF009BE084604220949CA
:107770000BF004BE0846042207490BF0FFBD084683
:10778000042206490BF0FABD704700BF949EFF1F0C
:10779000CC4C0100C84C0100C44C0100C04C01009D
:1077A00010B40A4B0A4C0A4693E8030083B02388BE
:1077B00002AC04E9030004EB8303104653F8081CF1
:1077C000052203B010BC0BF0D9BD00BFE44301009B
:1077D000F89EFF1F30B40A4B0A4D0C4693E8070091
:1077E00084B02B8804AD05E9070005EB8303204630
:1077F00053F80C1C042204B030BC0BF0BFBD00BF1A
:10780000EC430100849EFF1FF0B40C4D0C4F0E465C
:107810000FCD8CB001AC0FC40FCD0FC495E807009D
:107820003B8884E807000CAA02EB8303304653F838
:107830002C1C04220CB0F0BC0BF0A0BDF8430100DE
:10784000DA9EFF1F30B50A4B0A4D0C460FCB85B0B0
:107850000DF1100E0EE90F002B880EEB830320466E
:1078600053F8101C042205B0BDE830400BF086BD73
:1078700034440100FA9EFF1F30B50A4B0A4D0C46F6
:107880000FCB85B00DF1100E0EE90F002B880EEB1B
:107890008303204653F8101C042205B0BDE8304095
:1078A0000BF06CBD34440100889EFF1FF0B40B4DFB
:1078B0000B4F0E460FCD86B06C460FC495E8030003
:1078C0003B8884E8030006AA02EB8303304653F8A2
:1078D000181C042206B0F0BC0BF050BD444401005B
:1078E000929DFF1FF0B40A4D0A4F0E460FCD86B091
:1078F00001AC0FC42A683B88226006AA02EB83030E
:10790000304653F8141C0C2206B0F0BC0BF036BD08
:107910005C440100189DFF1FF0B40B4D0B4F0E4649
:107920000FCD88B06C460FC495E80F0084E80F00B7
:107930003B8808AA02EB8303304653F8201C04223C
:1079400008B0F0BC0BF01ABD704401001C9FFF1F73
:10795000164B1B880BB31BB283EAE370A0EBE370FA
:10796000002B30B584B21DDB012300E0134603EB8E
:10797000830252009042F9DA0D4894FBF3F280FB47
:1079800003E503FB1244DB173032D3EBA503A4B2AB
:1079900001F8012BF1D10B7030BD084604220549D6
:1079A0000BF0ECBC2D230B700131DDE75C9DFF1F5C
:1079B00067666666D04C010030B50A4B0A4D0C462E
:1079C0000FCB85B00DF1100E0EE90F002B880EEBDA
:1079D0008303204653F8101C042205B0BDE8304054
:1079E0000BF0CCBC90440100BC9CFF1F054B1B88D6
:1079F0001BB9054B18680860704708460422034904
:107A00000BF0BCBC689DFF1FFC4B0100F84B010054
:107A1000164B1B880BB31BB230B583EAE374A4EB9F
:107A2000E374002BA0B21CDB012300E0134603EB40
:107A3000830252009442F9DA0D4D90FBF3F285FB7C
:107A400003E403FB1200DB173032D3EBA40380B254
:107A500001F8012BF1D10B7030BD064B186808609E
:107A600070472D230B700131DEE700BF089DFF1F1B
:107A700067666666FC4B0100164B1B880BB31BB296
:107A800030B583EAE374A4EBE374002BA0B21CDBF3
:107A9000012300E0134603EB830252009442F9DA1B
:107AA0000D4D90FBF3F285FB03E403FB1200DB17A3
:107AB0003032D3EBA40380B201F8012BF1D10B706B
:107AC00030BD064B1868086070472D230B700131DC
:107AD000DEE700BFD09CFF1F67666666FC4B0100B7
:107AE000164B1B880BB31BB230B583EAE374A4EBCF
:107AF000E374002BA0B21CDB012300E0134603EB70
:107B0000830252009442F9DA0D4D90FBF3F285FBAB
:107B100003E403FB1200DB173032D3EBA40380B283
:107B200001F8012BF1D10B7030BD064B18680860CD
:107B300070472D230B700131DEE700BFEA9EFF1F67
:107B400067666666FC4B0100164B1B880BB31BB2C5
:107B500030B583EAE374A4EBE374002BA0B21CDB22
:107B6000012300E0134603EB830252009442F9DA4A
:107B70000D4D90FBF3F285FB03E403FB1200DB17D2
:107B80003032D3EBA40380B201F8012BF1D10B709A
:107B900030BD064B1868086070472D230B7001310B
:107BA000DEE700BFD49CFF1F67666666D44C010009
:107BB000174B1B881BB31BB270B583EAE375A5EBAB
:107BC000E375002BACB21EDB012300E0034603EBA0
:107BD000830040008542F9DA0E4E94FBF3F086FBF9
:107BE00003E503FB1044DB173030D3EBA503A4B24D
:107BF00001F8010BF1D108480B70106070BD074B04
:107C00001868086070472D230B700131DCE700BF56
:107C1000709DFF1F67666666D84C0100FC4B010033
:107C2000164B1B880BB31BB230B583EAE374A4EB8D
:107C3000E374002BA0B21CDB012300E0134603EB2E
:107C4000830252009442F9DA0D4D90FBF3F285FB6A
:107C500003E403FB1200DB173032D3EBA40380B242
:107C600001F8012BF1D10B7030BD064B186808608C
:107C700070472D230B700131DEE700BF649FFF1FAB
:107C800067666666FC4B0100164B1B880BB31BB284
:107C900030B583EAE374A4EBE374002BA0B21CDBE1
:107CA000012300E0134603EB830252009442F9DA09
:107CB0000D4D90FBF3F285FB03E403FB1200DB1791
:107CC0003032D3EBA40380B201F8012BF1D10B7059
:107CD00030BD064B1868086070472D230B700131CA
:107CE000DEE700BF389FFF1F67666666FC4B01003A
:107CF000164B1B880BB31BB230B583EAE374A4EBBD
:107D0000E374002BA0B21CDB012300E0134603EB5D
:107D1000830252009442F9DA0D4D90FBF3F285FB99
:107D200003E403FB1200DB173032D3EBA40380B271
:107D300001F8012BF1D10B7030BD064B18680860BB
:107D400070472D230B700131DEE700BF609FFF1FDE
:107D500067666666FC4B0100174B1B881BB31BB2A2
:107D600070B583EAE375A5EBE375002BACB21EDBBF
:107D7000012300E0034603EB830040008542F9DA6B
:107D80000E4E94FBF3F086FB03E503FB1044DB1778
:107D90003030D3EBA503A4B201F8010BF1D10848B0
:107DA0000B70106070BD074B1868086070472D237A
:107DB0000B700131DCE700BF369FFF1F6766666608
:107DC000D84C0100FC4B0100054B1B881BB1054B37
:107DD000186808607047044B18680860704700BF57
:107DE0005E9DFF1FEC4C0100E84C010070B5FAF7F6
:107DF00099F9164B1B7813B1154C237833B9154BF1
:107E00001020198801F01CFF012070BD124D134E87
:107E10002B783288B3FA83F382F008025B091146AB
:107E200042202B70328001F00BFF23780BB12B78AE
:107E30002BB90021212006F0C1FC002070BD0121DA
:107E4000212006F0BBFC002070BD00BFD89EFF1FA4
:107E50008A9EFF1FA89EFF1FA69EFF1F589FFF1F01
:107E6000184B1A8852B3184A128830B50A80B3F9F1
:107E70000030002B83EAE374A4EBE374BCBF2D2332
:107E80008B70A0B2ACBF02310331012300E0134676
:107E900003EB830252009442F9DA0C4D90FBF3F2AB
:107EA00085FB03E403FB1200DB173032D3EBA403A2
:107EB00080B201F8012BF1D10B7030BD044B186872
:107EC00008607047209DFF1FF04C010067666666E2
:107ED000FC4B010070B53C4D2B780646002B35D18C
:107EE0001C4673780BB9204670BDFAF71BF9374A68
:107EF000374B3848127831781B78007802EB43030F
:107F00004A1E03EB80030E2AEDD801A050F822F0A0
:107F1000797F00009B7F0000E77E0000797F0000F2
:107F2000E77E0000E77E0000E77E0000677F00003C
:107F3000E77E0000E77E0000E77E0000E77E0000AD
:107F4000E77E0000E77E0000637F0000AE2122484C
:107F500004F0D0FC204804F019FF00232B7001240A
:107F6000BFE707F099FCAF211B4804F0C3FC1B4A94
:107F7000012313702B70B6E783B9194803880429CD
:107F80004FF6FF7103F1FF320CBF01230B46134480
:107F900003F07F03013303800FE073B1013B114A0B
:107FA00032F813304BB10E4E0F481049104A33804F
:107FB0000123002606700B701370084A022101236A
:107FC00011702B70204670BD308AFF1F899FFF1FE4
:107FD0008A9FFF1F2C9FFF1FB89FFF1FA59FFF1F9A
:107FE000289FFF1F649EFF1F549DFF1FDD9CFF1FE6
:107FF00043A0FF1F10B5064B064C1A8820460121EE
:1080000001F00CFE21884220BDE8104001F018BEAE
:10801000389DFF1F589FFF1F10B5064B064C1A884E
:108020002046022101F0FAFD21884220BDE81040DF
:1080300001F006BE749DFF1F589FFF1F10B5064B31
:10804000064C1A882046042101F0E8FD21884220D0
:10805000BDE8104001F0F4BD9E9EFF1F589FFF1F1A
:1080600010B5064B064C1A882046062101F0D6FDB5
:1080700021884220BDE8104001F0E2BDAE9EFF1F06
:10808000589FFF1F10B5064B064C1A88204600214A
:1080900001F0C4FD21884220BDE8104001F0D0BDB0
:1080A000E69EFF1F589FFF1F08B5122001F0E2FD5A
:1080B000054B1988884206D0122001F0C1FDBDE8A9
:1080C000084001F05FBC08BDDA9EFF1F08B55820CC
:1080D00001F0D0FD054B1988884206D0582001F0E8
:1080E000AFFDBDE8084001F04DBC08BDEA9EFF1F92
:1080F00008B5142001F0BEFD054B1988884206D052
:10810000142001F09DFDBDE8084001F03BBC08BD16
:10811000829DFF1FF0B480EAE075A5EBE0750028B2
:10812000ACB21FDB1DBF2B230B704E1C0E46012370
:1081300000E0134603EB830252009542F9DA0B4F3D
:1081400094FBF3F287FB030503FB1244DB17303289
:10815000D3EBA503A4B206F8012BF1D13370084686
:10816000F0BC70472D230B704E1CE0E76766666617
:108170001A4B18880C2815D0192817D01A2819D08E
:108180001B281BD01C281DD01D281FD01E2821D025
:108190001F2803D00C3800B2FFF7BCBF104A10688C
:1081A000086070470F4A1068086070470E4A1068F0
:1081B000086070470D4A1068086070470C4A1068E4
:1081C000086070470B4A1068086070470A4A1068D8
:1081D00008607047094A106808607047269FFF1FB3
:1081E000144D0100F84C0100FC4C0100004D010051
:1081F000044D0100084D01000C4D0100104D01001F
:10820000034B1888A0EB8000400000B2FFF782BF4C
:108210001CA0FF1F024B1888643800B2FFF77ABF1A
:10822000789FFF1F024B1888643800B2FFF772BFB7
:108230004C9FFF1F024BB3F90000FFF76BBF00BF5D
:10824000289DFF1F024B1888033800B2FFF762BF5A
:10825000FE9EFF1F024B1888183800B2FFF75ABF66
:10826000049DFF1F024B1888183800B2FFF752BF59
:10827000029DFF1F024B1888183800B2FFF74ABF53
:10828000FA9CFF1FC3681888183800B2FFF742BF76
:10829000054B1B881BB9054B1868086070470846DA
:1082A000042203490BF06AB8089FFF1FFC4B010032
:1082B000F84B0100054B1B881BB9054B186808607B
:1082C00070470846042203490BF058B80A9DFF1F67
:1082D000FC4B0100F84B010030B5154C85B0012571
:1082E0002B463C2202212046009504F079FB2046D3
:1082F00004F04CFD00224021802320460191009390
:1083000011460C4B029505F0EFF9204604F04AFEA9
:1083100009480A490A4A00230360436003720B605C
:108320004B600B7213605360137205B030BD00BF19
:10833000B89FFF1F304501009C9FFF1F38A0FF1F03
:1083400024A0FF1F10B500EBC00000F10F02D2B255
:1083500093B284B09C1E981C3D2303918DE81900B4
:108360003921024805F024F904B010BDB89FFF1F61
:10837000014B01221A707047AD9FFF1FF0B57A4B79
:108380007A4C7B4F7B4E7C4D85B004228DE80C00EF
:1083900002932046794B4022802104F029F920469F
:1083A000774A7849784C09F071F9784A784B9761A7
:1083B000784FD761784F9F61784FDF61784FB76111
:1083C000784FF761784FAF61784FEF61784FA761D1
:1083D0007848794FE761794F87617949794FC7616B
:1083E000794F8F61794A7A4FCF617A4F97617A4B93
:1083F0007A4FD7617A4F9F617A4E7B4FDF617B4F17
:108400007B4DB7617B4FF7617B4F7C4CAF617C4FFD
:10841000EF617C4F7C48A7617C4FE7617C4F7D49D1
:1084200087617D4FC7617D4F7D4A8F617D4FCF61F1
:108430007D4F7E4B97617E4FD7617E4F7E4E9F6111
:108440007E4FDF617E4FB7617E4D7F4FF7617F4F7B
:10845000AF617F4C7F4FEF617F4FA7617F48804FB7
:10846000E761804F87618049804FC761804F8F618E
:10847000804A814FCF61814F9761814B814FD76196
:10848000814F9F61814E824FDF61824FB761824D84
:10849000824FF761824FAF61824C834FEF61834F10
:1084A000A7618348834FE761834F84498761844F85
:1084B000C761844F844A8F61844FCF61844F854B5D
:1084C0009761854FD761854F854E9F61854FDF61ED
:1084D000854F864DB761864FF761864F864CAF61F9
:1084E000864FEF61864F8748A761874FE761874FC7
:1084F00087618749874FC761874F8F61874A884F58
:10850000CF61884F9761884B884FD761884F9F61B3
:10851000884E894FDF61894F894DB761894FF76177
:10852000894F8A4CAF618A4F8A488B49EF618B4FE4
:108530008B4DA761E5618B4F8B4D8C4CDFF850E282
:108540008B4A8C4B8761C5618C618B4E8B4F8C4DF8
:108550008C4CC1F81CE08C488C499761D5619C61BA
:10856000D861B16005B0F0BD40420F00B89FFF1F59
:1085700045820000248CFF1F8C8FFF1F7091FF1F0E
:108580001C89FF1F49C60000E889FF1F688FFF1F75
:108590007C8EFF1F856B00003D6E0000F57F0000A4
:1085A000656E0000198000008D6E00003D800000A7
:1085B00035820000B48CFF1F956B0000B56E000083
:1085C000688DFF1F61800000A1770000908CFF1F65
:1085D000A56B0000DD6E00008C8DFF1F8580000004
:1085E00025820000F890FF1FB56B00001582000087
:1085F000D490FF1FC56B0000797A0000448DFF1FE7
:10860000CD76000001820000208DFF1F89720000DE
:10861000A1720000448FFF1F95720000D577000003
:10862000A48BFF1FED76000009780000F88FFF1F74
:10863000A9800000E17A00006C8CFF1FCD80000053
:10864000F9720000648BFF1FD56B0000056F0000FE
:108650008890FF1FF1800000497B0000488CFF1FBD
:10866000E56B0000B17B0000D48DFF1FF56B0000AF
:10867000217C0000EC8BFF1F056C0000597300008B
:10868000E48AFF1F156C0000457800004090FF1F32
:10869000256C0000B1730000E88EFF1F356C0000F0
:1086A00079780000C08AFF1F456C00000974000043
:1086B000B08DFF1F556C0000AD780000A08EFF1F2D
:1086C000656C000061740000D88CFF1F756C0000A1
:1086D000617E00000C8FFF1F856C0000E5780000B4
:1086E0004C91FF1F956C0000897C0000588EFF1F85
:1086F000A56C0000F17C00009C8AFF1FB56C000097
:10870000197900001C90FF1F0D770000597D0000B3
:10871000C48EFF1FC56C000071810000788AFF1FA6
:10872000D56C000051790000B090FF1FE56C00008F
:10873000B97900001C8BFF1FF56C0000B9740000B4
:10874000FC8CFF1F056D000015750000C88BFF1F16
:10875000156D00000C8AFF1F408BFF1F6D75000018
:10876000256D0000C5750000356D00001D76000008
:10877000B08FFF1F2891FF1F1C91FF1F757600000F
:10878000556D0000C97D0000656D00004D8D000035
:10879000456D0000F0B5461C83B00D46012703234C
:1087A00036B22AB2044631468DE888002348ADB27D
:1087B00004F094FE0C23AA1C12B200930197052327
:1087C00021B21E4804F08AFE1D4A1E4B12881B6807
:1087D000BA422AD023D3022A10D11B4CA3F6CA03D3
:1087E00084FB03241C44DB17C3EB24140A2CA8BF0E
:1087F0000A2424EAE474A2B223B202E000231A4657
:108800001C460D35AA1A01200093019012B2314680
:1088100003230A4804F0E0FD204603B0F0BD0B4CF2
:10882000A3F6FC0384FB0324DDE7094CA3F69803BD
:1088300084FB0324DB17C3EBA404D7E7B89FFF1F17
:10884000849EFF1FEC9EFF1F09CB3D8D1F85EB51C2
:10885000398EE3382DE9F0438FB283B0DFF84C80D6
:10886000BD1D461D2DB204B236B24FF001090AB249
:108870002346314640460095CDF8049004F0DEFDD5
:108880002A463346214640468DE8200204F0D6FDB4
:1088900007F10C020095334612B22146CDF8049040
:1088A000404604F0CBFD03B0BDE8F083B89FFF1F46
:1088B0002DE9F04F804685B0002959D1012131487A
:1088C00005F046F9304998F8062098F8083011F874
:1088D0000290994525DADFF8ACB04FEA89064D469B
:1088E0000C244FF0000AD8F80C309B595F68ABF8A5
:1088F00010403846ABF80EA00AF082FC394602461A
:10890000204808F053FB1F4808F066FB98F8083031
:1089100001350934AB42A4B206F1040601DD422C54
:10892000E1D1B9F1000F13D109F1060999450CDA2B
:108930003C2301213B2203910293009301923923AE
:108940003F223A210F4804F033FE05B0BDE8F08F16
:108950000F2301213B2203910293009301923923BB
:108960000C223A21074804F023FE98F80830DBE790
:1089700000213423009301913F230C22014804F08D
:108980002BFD9BE7B89FFF1F38A0FF1F38B50F4C8A
:10899000012320461946A3826382552505F0D8F8A5
:1089A0003423204602220A492382E58108F0FEFA98
:1089B00020460522074908F0F9FA204608F00CFB8A
:1089C0002046BDE8384004F0EDBA00BFB89FFF1F55
:1089D000604D0100644D0100F8B50F4606460AF0EF
:1089E0000FFC00EB40008400AFB338460AF008FCEF
:1089F00000EB4000400023185B10194D03F16002AA
:108A0000121A4FF0280E01212846C3F16004EA81B2
:108A1000A5F810E005F09CF838460AF0F1FB39465D
:108A20000246284608F0C2FA284608F0D5FA022184
:108A30000B4805F08DF8212330462B82EC810AF09B
:108A4000DFFB31460246064808F0B0FA0448BDE8AC
:108A5000F84008F0C1BA6410C4F16004004DE6E7C4
:108A6000B89FFF1F10B50D4B1B5C51F823402378B6
:108A700084B013B1012004B010BD04AA01A942F8CA
:108A8000103D2046A3699847A38A9B07F2D401A80A
:108A90000099FFF7A1FF012004B010BD9C9FFF1FAC
:108AA0002DE9F04F304DDFF8D0B0DFF8C8A00FCD82
:108AB00091B003AC0FC40FCD0FC40FCD0FC42B6802
:108AC00023600025A8462F462E4600E09846BAF8B7
:108AD000003026495BF82320DFF8A09011232846B8
:108AE000F7F76AFE00EBC00300EB8300204B83FB2B
:108AF00000340444C017C0EB6434C4F13C00C6F138
:108B00003C0207F14101012600B208F14103009047
:108B10001BB2019612B209B2484604F08FFC08EB72
:108B2000060305F211153C2B2646ADB24746CDD1C2
:108B30006B22342300214846A9F80E20A9F81030F2
:108B400005F006F80B4B1B8810AA02EB830353F8C1
:108B5000344C20460AF054FB21460246484611B0E8
:108B6000BDE8F04F08F022BAA0440100403E0100E9
:108B700009000280EE9CFF1FA43C0100B89FFF1F6C
:108B8000234B70B5B3F9003083EAE374A4EBE374CC
:108B9000002B82B0A1B234DB68466D46012300E0B1
:108BA000134603EB830252009442F9DA194E91FB0B
:108BB000F3F286FB03E403FB1211DB173032D3EB35
:108BC000A40389B205F8012BF1D119462B70FFF7E8
:108BD00003FF114B1B7813B1104B1B780BB902B07C
:108BE00070BD0F4C0121204604F0B2FF64253323F1
:108BF000204604220B49E581238208F0D7F902B010
:108C000070BD2D238DF800300DF101056846C5E7D4
:108C1000A89EFF1F676666668A9EFF1FA69EFF1FAF
:108C2000B89FFF1F6C4D010070B5404E404D82B0A3
:108C3000304604F0ABF82B78D3B93C4C06212046E3
:108C400004F086FF2B78012B38D9022B4FF003025A
:108C50004FF00A030CBF37493749E381204623828E
:108C600008F0A4F9204602B0BDE8704008F0B4B99D
:108C7000324B1A7801210523002A33D10191009348
:108C80001146304604F02AFC2D4B1A78002A34D0C5
:108C9000052301220192009300220A21234804F0B7
:108CA0009BFB284B1A78002A33D10121052301911F
:108CB000009314211D4804F011FCBEE7224B1988D3
:108CC000092930D963298CBF0A221F220A23174899
:108CD000F281338208F0D0F9144802B0BDE8704048
:108CE00008F07AB90022019100931146304604F051
:108CF00073FB134B1A78002ACAD105230121019175
:108D000000930A21094804F0E9FB0E4B1A78002A67
:108D1000CBD00122052301920093002214210348A5
:108D200004F05AFB89E73022D0E700BFB89FFF1F4D
:108D300043A0FF1F744D0100784D0100899FFF1F64
:108D40008A9FFF1F2C9FFF1F289FFF1F2DE9F047C1
:108D5000714E307848B9714B1B6899425FD3704AA5
:108D6000012313703370BDE8F0876E4D6B4F0C46D6
:108D7000284604F00BF804F6AC5331240022EC81B1
:108D80000124114628462A82AC826C823B603270F4
:108D900004F0DEFE05226449644E284608F006F918
:108DA000102728464FF00C0808F016F90B226049EE
:108DB000EF812846A5F8108008F0F8F85D490522F3
:108DC000284608F0F3F8284608F006F95A4BEF81D8
:108DD0001A68A2F69803C3EB031386FB03161E441E
:108DE000DB17C3EB662640F6CC3320219A4229825A
:108DF00006F124064FF022014FF0040011DCFFF7CA
:108E0000C9FC4E4BB3F800908246B9F1000F30D048
:108E1000B9F1010F4DD0B9F1020F47D02046BDE89E
:108E2000F087FFF717FD46490922284608F0BEF8EB
:108E30004449EF8181FB0637F317C3EBA7072A23C9
:108E4000394628462B8208F017F922463E49284623
:108E500008F0ACF807EB8701A6EB4101284608F0C3
:108E60000BF922462846394908F0A0F82046BDE80B
:108E7000F08737493A46284608F098F8284608F01F
:108E8000ABF82A232B825146EF8128462D4F08F05C
:108E9000F3F807222F49284608F088F8F31787FBD4
:108EA0000627C3EBA70739462846CCE742462A499E
:108EB000E1E742462949234C284608F077F828463E
:108EC00008F08AF82A232B8251462846EF8108F0C1
:108ED000D3F807221F49284608F068F8F31784FBE7
:108EE0000624C3EBA4042146284608F0C5F84A46E8
:108EF0001549284608F05AF804EB8401A6EB410115
:108F0000284608F0B9F84A462846104908F04EF8B5
:108F10004846BDE8F08700BF308AFF1FB49FFF1F9F
:108F2000A59FFF1FB89FFF1F7C4D01003B773B981B
:108F3000844D0100644D0100EC9EFF1F849EFF1FC5
:108F4000904D010067666666FC550100745501008E
:108F50009C4D0100B04D0100C84D0100B84D01000D
:108F60002DE9F041744C2278002A05460F4614BFC3
:108F70004FF001084FF000084ED1704E3368CB1A05
:108F8000B3F5FA6F04D86B78A3B94046BDE8F08119
:108F90006B4B6C486C49DFF8CCE11A70012303700D
:108FA0000988237026208EF8002000F049FE6B7897
:108FB000002BEAD03760F9F7B5F8644A644B65498D
:108FC000127828781B78097802EB4303421E03EBE2
:108FD00081030E2AD9D801A151F822F0C9900000CE
:108FE000959000008B8F0000C99000008B8F0000CF
:108FF0008B8F00008B8F00007D9000008B8F000016
:10900000339000008B8F00008B8F00008B8F00004F
:109010008B8F00002F900000AF214F48474E03F088
:1090200069FCFFF701FE002337602370ABE706F011
:1090300033FC494C204603F0A9FE2046022104F0EF
:1090400087FD23250F23238205224449E5812046FD
:1090500007F0ACFF204607F0BFFF1E230522404962
:1090600023822046E58107F0A1FF204607F0B4FFE8
:10907000204603F097FF00F0D5FC86E7394D2B78AA
:10908000012B50D9304B2620198800F0D9FD002340
:109090002B707AE7002B3FF478AF013B324A32F86D
:1090A0001330002B3FF471AF274C304825492D4A2F
:1090B00023804FF001080023037081F8008082F8BC
:1090C0000080FFF7B1FD60E793B1013B264A32F81B
:1090D000131019B31C4B254D1A4C224A1980002637
:1090E000012326202E702370137000F0A9FD15E0D7
:1090F000154C1E4922880B7004284FF6FF7002F1B0
:10910000FF310CBF012202460A440E4E154D02F0FB
:109110007F0201320121228031702B70FFF784FD24
:109120004FF0010831E70649064A01230020087084
:1091300013702370A6E700BF308AFF1F34A0FF1F03
:10914000A59FFF1FDD9CFF1F289FFF1F899FFF1FFB
:109150008A9FFF1F2C9FFF1FB89FFF1FD84D010044
:10916000E04D010043A0FF1F649EFF1F549DFF1FA1
:109170002DE9F04FAE4E4FF00109A6F81490A6F875
:109180001290838813EA09048BB005460F46934674
:1091900040F0AB80DFF8C48298F80030002B7BD120
:1091A000AA79A44CA35CA3B9DFF8B4A279781AF821
:1091B000029039B33B78013B072B00F2B280DFE825
:1091C00013F0EF005101B0006B01B000B000B0002F
:1091D000E7007E78002E00F0C580013BE868397812
:1091E00050F82360F0684B1E0788072B00F2A3801D
:1091F000DFE813F070015901A1006A01A100A1008C
:10920000A1009B008C4E3368C3EB0B03B3F5967F34
:1092100072D98A4B187801281ABF0120187019706A
:10922000874B18BF0146985CC0EB0900C0B2FFF73E
:1092300089F80124C6F800B0AB889B076DD57B7810
:10924000002B6AD0F8F76EFF7E4B7F4A7F481B7871
:10925000127839780078022515FB02330A2903EBCE
:10926000800300F049810C2957D1002B55D003F120
:109270001900774E774A013B0021400080B226F862
:1092800013100123157088F8003000F0D9FC724BE0
:10929000032220461A702CE0304603F077FD30465A
:1092A000494604F055FCF4813482AB88580725D434
:1092B0002C68204609F0A4FF21460246304607F0FC
:1092C00075FE304607F088FE092201238DE80C0068
:1092D00000217F23564804F0B1F800212846FFF70B
:1092E000E7FA002388F800305AE7836811463846C9
:1092F00098470BB0BDE8F08F0846FAE72B6804A842
:10930000984704A809F07CFF04A90246304607F0FC
:109310004DFE304607F060FED6E720460BB0BDE8B4
:10932000F08F00240AF8029086E70023A354304609
:10933000F3699847F0680780002425223C238DE8D4
:109340001400412118223A4804F046F8E968A87947
:10935000FFF788FB394A384B1470C3F800B00BB0E4
:10936000BDE8F08F34490B68C3EB0B03B3F5967F70
:1093700040F2E080314FC1F800B03C78012C00F0A1
:10938000AF800123E9683B701046FFF76BFBB0E745
:10939000304BE9791970012388F800300024C1E7C7
:1093A0002B7A013B4B45BCDD09F10104E4B2A14538
:1093B000B7D0234E16F802B0CBEB0900C0B20021A3
:1093C000FEF7C0FF2B7A052BD9461BD9CBEB040245
:1093D000042A40F3A980A4F1040BBBF1000FC0F2F2
:1093E000AD80063B5B45A8BF5B465FFA83F9AA796F
:1093F0001348B15C994205D000F80290012128463B
:10940000FFF756FAC9EB0400C0B201210B4EFEF77C
:1094100099FF00213423019100930B2231700448FD
:1094200040233F21A14603F0D7FF0124AA7979E721
:10943000B89FFF1F24A0FF1F20A0FF1F41A0FF1FF8
:1094400038A0FF1F899FFF1F8A9FFF1F2C9FFF1FB0
:10945000649EFF1FA59FFF1F43A0FF1F308AFF1FB1
:109460009C9FFF1F0FFA89F3E9685D4851F823B00C
:10947000036804935B499BF8003004980860002B54
:109480006CD0012B7FF44DAF57499BF8080088F84A
:1094900000300870002445E7B9F1000F4CD009F105
:1094A000FF34E4B283E7B38A03F004039BB2002BDA
:1094B0003FF43CAF336A984700283FF43BAFAB79A9
:1094C000F0680022E25436E7738ABB4240D9013784
:1094D000BFB230E7338ABB4234D2013FBFB22AE782
:1094E00025238DE8480041483E703C231822412145
:1094F00003F072FF2046FCE6002B3FF40EAF3C4A1F
:109500003C4E1188384A03F11900013B400080B2FB
:1095100026F81310012388F80030157000F090FB36
:10952000354B20461D70E4E6002A3FF75AAF04F1A0
:10953000FF3B52E73046DCE64C46F3E64FF00009CD
:109540004B4654E7B38AD9077FF5F5AE778AF2E642
:10955000B38ADA077FF5EFAE378AECE62749039343
:10956000885CC0EB090009F1010EC0B2012104F8CA
:1095700002E0FEF7E7FE039BDBF808B0019334231B
:109580001A4800930B2240233F2103F025FF0124BA
:1095900034230B228DE818003F214023134803F0A9
:1095A0009DFF2146114804F0D3FA584609F028FEE1
:1095B000A0EB800000F15F030F22F3813282584656
:1095C00009F01EFE59460246084807F0EFFC07481E
:1095D00007F002FDE968A879FFF744FAAA79A1E645
:1095E00060A0FF1F20A0FF1FA59FFF1FB89FFF1FA8
:1095F000289FFF1F649EFF1F43A0FF1F38A0FF1F6F
:109600002DE9F047DFF85C927F4B99F800601B680A
:10961000DFF854A282B0003601934FF0030018BF68
:109620000126019F9AF8008005F0CEF80546042037
:1096300005F0CAF80446052005F0C6F8800040EAA7
:109640004404062005F0C0F82C4364B26F4944EA94
:10965000C0000A7880F00F03DBB29A426C4A48D00F
:10966000176000226B480B7003788DF800808DF82E
:109670000120002B35D0684A12684EF66021BA1AD4
:109680008A4223D8022B65D0012B6BD0062B54D0F5
:10969000032B6FD0042B75D0052B00F08B80072B8C
:1096A00000F09080082B00F09580092B72D00A2BD7
:1096B00000F098800B2B00F09D800C2B72D016B11F
:1096C000564803F06FFC02B0BDE8F087544A554C91
:1096D000002301212370037013605360137289F813
:1096E00000103A4669465048FFF742FD3043C6B283
:1096F000E5E71268BA1A1E2A40F284809AF8002020
:10970000934222D0444C49488AF80030012B27600C
:1097100082EA030207609846A4D0042BA2D14348F2
:109720000068381AB0F5C87F9CD9414C2068381AB7
:10973000322897D927601A4694E73A4669463D4849
:10974000FFF716FD3043C6B2B9E7012B4FF0000218
:10975000E3D1E4E73A4669463748FFF709FD30436D
:10976000C6B2ACE73A4669463448FFF701FD3043DC
:10977000C6B2A4E73A4669463148FFF7F9FC3043E0
:10978000C6B29CE73A4669462E48FFF7F1FC3043E3
:10979000C6B294E73A4669462B48FFF7E9FC3043E6
:1097A000C6B28CE73A4669462848FFF7E1FC3043E9
:1097B000C6B284E73A4669462548FFF7D9FC3043EC
:1097C000C6B27CE73A4669462248FFF7D1FC3043EF
:1097D000C6B274E73A4669461F48FFF7C9FC3043F2
:1097E000C6B26CE73A4669461C48FFF7C1FC3043F5
:1097F000C6B264E73A4669461948FFF7B9FC3043F8
:10980000C6B25CE700222DE760A0FF1F44A0FF1F47
:10981000A89FFF1FA59FFF1F30A0FF1FB89FFF1F1E
:1098200024A0FF1F42A0FF1F344B010048A0FF1FD0
:10983000B09FFF1F644B01008C4A01005449010096
:109840001445010090540100985301002045010087
:10985000AC490100F45401001C91FF1F344A01007F
:1098600004450100308AFF1FAC9FFF1F28B110285C
:10987000044BA8BF102018607047024B01201860ED
:10988000704700BF4CA0FF1F08B5002006F0FCFE8B
:109890000028FAD108BD00BF70B50D461446064633
:1098A00005F0C2FD284605F0BFFD204605F0BCFDD1
:1098B000084B1B7813B1084B1B7803B970BD3046B9
:1098C00005F040FA284605F03DFA2046BDE8704014
:1098D00005F038BA8A9EFF1FA69EFF1F38B5164DA9
:1098E0002B78044641F6FF72A0F50050824203F146
:1098F000FF33A8BF02461B0202F5005203F4706357
:10990000100443F4604343F00E0300F4FE005204DD
:10991000184302F0FE42104306F0ECFD28680138BF
:1099200060F01F00C4F3C61204F07F01C0B2BDE8AE
:109930003840FFF7B1BF00BF4CA0FF1F70B5104EFD
:109940003378013B1B0203F47063044643F4304355
:109950000806220400F0FE4043F00B03034302F428
:10996000FE0018430D4606F0C5FD3068013860F072
:109970004F002A462146C0B2BDE87040FFF78CBFB9
:109980004CA0FF1F08B564210720FFF7D7FF7F21F8
:109990000B20BDE80840FFF7D1BF00BF70B5104EE7
:1099A0003378013B1B0203F47063044643F4104315
:1099B0000806220400F0FE4043F00903034302F4CA
:1099C000FE0018430D4606F095FD3068013860F042
:1099D0006F002A462146C0B2BDE87040FFF75CBF69
:1099E0004CA0FF1F38B50E4D2B78013B1B0203F432
:1099F0007063044643F41043000443F0090300F489
:109A0000FE00184306F076FD2868013860F06F000C
:109A10002146C0B20022BDE83840FFF73DBF00BF7D
:109A20004CA0FF1F10B500217B20FFF787FF00240B
:109A3000E0B2FFF7D7FF0134022004F0FBFE802CD8
:109A4000F6D110BD38B50C46054605F0EDFC2046B4
:109A500005F0EAFC074B1B7813B1074B1B7803B9E1
:109A600038BD284605F06EF92046BDE8384005F0BF
:109A700069B900BF8A9EFF1FA69EFF1F38B50D4D16
:109A80002B78013B1B0203F47063044643F45043FC
:109A9000000443F00D0300F4FE00184306F02AFD15
:109AA0002868013860F02F002146C0B2BDE8384078
:109AB000FFF7C8BF4CA0FF1F38B50E4D2B78013BF8
:109AC00001381B02C4B203F47063200443F4404322
:109AD00043F00C0300F4FE00184306F00BFD286869
:109AE000013860F03F002146C0B2BDE83840FFF7C2
:109AF000A9BF00BF4CA0FF1F38B504460D46F0209B
:109B000005F092FC35B1254414F8010B05F08CFCEE
:109B1000AC42F9D1F720BDE8384005F085BC00BF64
:109B200000B50B4B83B00246998818680090032A51
:109B3000ADF8041002D903B05DF804FB68460621B5
:109B40008DF80520FFF7D8FF03B05DF804FB00BFD8
:109B50003455010000B50B4B024683B01868998854
:109B60000090131F4C2BADF8041002D903B05DF820
:109B700004FB684606218DF80520FFF7BDFF03B002
:109B80005DF804FB3C550100030203F4FE43C0F3FF
:109B9000C6101843704700BF03784078DB0103F418
:109BA0007E5300F07F001843704700BF82B002AAC6
:109BB000114642F8040D002012F8013B03F07F0328
:109BC000914243EA0020F7D102B0704710B547F642
:109BD000122104460D4807F0A3F805F045FC0C4B94
:109BE0001B7833B974B1102C0A4BA8BF10241C6029
:109BF00010BD47F61221084806F0E2FF05F05EF9B5
:109C0000002CF0D1034B01241C6010BD4C93FF1FAE
:109C10008A9EFF1F4CA0FF1F3893FF1F003210B415
:109C200003884FF0010404FA01F418BF012202FA7C
:109C300001F123EA04020A43028010BC704700BF0E
:109C400070B5CEB20C46054604F04EFA864203D0FB
:109C50003146284604F062FA0135284604F044FAF9
:109C6000240A844205D021462846BDE8704004F00D
:109C700055BA70BD38B5054604F036FA4FF0000409
:109C800060F30704681C04F02FFA60F30F24A0B2FD
:109C900038BD00BFF8B504460020FFF7EBFF002CED
:109CA00000F087814FF4AF610220FFF7C9FF042065
:109CB0004FF47A61FFF7C4FF0B2004F085FD002804
:109CC00040F085874FF496610620FFF7B9FF4FF407
:109CD000FA610820FFF7B4FF4FF4FA610A20FFF79A
:109CE000AFFF40F6B8310C20FFF7AAFF4FF42F6109
:109CF0002220FFF7A5FF40F6AC512420FFF7A0FF7C
:109D00007D212A20FFF79CFF0C210E20FFF798FFF2
:109D100001211020FFF794FF02211220FFF790FF8E
:109D200000211420FFF78CFF00211620FFF788FF89
:109D300002211820FFF784FF01211A20FFF780FF7E
:109D400001211C20FFF77CFF04211E20FFF778FF74
:109D500014212020FFF774FF01212620FFF770FF58
:109D600003212820FFF76CFF04212C20FFF768FF58
:109D700014212E20FFF764FF00213020FFF760FF41
:109D80000C213220FFF75CFF00213420FFF758FF41
:109D900000213620FFF754FF00213820FFF750FF45
:109DA00000213A20FFF74CFF00213C20FFF748FF3D
:109DB00000213E20FFF744FF00214020FFF740FF35
:109DC00000214220FFF73CFF1F214420FFF738FF0E
:109DD00013214620FFF734FF0E214820FFF730FF04
:109DE00011214A20FFF72CFF0A214C20FFF728FF02
:109DF00000214E20FFF724FF06215020FFF720FF0F
:109E000002215220FFF71CFF0C215420FFF718FFFE
:109E100000215620FFF714FF00215820FFF710FF04
:109E200001215A20FFF70CFF08215C20FFF708FFF3
:109E30000F215E20FFF704FF00216020FFF700FFE5
:109E400004216220FFF7FCFE01216420FFF7F8FEE9
:109E500000216620FFF7F4FE0B216820FFF7F0FEDB
:109E60007F216A20FFF7ECFE00216C20FFF7E8FE5F
:109E700000216E20FFF7E4FE00217020FFF7E0FED6
:109E800000217220FFF7DCFE00217420FFF7D8FECE
:109E90001F217620FFF7D4FE13217820FFF7D0FE94
:109EA0000E217A20FFF7CCFE11217C20FFF7C8FE9F
:109EB0000A217E20FFF7C4FE1F218020FFF7C0FE8D
:109EC00013218220FFF7BCFE0E218420FFF7B8FE8D
:109ED00011218620FFF7B4FE0A218820FFF7B0FE8B
:109EE00000218A20FFF7ACFE00218C20FFF7A8FE9E
:109EF00000219620FFF7A4FE00219820FFF7A0FE86
:109F000000219A20FFF79CFE05219C20FFF798FE78
:109F100006219E20FFF794FE0021A020FFF790FE6F
:109F20007F21A220FFF78CFE40F2A461A420FFF75E
:109F300087FE4FF4E161A620FFF782FE0021A820F2
:109F4000FFF77EFE0021AA20FFF77AFE0221AC2057
:109F5000FFF776FE0121AE20FFF772FE0121B0204F
:109F6000FFF76EFE0B21B220FFF76AFE6421B420DA
:109F7000FFF766FE6421B620FFF762FE0321B820DA
:109F8000FFF75EFE0121BA20FFF75AFE2D210020C7
:109F9000FFF756FE0220FFF76DFEB0F5805F034627
:109FA00016D34FF4AF610220FFF74AFE4FF4AF63C0
:109FB0000EE04FF6FF7398423FF474AE2D2840F048
:109FC00012860220FFF756FEB0F5805F0346E8D206
:109FD000D24A04201380FFF74DFEB0F5805F0346A0
:109FE00080F0E085CE4A06201380FFF743FEA0F5FF
:109FF0002F739BB2B3F57A6F024606D940F628213B
:10A000000620FFF71DFE40F62822C64B08201A80C6
:10A01000FFF730FEA0F52F739BB2B3F57A6F0246BF
:10A0200006D940F6E4410820FFF70AFE40F6E44274
:10A03000BD4B0A201A80FFF71DFEA0F5FA739BB2F4
:10A0400040F6AC518B42024606D94FF4FA610A2021
:10A05000FFF7F6FD4FF4FA62B44B0C201A80FFF7BD
:10A0600009FEA0F5FA739BB240F6AC518B42024652
:10A0700006D940F6B8310C20FFF7E2FD40F6B832C1
:10A08000AB4B0E201A80FFF7F5FD1828034600F2AF
:10A090008285A84A10201380FFF7ECFD431E9BB277
:10A0A0000F2B024604D901211020FFF7C9FD012220
:10A0B000A14B12201A80FFF7DDFD0A28034600F2AB
:10A0C00063859E4A14201380FFF7D4FD01280346C0
:10A0D00004D900211420FFF7B3FD0023984A16206D
:10A0E0001380FFF7C7FD7F28034600F24685954A97
:10A0F00018201380FFF7BEFD0528034600F23685C1
:10A10000914A1A201380FFF7B5FD0C28034600F290
:10A1100026858E4A1C201380FFF7ACFD04280346D9
:10A1200000F216858A4A1E201380FFF7A3FD092836
:10A13000034600F20685874A20201380FFF79AFD28
:10A140004628034600F2F684834A22201380FFF754
:10A1500091FDA0F5FA739BB240F6AC518B420246DA
:10A1600006D94FF42F612220FFF76AFD4FF42F62CA
:10A170007A4B24201A80FFF77DFDA0F5FA739BB27D
:10A1800040F6AC54A342024604D921462420FFF7EE
:10A1900057FD2246724B26201A80FFF76BFD7F2861
:10A1A000034600F2C0846F4A28201380FFF762FD47
:10A1B0000628034600F2B0846B4A2A201380FFF77A
:10A1C00059FDA0F132039BB2B3F5967F024604D944
:10A1D0007D212A20FFF734FD7D22644B2C201A803C
:10A1E000FFF748FD0C28034600F28F84604A2E20BA
:10A1F0001380FFF73FFD1E28034600F27F845D4A6F
:10A2000030201380FFF736FD0928034600F248840A
:10A21000594A32201380FFF72DFD1F28034600F214
:10A220003884564A34201380FFF724FD7F280346E4
:10A2300000F22884524C36202380FFF71BFD7F2834
:10A24000034600F2188438206380FFF713FD7F284F
:10A25000034600F209843A20A380FFF70BFD7F2814
:10A26000034600F2FA833C20E380FFF703FD7F28DA
:10A27000034600F2EC833E202381FFF7FBFC7F289E
:10A28000034600F2DE8340206381FFF7F3FC7F2862
:10A29000034600F2D0834220A381FFF7EBFC394D47
:10A2A00028804420FFF7E6FC3028034600F2BD83F7
:10A2B000354A46201380FFF7DDFC3028034600F2C4
:10A2C000AE83324C48202380FFF7D4FC302803466D
:10A2D00000F29F834A206380FFF7CCFC30280346BE
:10A2E00000F291834C20A380FFF7C4FC3028034682
:10A2F00000F283834E20E380FFF7BCFC0128034675
:10A3000004D900214E20FFF79BFC0023204A502057
:10A310001380FFF7AFFC431E3CE000BF8C9DFF1F86
:10A32000569FFF1F3C9DFF1F249FFF1FF09EFF1F96
:10A33000009DFF1FCE9CFF1FA89EFF1FDA9EFF1FE0
:10A34000829DFF1FD49CFF1F929DFF1F209DFF1F1A
:10A35000189DFF1F089DFF1F369FFF1FA49EFF1F14
:10A36000A09EFF1F289FFF1FFE9EFF1F4E9FFF1FE7
:10A37000EE9CFF1F709DFF1F649FFF1F269FFF1F06
:10A38000649EFF1F589FFF1FFA9CFF1F009FFF1F27
:10A39000169DFF1F9BB20B2B024604D906215020AD
:10A3A000FFF74EFC0622CF4B52201A80FFF762FCCB
:10A3B0000428034600F21B83CB4A54201380FFF786
:10A3C00059FC431E9BB21D2B024604D90C2154207C
:10A3D000FFF736FC0C22C54B56201A80FFF74AFCCB
:10A3E0000128034604D900215620FFF729FC002349
:10A3F000BF4A58201380FFF73DFC7F28034600F238
:10A40000F082BC4A5A201380FFF734FC431E9BB2F3
:10A41000092B024604D901215A20FFF711FC012221
:10A42000B54B5C201A80FFF725FC431E9BB2102B16
:10A43000024604D908215C20FFF702FC0822AF4B3A
:10A440005E201A80FFF716FC431E9BB21D2B0246AE
:10A4500004D90F215E20FFF7F3FB0F22A84B6020E9
:10A460001A80FFF707FC0228034600F2B482A54ACF
:10A4700064201380FFF7FEFB0128034604D9012165
:10A480006420FFF7DDFB01239F4A62201380FFF762
:10A49000F1FBC31E9BB2012B024604D904216220AA
:10A4A000FFF7CEFB0422994B66201A80FFF7E2FBF0
:10A4B0007F28034600F28982954A68201380FFF7BF
:10A4C000D9FB7F28034600F27A82924A6A201380E1
:10A4D000FFF7D0FB7F28034600F26B828E4A6C2088
:10A4E0001380FFF7C7FB0328034600F25C828B4A08
:10A4F0006E201380FFF7BEFB1928034600F24D8241
:10A50000874A70201380FFF7B5FB0228034600F24C
:10A510003E82844A72201380FFF7ACFB0628034674
:10A5200000F22F82804A74201380FFF7A3FB0728D4
:10A53000034600F220827D4A8A201380FFF79AFBAF
:10A540000A28034600F21182794A8C201380FFF713
:10A5500091FB0428034600F20282764A9820138079
:10A56000FFF788FB0128034604D900219820FFF754
:10A5700067FB0023704A9A201380FFF77BFB0128BA
:10A58000034604D900219A20FFF75AFB00236B4AA7
:10A5900096201380FFF76EFB0B28034600F2D9814B
:10A5A000674A9C201380FFF765FB831E9BB2032B39
:10A5B000024604D905219C20FFF742FB0522614B8E
:10A5C00076201A80FFF756FB3028034600F2BB8145
:10A5D0005D4A78201380FFF74DFB3028034600F2D8
:10A5E000AC815A4C7A202380FFF744FB3028034685
:10A5F00000F29D817C206380FFF73CFB30280346FE
:10A6000000F28F817E20A380FFF734FB30280346C1
:10A6100000F281818020E380FFF72CFB3028034685
:10A6200000F273814A4A82201380FFF723FB30280F
:10A63000034600F26481474C84202380FFF71AFB15
:10A640003028034600F2558186206380FFF712FB15
:10A650003028034600F247818820A380FFF70AFBD9
:10A660003028034600F23981A020E380FFF702FB87
:10A670000128034604D90021A020FFF7E1FA0023B6
:10A68000354A9E201380FFF7F5FAC31E9BB20C2BB0
:10A69000024604D906219E20FFF7D2FA06222F4B4C
:10A6A000A2201A80FFF7E6FA431E9BB27E2B0246D9
:10A6B00004D97F21A220FFF7C3FA7F22284BA420D0
:10A6C0001A80FFF7D7FAA0F5AF639BB2B3F5167FF8
:10A6D000024647D940F2A461A420FFF7B1FA40F244
:10A6E000A4623FE03689FF1F4889FF1FC489FF1F0E
:10A6F0005E9DFF1FEA9EFF1FC89CFF1FC889FF1FAA
:10A700004089FF1F9C9EFF1FF89EFF1F289DFF1F73
:10A71000389FFF1F5C9DFF1F0C9DFF1FBC9CFF1FF0
:10A720008C9FFF1F849EFF1F609FFF1F1C9FFF1FAA
:10A73000AA9EFF1F949EFF1F0A9DFF1F689DFF1F7B
:10A74000E49EFF1FF09CFF1F029DFF1F749EFF1FD2
:10A75000049DFF1F7C9EFF1F089FFF1FB089FF1FE6
:10A760002A9FFF1FD24BA6201A80FFF783FAA0F57D
:10A77000AF639BB2B3F5167F024606D94FF4E16191
:10A78000A620FFF75DFA4FF4E162CA4BA8201A80B9
:10A79000FFF770FA0628034600F29980C64AAA20FD
:10A7A0001380FFF767FA0328034600F28A80C34A42
:10A7B000AC201380FFF75EFA032803467BD8C04A1B
:10A7C000B0201380FFF756FA032803466DD8BD4A20
:10A7D000AE201380FFF74EFA7F2803465FD8BA4AAF
:10A7E000B2201380FFF746FA7F28034651D8B74AB4
:10A7F000B4201380FFF73EFA431E9BB2C62B0246DD
:10A8000004D96421B420FFF71BFA6422B04BB620B0
:10A810001A80FFF72FFA431E9BB2C62B024604D9BB
:10A820006421B620FFF70CFA6422AA4BB8201A80E4
:10A83000FFF720FA0828034600F2C381A64ABA208F
:10A840001380FFF717FA032800F2B5812B88DFF891
:10A85000A8E2A24FA24AA34DA34EA44CA44903F0E0
:10A86000010CAEF800C0C3F3400EA7F800E0C3F33C
:10A8700080071780C3F3C0079E4A2F70C3F30017E9
:10A88000C3F34015C3F38013378025800B801080FD
:10A89000F8BD0B21B220FFF7D3F90B23A7E7012165
:10A8A000AE20FFF7CDF9012399E70121B020FFF792
:10A8B000C7F901238BE70221AC20FFF7C1F902237E
:10A8C0007DE70021AA20FFF7BBF900236FE70021F5
:10A8D000A820FFF7B5F9002360E70A218820FFF7D9
:10A8E000AFF90A23C0E611218620FFF7A9F9112349
:10A8F000B2E60E218420FFF7A3F90E23A4E613216C
:10A900008220FFF79DF9132395E61F218020FFF792
:10A9100097F91F2386E60A217E20FFF791F90A2383
:10A9200078E611217C20FFF78BF911236AE60E21CE
:10A930007A20FFF785F90E235CE613217820FFF7D4
:10A940007FF913234DE61F217620FFF779F91F23A6
:10A950003EE600219620FFF773F9002320E6002150
:10A960008C20FFF76DF90023F7E500218A20FFF71F
:10A9700067F90023E8E500217420FFF761F900235F
:10A98000D9E500217220FFF75BF90023CAE5002119
:10A990007020FFF755F90023BBE500216E20FFF77B
:10A9A0004FF90023ACE500216C20FFF749F90023A3
:10A9B0009DE57F216A20FFF743F97F238EE50B2178
:10A9C0006820FFF73DF90B237FE500216620FFF7A4
:10A9D00037F9002370E500216020FFF731F90023EB
:10A9E00045E500215820FFF72BF9002309E5022156
:10A9F0005220FFF725F90223DEE40A214C20FFF75D
:10AA00001FF90A2376E411214A20FFF719F91123CF
:10AA100068E40E214820FFF713F90E235AE41321AE
:10AA20004620FFF70DF913234BE41F214420FFF7C5
:10AA300007F91F233CE400214020FFF701F9002320
:10AA400029E400213E20FFF7FBF800231BE400214E
:10AA50003C20FFF7F5F800230DE400213A20FFF732
:10AA6000EFF80023FFF7FFBB00213820FFF7E8F8DD
:10AA70000023FFF7F0BB00213620FFF7E1F80023A9
:10AA8000FFF7E1BB00213420FFF7DAF80023FFF7DE
:10AA9000D1BB0C213220FFF7D3F80C23FFF7C1BB49
:10AAA00000213020FFF7CCF80023FFF7B1BB00BF37
:10AAB000909DFF1F109FFF1FCA9CFF1F409DFF1FFF
:10AAC000FA9EFF1F889EFF1F149DFF1F329DFF1FD0
:10AAD0004C9FFF1F789FFF1FD09CFF1F389DFF1FBB
:10AAE000749DFF1FA69EFF1F9E9EFF1F3A9DFF1F86
:10AAF000AE9EFF1F729EFF1FE69EFF1F14212E2099
:10AB0000FFF79EF81423FFF77ABB04212C20FFF7F0
:10AB100097F80423FFF76ABB03212820FFF790F87A
:10AB20000323FFF749BB01212620FFF789F8012302
:10AB3000FFF739BB14212020FFF782F81423FFF719
:10AB400003BB04211E20FFF77BF80423FFF7F3BAB1
:10AB500001211C20FFF774F80123FFF7E3BA01215C
:10AB60001A20FFF76DF80123FFF7D3BA022118204E
:10AB7000FFF766F80223FFF7C3BA00211620FFF79C
:10AB80005FF80023FFF7B3BA02211220FFF758F84D
:10AB90000223FFF796BA0C210E20FFF751F80C2381
:10ABA000FFF777BA4FF47A610420FFF749F84FF4C2
:10ABB0007A63FFF717BABA200121FFF741F80120A5
:10ABC00044E60321B820FFF73BF8032336E640F6BE
:10ABD00028210620FFF734F840F6E4410820FFF76B
:10ABE0002FF8FFF779B817287FF65CA819287FF6A9
:10ABF000CBA81B287FF6E8A81C283FF4FDA81E2838
:10AC00007FF602A91F283FF407A920283FF420A9B6
:10AC100021283FF429A922283FF42EA923283FF414
:10AC200037A924283FF468A925283FF46DA92628D0
:10AC30003FF46EA927283FF473A928283FF47EA982
:10AC400029283FF483A92A283FF490A92B283FF410
:10AC500095A92C287FF49AA9FFF794B9F8B5CD20CF
:10AC600007F032FD204B214A054603CB1368C5F897
:10AC700003001A0CBC20C5F807102B80AA70FEF741
:10AC800083FF2E46002426F80B0FA0B2FEF7F2FF3A
:10AC9000FEF77AFF0234BC2C26F8020FF5D16C1EA9
:10ACA00005F1C8064FF0FF3014F8013F082758405F
:10ACB0000F4B40F300017A1E0B4012F0FF0783EAAE
:10ACC0005000F5D1B442EFD1C043FEF76FFF3A46D2
:10ACD000C5F8C900CD21284605F05AFC2846BDE834
:10ACE000F84007F0F9BC00BF485501004455010089
:10ACF0002083B8EDF0B50E4B0E4C054693E80700E7
:10AD000085B024682E88AD7801AB83E80700270C56
:10AD1000184600220B21ADF804408DF80670ADF8FE
:10AD20000C608DF80E5005F033FC05B0F0BD00BF8F
:10AD30005455010044550100F0B5124B124D1E68E8
:10AD4000124F0FCD87B06C460FC495E8030044F84E
:10AD5000040B38683B79CDF80D00320C2D20218092
:10AD60008DF802208DF81130ADF80060FEF70CFF71
:10AD70000022ADF80B001221684605F009FC07B06F
:10AD8000F0BD00BF4455010060550100644D010055
:10AD9000002005F079BC00BF03F05EB970B5104C1F
:10ADA00082B000254023064629462046009301959F
:10ADB0008023202202F010FB012320223046228231
:10ADC000A3826382E58108F01BFA314602462046E1
:10ADD00006F0ECF8204602B0BDE8704002F0E2B8A0
:10ADE000B89FFF1FF0B5CC2983B075D90546441E26
:10ADF00000F1C8064FF0FF3014F8012F082750402B
:10AE0000404A40F300017B1E0A4013F0FF0782EA2C
:10AE10005000F5D1B442EFD1C043FEF7C7FE014662
:10AE2000D5F8C9000190019A914202D0B2F17F2F6A
:10AE30000BD105F10B00FEF7AFFEBC280BD032485A
:10AE4000FFF7ACFF002003B0F0BD3048FFF7A6FFCE
:10AE5000384603B0F0BD05F10D00FEF79DFE2D282C
:10AE600040D1002440F6AC5613E004281AD006283E
:10AE700021D008281FD00A2828D00C2822D1A1F5DB
:10AE8000FA7292B2B24201D8FEF7DAFE0234BC2C5A
:10AE90000ED004F10D002844FEF77EFE022C014680
:10AEA000A0B2E2D1B1F5805FEED30234BC2CF0D178
:10AEB000012003B0F0BDA1F52F7292B2B2F57A6F06
:10AEC000E4D8E1E7222801D0242811D1A1F5FA72B3
:10AED00092B2B242DAD8D7E70D48FFF75FFF002001
:10AEE00003B0F0BD0B48FFF759FF002003B0F0BDE1
:10AEF0002A28C9D1A1F1320292B2B2F5967FC5D803
:10AF0000C2E700BF2083B8EDA455010090550100B1
:10AF100078550100B855010003290CD970B5461CBD
:10AF200082B005460C46304603222A4908F0D6F97D
:10AF300010B102B070BD70470B2C05D9052226490F
:10AF4000281D08F0CBF940B12448FFF727FF24481B
:10AF500002B0BDE87040FFF7CDBE05F10901032244
:10AF600001A808F00BFA01A803221E4908F0B6F95F
:10AF7000D8B103221C4901A808F0B0F908B301A810
:10AF800003221A4908F0AAF9B0B91948FFF706FFD9
:10AF9000A11E89B23046FFF725FF0028C9D0154809
:10AFA00002B0BDE87040FFF7F9BE1348FFF7F6FEA8
:10AFB000FFF754FE1148F3E71148FFF7EFFE114881
:10AFC000C6E71148FFF7EAFE02B0BDE87040FFF7A0
:10AFD000B3BE00BF445501007C4D0100D0550100B7
:10AFE000E4550100E8550100105601002856010003
:10AFF0002C56010040560100EC550100005601009E
:10B000005456010068560100145601002DE9F04322
:10B01000174D2B6883B081460F469046F3B1154E0D
:10B0200034880A1992B218461146328007F0CAFED7
:10B0300028603A464946204402F092FDB8F1000FDC
:10B0400009D031882868FFF767FF286807F044FBBC
:10B0500000232B60338003B0BDE8F083054E0193DD
:10B060000846318007F030FB019B28601C46E0E772
:10B0700054A0FF1F50A0FF1F10B51D4C4FF4FA70D5
:10B08000FBF714FC204601F081FE00231946012243
:10B090002046E3812382A282628202F059FD0B22C4
:10B0A0001449204605F082FF204605F095FF0F2247
:10B0B0001149204605F07AFF204605F08DFF0F4923
:10B0C0000722204605F072FF204605F085FF204646
:10B0D00001F068FF0A4B0B4A1A604FF4FA70FBF755
:10B0E000E5FBFFF729FE0848BDE81040FFF756BE14
:10B0F000B89FFF1F6C56010078560100885601006A
:10B1000068A2FF1F0DB0000090560100002070479C
:10B1100090F8392090F83800101A704790F83830BD
:10B1200090F839209A4205D95A1C034480F83820F7
:10B13000187E70474FF0FF30704700BF90F83830EE
:10B1400090F839209A4286BF1B18187E4FF0FF30C6
:10B15000704700BF704700BF38B50546B0F85E00C5
:10B1600090B195F85D301446C3F1210294420CD899
:10B1700005F13B001844224602F0F2FC95F85D30E0
:10B18000234485F85D30204638BD012014462871DF
:10B19000EEE700BFB0F85E306BB190F85D30202B69
:10B1A00007D8C218013380F85D30012082F83B10C7
:10B1B0007047012303710020704700BF00234269DC
:10B1C00080F8383080F8393080F85C3080F85D30B5
:10B1D00080F85E3080F85F3006CA30B40D680469CC
:10B1E00043662A4383660A60A370426990F861301F
:10B1F0001649146813441D7A5B7B01EBC5051B02DD
:10B200006D6803F4E06343F064032B6090F86230F0
:10B2100013449D7CDB7D01EBC5011B02496803F4EF
:10B22000E06343F064030B6021685368194205D062
:10B23000036927225A70036904229A710369202244
:10B240005A71036980229A7030BC7047B461010062
:10B2500043690CCB12681A420CD0094B99420AD9A7
:10B26000084B9942036994BF1A220D225A70036950
:10B2700004229A717047036927225A70F7E700BFCA
:10B280007F1A06003F420F0010B50269D378DBB287
:10B29000D90604463DD510215806D17038D503F0A3
:10B2A000040303F0FF02002B51D03D49626E0023DE
:10B2B0000B7084F85D30002A5BD0904794F85D30C5
:10B2C000002B56D02369D0229A70236994F83B2032
:10B2D0001A712369012284F85C200222DA7010BD01
:10B2E000304B84F860009C424AD02F4B9C4252D095
:10B2F00094F8391013791F29DBB207D82848007851
:10B3000020B16018013184F8391003760223D3701C
:10B3100010BD5906C3D4917801F0100101F0FF006F
:10B320000029DDD013F001031ED194F85C1094F8CD
:10B330005D00884281BF4B1C091984F85C3091F88C
:10B340003B3013712369D0229A702269DEE72369AA
:10B3500084F83920C0229A702369114A1979012191
:10B3600011700222DA7010BDC02393702269137924
:10B37000CCE70122002384F85D2084F83B30A1E76C
:10B38000626994F86130094913440322187A02F083
:10B39000B3FF2269ACE7626994F861300449F3E7CE
:10B3A00058A0FF1F7091FF1FDC91FF1F11B4000018
:10B3B0001DB400000369DB7803F0200373B190F83B
:10B3C00060300133DBB2012B80F860301AD942695A
:10B3D00090F861301344187A03F00AB870B54269E6
:10B3E00003F0FF0590F8613013440446187A02F028
:10B3F000FFFFA36E5BB184F8385094F83900BDE8C4
:10B400007040184790F85F30002BE0D0704770BD57
:10B410000148FFF7CFBF00BF7091FF1F0148FFF742
:10B42000C9BF00BFDC91FF1F2DE9F047374FDFF8A0
:10B43000E0903B68026982B006460093DDF8008028
:10B440000021A025D3789B065BD53B680193019B27
:10B45000C8EB03030F2BF5D949B1102BF2D0002014
:10B460009070336980229A7002B0BDE8F0877269EB
:10B4700096F8613013440521187A03F0B3F9726924
:10B4800096F861301344012193F812A0504603F05E
:10B49000A9F909240021504603F090F92B46013BFD
:10B4A000FDD10121504603F089F92B46013BFDD126
:10B4B000013CEFD1706996F8611001444FF4A0721D
:10B4C0000C7A4B7B09EBC4011B02496803F4E0636F
:10B4D00043F064030B6096F862300344997CDB7D93
:10B4E00009EBC1011B02496803F4E06343F0640304
:10B4F0000B60013AFDD13269D3789B064FF0010110
:10B50000A3D4012002B0BDE8F08700BF60A0FF1FF8
:10B51000B4610100F0B503691222DA700269937810
:10B5200003F0200385B004460D46002B5ED0B42303
:10B5300093703C4922690B680093009E05E00B68FC
:10B540000193019B9B1B042B42D8D37803F020036B
:10B5500003F0FF00002BF2D094F85D30002B31D0C7
:10B560004FF0000E4FF0020C04EB0E0393F83B304B
:10B5700013710B680393039F206907E09B060DD5A9
:10B580000B680293029BDB1B052B28D8C378DBB228
:10B5900003F0020202F0FF06002AEFD080F803C099
:10B5A0002669F378DBB2DF0632462DD49F062BD511
:10B5B000DB0731D40EF1010E94F85D305FFA8EFE98
:10B5C0007345D1D800201DBB002384F85E3004E011
:10B5D0009070236980229A70042005B0F0BD8670B7
:10B5E0002369802204209A7005B0F0BD03F0FF06A5
:10B5F000FFF71AFF10B9042005B0F0BD236984F8E5
:10B600005F60B0229A7094E78023B3700420DAE779
:10B6100026698023B370D7E7BEF1000F0CBF02206C
:10B620000320F6E760A0FF1F2DE9F0410669002521
:10B63000122780F8385080F83950F770D0F810C0D1
:10B640009CF802E00EF0200E88B0044688461546AD
:10B650001E46BEF1000F49D0B4238CF80230784B5F
:10B6600021691A680092DDF800E006E01A6801928C
:10B670000198CEEB0000042830D8C87800F02000F4
:10B6800000F0FF070028F1D04FEA480242F0010223
:10B69000D2B20A711A680292DDF808E0206906E069
:10B6A0001A6803920399CEEB010105292AD8C178C3
:10B6B00001F0020101F0FF070029F1D04FF0020C68
:10B6C00080F803C02269D17811F0110722D12DBB77
:10B6D000002E0CBFA0238023937003E08F7023699A
:10B6E00080229A70384608B0BDE8F0810EF0FF075E
:10B6F000FFF79AFE0028F5D0236984F85F70B02226
:10B700009A70ACE787702369802238469A7008B037
:10B71000BDE8F081802393700027E3E7012D75D009
:10B72000A021917021690A79BE4667464FF0A80CA6
:10B730001A680492049805E01A680592059A121A8C
:10B74000052A4AD8CA7802F0020202F0FF08002A4D
:10B75000F2D0CF702169CA78D2B212F0100F084629
:10B760005AD1920658D5013DEDB2012D49D0BEF116
:10B770001F0F3BD90A79012DDAD11A680692069D6E
:10B7800005E01A680792079A521B052A46D8C27824
:10B7900002F0020202F0FF01002AF2D00223C3707D
:10B7A0002269D378DBB2D9063AD49B0634D5B023CC
:10B7B000BEF11F0F93703FD8226904EB0E0312797C
:10B7C0001A760EF1010E5FFA8EFE16B12369802201
:10B7D0009A7084F839E0774684E781F8028023691B
:10B7E00080229A70774684F839E07BE704EB0E02FA
:10B7F00091F8048082F818800EF1010E5FFA8EFE37
:10B80000B9E781F802C021690846B0E7A821917024
:10B810002069BE460279B0E7774663E78170DEE7CC
:10B820001021A023D170013BFDD12269937803F050
:10B83000F7037746937055E723691B79C5E700BF87
:10B8400060A0FF1F0148FFF71FBD00BF7091FF1FE1
:10B850000148FFF719BD00BFDC91FF1F0022026005
:10B86000704700BF30B5056889B0012300240A463F
:10B870000193294602A8009400F006F902A800F0FE
:10B88000ADF9C0B209B030BD30B5056889B001244A
:10B8900000230A468DE818002946022302A800F07A
:10B8A000F3F802A800F09AF980B209B030BD00BFE9
:10B8B0000C2901D9002070470231490001F0FE0136
:10B8C000FFF7E2BF2DE9F04303688FB001260024A3
:10B8D0000D4607461946904633465E2202A8019659
:10B8E000009400F0D1F802A800F078F95E2D03D0A2
:10B8F000A5F17303072B10D80123002439680193A5
:10B900002A4608A8009400F0BFF82246414608A83D
:10B9100000F006F90FB0BDE8F083814622462146CB
:10B9200002A800F0FDF8396833462A468DE8500039
:10B9300008A800F0A9F82246414608A800F0F0F84F
:10B9400022465FFA89F102A800F0EAF80FB0BDE8DC
:10B95000F08300BFF8B505460F4616464124214640
:10B960003A462846FFF7AEFF611C0234C9B23246A0
:10B970002846E4B2FFF7A6FF592CF0D1F8BD00BF6E
:10B980002DE9F843044600689DF820900E461746BE
:10B99000984610B1102105F081FB102005F07CFBCA
:10B9A0003A460546314600F057F925602846012100
:10B9B00000F078F9054618B900252846BDE8F88357
:10B9C000632280212046FFF77DFF012002F032FF35
:10B9D00000225E212046FFF775FF5D212046FFF71C
:10B9E00041FF2428E8D14A4641462046FFF7B2FFEE
:10B9F000204601222B21FFF765FF204601222C2142
:10BA0000FFF760FF20460E222D21FFF75BFF204647
:10BA100000222E21FFF756FF204601222F21FFF79B
:10BA200051FF204605223021FFF74CFF204601221E
:10BA30003121FFF747FF204600223221FFF742FF66
:10BA4000204600223321FFF73DFF2046002234210B
:10BA5000FFF738FF204600223521FFF733FF20464D
:10BA600000225B21FFF72EFF204610225C21FFF70A
:10BA700029FF204620225D21FFF724FF20468C224B
:10BA80005E21FFF71FFF98E770B49DF810609DF8E6
:10BA90000C5001600021467385734281037341613C
:10BAA000416070BC704700BFF0B54389056885B040
:10BAB000DCB21B128DF80C408DF80D304DB1437B7C
:10BAC000019303AB00932846012300F0FBF805B077
:10BAD000F0BD43680BB31746027A0E466AB904F00C
:10BAE0007F048DF80C40427B009231463A4618465E
:10BAF00003AB00F055FA05B0F0BD022A04D164F0A2
:10BB00007F048DF80C40EEE7012AECD104F07F04AD
:10BB100044F040048DF80C40E5E71846D7E700BF35
:10BB200002B9027B042A1AD8F0B4416100F10F0770
:10BB30007AB102F10E03867B3C46034400F10E0508
:10BB40005EB92170013BAB424FEA112104F10104BF
:10BB5000F6D13946F0BCFFF7A7BF1970F2E7002015
:10BB6000704700BF70B54489066884B0E5B22412FE
:10BB70008DF80C508DF80D405EB1437B009200248F
:10BB80001A4630460B46019403A900F00BF904B0A5
:10BB900070BD4468FCB1037A7BB965F07F058DF810
:10BBA0000C50437B0092FF251A4620460B46019518
:10BBB00003A900F08BFA04B070BD022B04D105F08C
:10BBC0007F058DF80C50ECE7012B04BF65F03F05B5
:10BBD0008DF80C50E5E72046D9E700BF38B500F1F5
:10BBE0000F042146027B0546FFF7BCFF10B94FF05A
:10BBF000FF3038BD287B0028FBD00E302B18AA7BE5
:10BC000021460E35002007E01C78013BAB4240EA9C
:10BC1000040001F101010AD00002002AF4D00C78DE
:10BC2000013BAB4240EA040001F10101F4D138BD0F
:10BC300070B5044640681E4603685B681546984721
:10BC4000854201D0002070BD31466068FFF762FC7C
:10BC5000B0FA80F0400970BD30B400252024057290
:10BC6000C4600170426030BC704700BF037A10B5F9
:10BC7000044683B1227863680121520083F83B2097
:10BC800083F85E1083F85D106068FFF743FCB0FA3C
:10BC900080F0400910BD012100F004F80028E9D12E
:10BCA00010BD00BF38B5044640680D46FFF786FA60
:10BCB0000120207205B938BD2046BDE83840FFF7A5
:10BCC000D5BF00BF2DE9F041079EC468DDF818E03C
:10BCD0009519A54219D815460278984643680F462B
:10BCE00052000121044683F83B2083F85E1083F85C
:10BCF0005D106EB1BEF1000F0AD040680368714656
:10BD00005B6832469847864202D00020BDE8F08149
:10BD100043462A4639462046BDE8F041FFF788BF32
:10BD20002DE9F843C468A24202D90020BDE8F88397
:10BD300016468846074601784068D2B2FFF774FC81
:10BD40008642F2D136B30023DFF854901C4612E04D
:10BD500090F8383090F839209A4203F1010E00EB48
:10BD600003011AD980F838E0087E28700134A4B2A3
:10BD7000A64223460ED97868026852694A4508EB04
:10BD80000305E5D090470134A4B2C0B2A6422870A2
:10BD90002346F0D80120BDE8F883FF20E5E700BF87
:10BDA0001DB100002DE9F041C568069F9DF81C609B
:10BDB000AA4202D90020BDE8F08190F800C0D0F876
:10BDC00004E04FF001084FEA4C0C1D468EF83BC0D2
:10BDD00033468EF85E808EF85D800446FFF728FFBC
:10BDE0000028E7D043463A4629462046BDE8F041C0
:10BDF000FFF796BF2DE9F047046813460A4624B1C1
:10BE00002046BDE8F04700F035BB057B0C7886681E
:10BE10006249B1FBF6F1002D0CBF4FF001094FF064
:10BE2000800919EA040F0CBF4FF0010C4FF0000C11
:10BE3000CDB2002B00F0AF804F0107F4FF57114641
:10BE400002EB030811F801EB4B460026002D50D001
:10BE5000002F4ED03A46013AFDD1427B12F0F70F47
:10BE600040F08D8090F91020013212D01EEA0302BA
:10BE700014BF0124002464450BD0002A6CD044690F
:10BE800090F8242094F800C04CEA020222704FF08F
:10BE9000010C846990F8262094F800A04AEA020276
:10BEA00022701DB117B13A46013AFDD190F9112027
:10BEB000013206D0C26990F825401278224218BF9C
:10BEC0001E43826990F826A0147824EA0A041470AC
:10BED00090F91120013201D001F8016C027B002A97
:10BEE00035D15B00DBB2002BB0D18845AAD1BDE8CB
:10BEF000F087427B12F0F70FB4D0846990F82620C7
:10BF000094F800A04AEA0202227090F9102001324F
:10BF10000AD01EEA030F44692AD090F8242094F82E
:10BF200000A04AEA02022270846990F826A02278D2
:10BF300022EA0A02227090F911200132CED0C269A1
:10BF400090F825401278224218BF1E43C4E75B08D0
:10BF5000002B7FF47BAFC8E7D0F814A090F824C082
:10BF60009AF8004024EA0C048AF80040944690E7CE
:10BF700090F824A0227822EA0A022270D4E7846989
:10BF800090F8262094F800A04AEA020222703A466D
:10BF9000013AFDD1B9E7BDE8F08700BF20A1070055
:10BFA0002DE9F0430C4683B001680A9F064690468F
:10BFB0001D4681B14268CB7A1268002B4ED10B68C6
:10BFC000D968914207D0394818603949DA6042F09F
:10BFD0008040186119600021B07B02F0EFFB77B15F
:10BFE00005EB07090DF1070715F8013B8DF8073040
:10BFF000012239463046FFF7FDFEA945F4D1B8F1DC
:10C00000000F0ED004EB08050DF1070714F8013BF3
:10C010008DF80730012239463046FFF7EBFEA54286
:10C02000F4D10121B07B02F0C9FB336893B1DA7A15
:10C0300082B1D00703D51F4A99691160DA7A910756
:10C0400003D51D4AD9691160DA7A520702D51B4A15
:10C050001B6A1360012003B0BDE8F08372B6CB7A8F
:10C06000D80709D5DFF858E0C868DEF8003003408B
:10C070008B61CEF80030CB7A980709D5DFF844E021
:10C080000869DEF800300340CB61CEF80030CB7A8F
:10C090005B0708D5DFF830E04869DEF80030034080
:10C0A0000B62CEF8003062B689E700BF01403F0066
:10C0B00000003F8000E100E004E100E008E100E072
:10C0C00080E100E084E100E088E100E02DE9F04754
:10C0D0000D4682B00168DDF828909DF82C80064658
:10C0E00017461C4681B14268CB7A1268002B4FD1AB
:10C0F0000B68D968914207D0394818603949DA602D
:10C1000042F08040186119600021B07B02F056FBBC
:10C1100077B105EB070A0DF1070715F8013B8DF81C
:10C120000730012239463046FFF764FEAA45F4D1B4
:10C13000B9F1000F0FD0A1440DF1070701223946D4
:10C1400030468DF80780FFF755FE9DF8073004F85C
:10C15000013BA145F2D10121B07B02F02FFB3368F6
:10C1600093B1DA7A82B1D00703D51F4A9969116079
:10C17000DA7A910703D51D4AD9691160DA7A520734
:10C1800002D51B4A1B6A1360012002B0BDE8F0878C
:10C1900072B6CB7AD80709D5DFF858E0C868DEF860
:10C1A000003003408B61CEF80030CB7A980709D578
:10C1B000DFF844E00869DEF800300340CB61CEF8D8
:10C1C0000030CB7A5B0708D5DFF830E04869DEF84D
:10C1D000003003400B62CEF8003062B688E700BF43
:10C1E00001403F0000003F8000E100E004E100E08A
:10C1F00008E100E080E100E084E100E088E100E0A7
:10C200002DE9F0410468E56815F0807F794D2560DF
:10C2100052D1DF0740F1B380002900F0E3800D78B0
:10C22000012B18BF45F000456563013190F824806B
:10C2300003F1FF3C48EA0828BCF1000F00F0A88099
:10C2400021B14D7811F8028B45EA082845682E7A0D
:10C25000BCF1020F06F1FF364FEA06360CBF48F07C
:10C26000805548F01045B6B26563ACF1020C08E0A9
:10C270000AB114700132013B05F47045B54216D97C
:10C280000468E56A15F0F00FF6D0A46B13F0010F07
:10C2900017464FEA242EEBD11AB107F802EB54707F
:10C2A0003A4605F47045B542A3F10203E8D8BCF163
:10C2B000000F6DD00468C3E7DD074CD5002900F0FE
:10C2C00089800D78012B18BF45F000456563013169
:10C2D00003F1FF3E90F824C0BEF1000F41D029B118
:10C2E00091F801C00D78023145EA0C2C45682E7A90
:10C2F000BEF1020F06F1FF364FEA06360CBF4CF0D6
:10C3000080554CF01045B6B26563AEF1020E08E000
:10C310000AB114700132013B05F47045B54215D9DC
:10C320000468E56A15F0F00FF6D013F0010F174618
:10C33000A46BEDD122B107F8024B241254703A4697
:10C3400005F47045B542A3F10203E9D8BEF1000F30
:10C3500007D00468C3E79E4690F824C0BEF1000FE2
:10C36000BDD11BB30468E16A11F0F00FFBD0A16BE3
:10C37000DC071DD50AB111700132013BF1E790F8DD
:10C3800024809C4648EA0828BCF1000F7FF458AF8F
:10C3900063B10468E16A11F0F00FFBD0DE07A16B16
:10C3A0000FD50AB111700132013BF1E7BDE8F08110
:10C3B0002AB114460D1204F8021B55702246023BA6
:10C3C000CFE72AB114460D1204F8025B51702246E1
:10C3D000023BDDE790F82450012B18BF45F00045E3
:10C3E000656375E790F82450012B18BF45F00045B0
:10C3F00065631BE700041F8090E80C00F0B41C6824
:10C4000059682568164F174E29432160164D174964
:10C410001760D66015611160417A154A5C180A31BF
:10C4200094F8244053F8215002EBC40149680D6090
:10C43000017A5C1803EB8101247ECD6902EBC40113
:10C4400049680D60817A581803EB810390F8300039
:10C45000596B02EBC002F0BC53681960704700BF13
:10C4600001401F00011000380110007800001F80FB
:10C47000B46101000BB1FFF7C3BE7047704700BF46
:10C48000F0B50C1EBDF8146034DBB0F90670191954
:10C49000B942C4BF3B1B1BB2002BA6461CDD002AC1
:10C4A0001146B8BFD11D02F00705CC10826A0120E9
:10C4B00007FB04E1A840012E0A44C0B21ED00CD3F1
:10C4C000022E09D1013B12FA83F3013A12F8011F3F
:10C4D00041409A421170F9D1F0BDC043013B12FABC
:10C4E00083F3C0B2013A12F8011F01409342117068
:10C4F000F9D1F0BD23441BB20024C6E7013B12FA78
:10C5000083F3013A12F8011F01439A421170F9D1E5
:10C51000F0BD00BF00291EDB30B4B0F90A408C42E8
:10C5200018DD002A16DBB0F90C40944212DD047EBF
:10C53000022C54D0032C4CD0012C06D15140C4887D
:10C540004A405140013C611A09B2012B2DD017D34A
:10C55000022B01D030BC7047002AB0F90630856A42
:10C560001446B8BFD41D44F3CF0404FB031102F0FA
:10C5700007026B5C012000FA02F25A406A54E9E7B4
:10C58000002AB0F90630856A1446B8BFD41D44F3BA
:10C59000CF0404FB031102F007026B5C012000FAD8
:10C5A00002F223EA02026A54D4E7002AB0F9063004
:10C5B000856A1446B8BFD41D44F3CF0404FB0311AD
:10C5C00002F007026B5C012000FA02F21A436A547F
:10C5D000C0E70489013C641A114622B2B5E7C58858
:10C5E0000489013D013C691AA21A09B212B2ACE7F2
:10C5F0002DE9F041079E9DF91880089D04461F46CD
:10C6000000F0BCFF0D4B0E480E4984F83380FF222A
:10C61000002F08BF1F4684F82F20002384F8302005
:10C6200084F8312084F8322020606665A565676251
:10C6300021662362A3622046BDE8F0817091FF1F4E
:10C640001C5701000110013810B50446806A034BE5
:10C65000236008B106F040F8204610BD1C570100C9
:10C66000F8B5436ADBB190F82C200125AA4083F885
:10C670003B2083F85E5083F85D500446406A0368AF
:10C680000E461B6800219847606A036831461B68A4
:10C6900098472946606ABDE8F840FEF73BBFC26B89
:10C6A000C56C1368046A23EA050313604CB1226861
:10C6B0004FF00043D3625163D36A002BFCDA936BD3
:10C6C000F8BD836B466B0825802410E03768426C08
:10C6D0003A4332601F68826C3A431A601A68876C6A
:10C6E000013D22EA07024FEA54041A6007D02142B2
:10C6F000ECD13268476C22EA07023260EAE7F8BD03
:10C7000070B50446406A0D4600282BD0616DFEF7D7
:10C710009FFD002D20460CBFA621A721FFF7A0FFFB
:10C72000606A20B1A16DBDE87040FEF791BD216C3B
:10C73000226D0868236A02430A6093B1DA7A82B1F3
:10C74000D00703D5224A99691160DA7A910703D597
:10C75000204AD9691160DA7A520702D51E4A1B6A4B
:10C76000136070BD236A002B2BD0D97A226EE1B101
:10C7700072B6D97ACE0706D51848D968066831400E
:10C7800099610160D97A880706D515481969066844
:10C790003140D9610160D97A4E0705D511485969F0
:10C7A000066831401962016062B61B68D96891421F
:10C7B00007D00D4818600D49DA6042F080401861DA
:10C7C0001960226C216D136823EA01031360A0E74E
:10C7D00000E100E004E100E008E100E080E100E0C9
:10C7E00084E100E088E100E001403F0000003F807C
:10C7F000436A2DE9F04105460E469046002B3ED097
:10C8000090F82C100124A14083F83B1083F85E407F
:10C8100083F85D40406A036800211B6808F1FF3718
:10C820009847FFB2B8F1000F23D03744A046013E2D
:10C83000686A16F8011F03681B6898470134B742FD
:10C84000A4B216D01F2CF3D90121686AFEF762FE4C
:10C8500095F82C206B6A520083F83B2083F85E80A9
:10C8600083F85D80686A036800211B68984701248B
:10C87000DEE7686A0121BDE8F041FEF74BBEC26BFE
:10C88000C16C136823EA010306EB080413604FF040
:10C890000048A6420ED02B6A16F801EB63B11A6865
:10C8A000C2F82C80C2F834E0D36A002BFCDAA6422E
:10C8B000936BF0D1BDE8F081AB6BD5F834C00820A4
:10C8C0008021DCF800206F6C1EEA010F14BF3A4390
:10C8D000BA43CCF800201A68AF6C3A431A601A6861
:10C8E000AF6C013822EA07024FEA51011A60E8D121
:10C8F000CFE700BF70B50446406A0D46002828D037
:10C90000616DFEF7A5FC20462946FFF7A9FE606A87
:10C9100020B1A16DBDE87040FEF79ABC216C226D7C
:10C920000868236A02430A6093B1DA7A82B1D007B9
:10C9300003D5234A99691160DA7A910703D5214A10
:10C94000D9691160DA7A520702D51F4A1B6A13604F
:10C9500070BD236A002B2BD0D97A226EE1B172B65A
:10C96000D97ACE0706D51948D96806683140996149
:10C970000160D97A880706D51548196906683140DB
:10C98000D9610160D97A4E0705D512485969066800
:10C9900031401962016062B61B68D968914207D0C4
:10C9A0000D4818600D49DA6042F080401861196046
:10C9B000226C216D136823EA01031360A3E700BF13
:10C9C00000E100E004E100E008E100E080E100E0D7
:10C9D00084E100E088E100E001403F0000003F808A
:10C9E0002DE9F041044686B0806A9DF830801E46ED
:10C9F0000F461546B4F90830002800F04B81DA1DC7
:10CA000048BF03F10E02B4F90630D21003FB02F264
:10CA1000002106F085F9B4F90820202A00F3A78048
:10CA2000B4F90610A74B0120203A733902EBD272F9
:10CA300001EBD1714FF0200E029073208DE8014080
:10CA400042F34F0241F34F01204600F04DFE606A71
:10CA500084F82D70002800F05181002D40F09F8057
:10CA6000B4F90830202B14BF3D253C2584F82C5008
:10CA7000B8F1000F40F09A8006B394F93300002813
:10CA800018DBC0B2012101F0ADFE012194F83300A2
:10CA900001F094FE012001F0CDFE002194F8330056
:10CAA00001F08CFE0A2001F0C5FE012194F833004C
:10CAB00001F084FE606A002800F09880616DFEF746
:10CAC000C7FB042280492046FFF792FE217A0139F4
:10CAD000C9B22046FFF7C4FD7C4904222046FFF777
:10CAE00087FE94F92D30012B14BF1421102120460C
:10CAF000FFF7B6FD042276492046FFF779FEB4F928
:10CB000006308F22802B84F85C2000F0A580602BFB
:10CB100000F0B1800225DA212046FFF7A1FD294669
:10CB20002046FFF79DFD81212046FFF799FD94F8EF
:10CB30005C102046FFF794FDD9212046FFF790FDB9
:10CB400094F92D30012B14BFF12122212046FFF74B
:10CB500087FD204606225F49FFF74AFE606A58B308
:10CB6000A16DFEF775FB012006B0BDE8F081B4F9B8
:10CB70000610594B0120403A52394FF0400E0290B6
:10CB800002EBD272522001EBD1718DE8014042F3E9
:10CB90004F0241F34F01204600F0A6FD57E76DB26A
:10CBA00084F82C50B8F1000F3FF466AFFEF706FB97
:10CBB000002E3FF47FAF60E7216C226D0868236A86
:10CBC00002430A6073B1DA7A62B1D00703D5434AEF
:10CBD00099691160DA7A91076FD4520702D5404AF9
:10CBE0001B6A1360012006B0BDE8F081236A002BA8
:10CBF0002BD0D97A226EE1B172B6D97ACF0706D599
:10CC00003848D9680568294099610160D97A8E074A
:10CC100006D53548196905682940D9610160D97A76
:10CC20004D0705D5314859690568294019620160E9
:10CC300062B61B68D968914207D02D4818602D490B
:10CC4000DA6042F0804018611960226C216D13682F
:10CC500023EA0103136034E7B4F90830402B7FF472
:10CC600059AF94F92D30012B14BFCF239F2384F8A3
:10CC70005C3012254FE7B4F90830102B7FF44AAF2F
:10CC800094F92D30012B14BFAF23102384F85C30AE
:10CC9000022540E7DA1D48BF03F10E02B4F9063061
:10CCA000D21003FB02F21046059205F00DFDA062C2
:10CCB00000283FF459AF059AAAE60F4AD9691160D6
:10CCC000DA7A8AE76C5701004C590100505901008B
:10CCD00054590100585901006059010000E100E079
:10CCE00008E100E080E100E084E100E088E100E0AC
:10CCF00001403F0000003F8004E100E0012194F882
:10CD00003100214F01F06EFD94F83200012101F055
:10CD100069FD94F9312094F9323057F83220E263FA
:10CD200057F83330206A23640125E56425651A68C5
:10CD30002A431A6048B1B8F1000F3FF439AFFFF74A
:10CD40005BFB002E3FF4B6AE97E6294694F82F0021
:10CD500001F048FD294694F8300001F043FD94F9B4
:10CD60002F2094F9303057F83220626357F833306F
:10CD70006564A5641A68A36322F001021A60002E9C
:10CD80003FF498AE79E600BFB4610100B0F9082025
:10CD9000D31D48BF02F10E03B0F90620806ADB10F4
:10CDA00002FB03F2002105F0BBBF00BFF0B5002974
:10CDB000BDF814502EDBB0F90660B1422ADA002A21
:10CDC00059DBB0F9087014461C44BC42C4BFBB1AFE
:10CDD0001BB2002B1EDDD2B2D408D0F828E016FB1F
:10CDE000041112F00702DBB20EEB010421D0C2F1F4
:10CDF0000807FAB2374F9342BF5C0CD2C3EB020C68
:10CE0000FF2646FA0CF6012D07EA06073FD005D3A8
:10CE1000022D36D0F0BD012D39D030D21EF8016080
:10CE200026EA07070EF801709342F3D3B0F9061013
:10CE30000C449A1AD2B2072A10D9022D36D0002DEE
:10CE400014BFFF26002613462670083BB0F90610D3
:10CE5000DBB2072B0C44F7D802F00702002AD9D026
:10CE60001D4B012D9B5C1DD017D3022DD2D12278F2
:10CE700053402370F0BD13441BB20022A1E7022DE2
:10CE800025D11EF8016077400EF80170CCE71EF83E
:10CE9000016037430EF80170C6E7227822EA0303E7
:10CEA0002370F0BD227813432370F0BD1146237820
:10CEB000DB4323700839B0F90630C9B207291C4496
:10CEC000F5D812F00702A5D0034B9B5CCFE73444A2
:10CED000AFE700BF0C570100FC56010070B4047EA0
:10CEE000BDF80C50022C18D0032C1FD0012C0BD0F5
:10CEF000002A03DBB0F90840944201DC70BC7047A3
:10CF0000039570BCFFF7BCBAC4880395013CA41A12
:10CF10000A4621B270BCFFF749BF0689C488013EAA
:10CF2000641AB21AE41A12B221B2E1E70489039535
:10CF3000E41A641A114622B270BCFFF737BF00BF73
:10CF400070B4057EBDF80C60022D1AD0032D12D0EE
:10CF5000012D03D0039670BCFFF728BFC488E41AE4
:10CF6000A41A0A4621B2002A03DBB0F90840944211
:10CF700013DC70BC70470489013C641A114622B26C
:10CF8000F1E7C48805890396013CAD1AED1A621ACF
:10CF900011B22AB270BCFFF709BF039670BCFFF74D
:10CFA0006FBA00BF2DE9F8430446406A002863D0F9
:10CFB000616DFEF74DF9052274492046FFF718FC14
:10CFC000A1790139C9B22046FFF74AFBB4F908201C
:10CFD000E588A66AD31D48BF02F10E03DB10626A22
:10CFE00015FB03F51FFA85F8002A7BD094F82C3046
:10CFF0000125AB4082F83B3082F85E5082F85D50EC
:10D00000606A036840211B6808F1FF379847BFB288
:10D01000B8F1000F23D03744A846013E606A16F8E5
:10D02000011F03681B6898470135B742ADB216D09F
:10D030001F2DF3D90121606AFEF76CFA94F82C20B9
:10D04000636A520083F83B2083F85E8083F85D803A
:10D05000606A036840211B6898470125DEE70121CB
:10D06000606AFEF757FA606A002800F08D80A16DB3
:10D07000BDE8F843FEF7ECB8236A002B2BD0D97A31
:10D08000226EE1B172B6D97ACE0706D54048D9688A
:10D090000568294099610160D97A8D0706D53D4818
:10D0A000196905682940D9610160D97A480705D511
:10D0B00039485969056829401962016062B61B68E0
:10D0C000D968914207D0354818603549DA6042F096
:10D0D000804018611960226C216D136823EA0103F6
:10D0E000136068E7E26BE36C1168276A0B4306EB99
:10D0F000080913604FF0004E4E450DD016F801CBD5
:10D100002FB33A68C2F82CE0C2F834C0D36A002BBF
:10D11000FCDA4E45936BF1D1226C236D11680B4301
:10D12000136097B1FB7A83B1D90703D51D4BBA6958
:10D130001A60FB7A9A0703D51B4BFA691A60FB7ACF
:10D140005B0702D5194B3A6A1A60BDE8F883A36BF6
:10D15000D4F8348008208021D8F80020656C1CEABF
:10D16000010F14BF2A43AA43C8F800201A68A56C0F
:10D170002A431A601A68A56C013822EA05024FEAB0
:10D1800051011A60E8D1B7E7276AC5E704570100E3
:10D1900080E100E084E100E088E100E001403F0040
:10D1A00000003F8000E100E004E100E008E100E071
:10D1B0002DE9F04F85B09946BDF93870BDF83CA017
:10D1C000BB1AC1EB090B002BB8BF5B42BBF1000FD0
:10D1D000B8BFCBF1000B5B450D4616460093804669
:10D1E00048DC4D453A4633464CDC194613460A4660
:10D1F000C5EB09019B1A89B2002B0CB2B8BF5B4288
:10D2000004EBD474BE42ACBF4FF0FF3201224D4557
:10D21000039102924FEA640429DC9BB201930DE072
:10D22000D8F80070BF69B847019BE41AA3B21CB2DA
:10D230000135002C2DB211DBA94518DB009B5B45A5
:10D240002A46534631464046EADCD8F80020534689
:10D250009769294632464046B847E5E7029A1644A0
:10D26000039AA94502EB030436B224B2E6DA05B00C
:10D27000BDE8F08F4A462B46B94635464D45174620
:10D280001E46B2DD304629463E464D460746894693
:10D29000AEE700BF10B404682469A44610BC604720
:10D2A00030B40468BDF808500295A46BA44630BCA5
:10D2B000604700BF30B40468BDF808500295E46BC5
:10D2C000A44630BC604700BF70B40468BDF90C6070
:10D2D000BDF8105003960495246CA44670BC6047BA
:10D2E000704700BF10B582B0B0F90C200191016801
:10D2F000009200220C6CB0F90A301146A04702B02F
:10D3000010BD00BF704700BF01F003010129017685
:10D3100006D0032904D0C2880389428183817047E3
:10D320000289C38842818381704700BF2DE9F041A3
:10D330000568134E6F6986B0B7420446BDF8308069
:10D3400010D1013B13441BB20093CDF804800B466F
:10D35000AD6A2046A8472368DB6AB3420AD106B00B
:10D36000BDE8F081059304920391B84703A92568AD
:10D370000EC9E6E7204606B0BDE8F041184700BFF9
:10D38000E1D200002DE9F0410568124E6F6986B0C8
:10D39000B7420446BDF830800FD1013BCDF8048080
:10D3A0000B4400921BB2AD6A2046A8472368DB6A93
:10D3B000B3420AD106B0BDE8F0810593049203910F
:10D3C000B84703A925680EC9E7E7204606B0BDE8BF
:10D3D000F0411847E1D200002DE9F04F0568DFF871
:10D3E00058B06F6985B05F450646BDF93890BDF805
:10D3F0003CA00C46904615D11F19BC420CDACDF862
:10D4000000A0214601342D6A4B464246304624B2E4
:10D41000A847BC423568F2DBEB6A5B4507D105B033
:10D42000BDE8F08F0393B8473568039BE4E73046C7
:10D4300005B0BDE8F04F1847E1D200002DE9F043F8
:10D4400087B099420546BDF93840BDF83C6025D00B
:10D45000A24212D00768DFF88080D7F81490C14547
:10D4600032D18DE850002846BC6AA0472B68DB6AA1
:10D47000434524D107B0BDE8F083994202DD084658
:10D480001946034628680E96C46B01335B1A1BB21B
:10D490002846A44607B0BDE8F0436047A24202DD3B
:10D4A000134622461C4628680E96631C846B9B1A02
:10D4B0001BB22846A44607B0BDE8F04360472846A3
:10D4C00007B0BDE8F0431847059304920391C8479D
:10D4D00003A92F680EC9C4E7E1D200002DE9F04F7F
:10D4E000D0F800E0DFF89090DEF814B083B0CB45C0
:10D4F0000446BDF93080BDF834A00D4617461E46DF
:10D5000031D1CDF800A0DEF824B0294633463A46A2
:10D510002046D8472368CDF800A008F1FF323A44EE
:10D52000D3F824B0294612B233462046D8472368A0
:10D53000CDF800A02946D3F820B03A46434620460D
:10D54000D8472068CDF800A0711E29444346056ADB
:10D5500009B23A462046A8472368DB6A4B4506D104
:10D5600003B0BDE8F08FD847D4F800E0C9E7204603
:10D5700003B0BDE8F04F1847E1D20000F0B400243A
:10D5800001254FF6FF76094F076004710476C481C8
:10D5900004828476C461C575857545768682468227
:10D5A000C180028141818281F0BC7047285C01000A
:10D5B0002DE9F04F85B00668BDF84450BDF93880BC
:10D5C000CDF8008004460195D6F848B00392BDF925
:10D5D0003C60BDF9407089469A46D847236801955A
:10D5E000009742465146D3F8488020463346C0470C
:10D5F0002068039B0E930F95856C4B463A46314647
:10D600002046AC4605B0BDE8F04F60472DE9F04F2D
:10D6100087B01746BDF9404000912546E91D0593A6
:10D6200044BF2B4603F10E010268BDF84860536900
:10D630000294C91003912B49BDF9444001968B42D5
:10D64000824645D1002C3CDD029B3C445E1EB6B2B6
:10D650004FF0000923B2049301364D46029B002B84
:10D6600028DD059B002403EB090806E0EDB22B063C
:10D6700004F1010411D4A6421CD0A1B211F0070F8D
:10D6800023B24FEA4505F1D1002BB8BF0733DB10B9
:10D69000013418F803502B06EDD5009BD2F818B0D2
:10D6A00019443A4609B2019B5046D847A642DAF8D7
:10D6B0000020E2D1039B01379944049B3FB2BB4257
:10D6C000CCD1D36A074A934206D107B0BDE8F08FA8
:10D6D0009847DAF80020B5E7504607B0BDE8F04FAC
:10D6E000184700BFE1D2000070B4BDF90C60BDF96D
:10D6F0001050BDF8144003960495059470BCFFF7D4
:10D7000085BF00BF2DE9F04F91B083460591C169F7
:10D71000BDF8680006909DF87400BDF86C709DF827
:10D7200070A0039002929946002900F0CC800B7AF9
:10D7300048680A68C3EB0903DBB2154600EBC30275
:10D7400030F83360D3780993BAF1010F92F90530BC
:10D7500092F802800E9392F9064079D9BDF93830DB
:10D76000089323B20B93A94BDBF800200F931946C3
:10D7700053698B4240F0A280099B002B53D0BDF827
:10D7800008300C930021234407910D930F460C465B
:10D79000A946B8F1000F3FD0BDF81C100B9BBDF897
:10D7A0000C000297CB1813FB00F30C9803440D9860
:10D7B0001BB2014404930BB20A93002505E0013526
:10D7C000EBB264009845E4B223D9029B2B4459077D
:10D7D00003D1731C19F806409EB22306EFD5089BAF
:10D7E000E918059B11FB0AF1BAF1010F194402D1A6
:10D7F000039B012B1ED0069B0193039B0093D369CF
:10D80000049A1F4609B253465846B847DBF8002031
:10D81000D5E7029F4744FFB2079B0999013307935D
:10D82000DBB29942B5D8D36A0F9A934241D111B075
:10D83000BDE8F08F0E9B0599591893690A9A2944FF
:10D840001F4609B2069B5846B847DBF80020B6E7EA
:10D85000039B012B82D800230B93089383E707993E
:10D86000099A0131013A49B212F0FF020791099277
:10D8700060D1069A4A454F4617D0BAF1010F03D13D
:10D88000039A012A00F0B5800A9A089802EB8201F7
:10D89000039AD2008DE88400084401B2DC69029A40
:10D8A00053465846A047DBF80030DB6A0F9A934294
:10D8B000BDD0584611B0BDE8F04F184758469847BC
:10D8C000DBF8002058E7BBF90A3005998B42AEDD42
:10D8D000BBF90C3002988342A9DD062313FB0A131F
:10D8E000002BA4DD039B00EBC303002B9FDD9BF803
:10D8F0001A3033B9B9F1AF0F84BF09F101035FFAF0
:10D9000083F9424ADBF800300F9211465A698A4285
:10D910006AD1BDF8142008920522099200220792CC
:10D920001FFA8AF20A92CDF830900FFA8AF2B946BD
:10D93000039F05920799BDF83040089D05221046C7
:10D9400010FB04120A98324C0646084601FB0651A9
:10D95000A65C15FA80F209B212B204910B92082467
:10D9600000251CE0BAF1010F01D1012F24D0069A45
:10D970000192029A009705FB0722D3F81C800499B4
:10D98000059B12B25846C047DBF80030013C013518
:10D9900014F0FF046DB24FEA56063FF460AFF00793
:10D9A000E0D4069A4A45F1D0BAF1010F01D1012F16
:10D9B0000ED0CDF80490DCE7029AD3F818800B99CA
:10D9C000069BAA1812B25846C047DBF80030DDE7C4
:10D9D000029AD3F818800B99AA184B4612B25846EF
:10D9E000C047DBF80030D1E758469047DBF80030FD
:10D9F0008FE70899CDF8009005311C6A029A082338
:10DA000009B25846A047DBF800304EE7E1D20000EB
:10DA1000785C0100F0B5C36985B004463BB30A29C0
:10DA20006FD00D294FD01A7A91424CD3987A884200
:10DA300049D38A1A5D68D2B205EBC205AA78002ADA
:10DA400056D0E878002853D0607E00283ED095F963
:10DA500005E0B4F90E00A67DB4F90A70724406FB25
:10DA60000202BA4269DCE77DB4F9102034E00A29E9
:10DA70005CD00D2927D0427E002A50D0B0F90E008C
:10DA8000A57DB4F90A60062212FB0502B242E67DCA
:10DA900042DD228AE38102EBC60212B218462282DC
:10DAA000B4F814E0678A03960B46029501468DE8A8
:10DAB00080402046FFF726FEA37DE28903EB430367
:10DAC00002EB4303E381012005B0F0BDA67DE77DB5
:10DAD000B4F90E00B4F91020B4F814E00397678A83
:10DAE00002960B468DE8804001462046FFF70AFE6D
:10DAF0002979E389A27D012001FB0233E38105B08E
:10DB0000F0BD0022C2811A7BC17D038A01FB023372
:10DB10000382012005B0F0BDB4F91020C0E7857D77
:10DB2000C67DB4F91020B0F90E00B9E7028AC17DB4
:10DB3000C38102EBC1030382C5E70020E0811B7BA8
:10DB4000228AE77D03FB072212B22282C4E700BFCC
:10DB500011B18175C175704701218175C17570471B
:10DB6000844641EA000313F003036DD1403A41D3E8
:10DB700051F8043B40F8043B51F8043B40F8043BA7
:10DB800051F8043B40F8043B51F8043B40F8043B97
:10DB900051F8043B40F8043B51F8043B40F8043B87
:10DBA00051F8043B40F8043B51F8043B40F8043B77
:10DBB00051F8043B40F8043B51F8043B40F8043B67
:10DBC00051F8043B40F8043B51F8043B40F8043B57
:10DBD00051F8043B40F8043B51F8043B40F8043B47
:10DBE00051F8043B40F8043B51F8043B40F8043B37
:10DBF000403ABDD2303211D351F8043B40F8043BD7
:10DC000051F8043B40F8043B51F8043B40F8043B16
:10DC100051F8043B40F8043B103AEDD20C3205D3E6
:10DC200051F8043B40F8043B043AF9D2043208D0DE
:10DC3000D2071CBF11F8013B00F8013B01D30B8850
:10DC400003806046704700BF082A13D38B078DD02E
:10DC500010F003038AD0C3F10403D21ADB071CBF00
:10DC600011F8013B00F8013B80D331F8023B20F86A
:10DC7000023B7BE7043AD9D3013A11F8013B00F8A3
:10DC8000013BF9D20B7803704B7843708B7883702B
:10DC900060467047374A384913681B06FCD40B6846
:10DCA00013F08003F8D172B634490A78002A5FD0A5
:10DCB000334A3448F0B4344C176806682568D46891
:10DCC0000C303E44143200681268304F35442C4406
:10DCD00020440244C2F34E022D4E2E482E4D2F4CAE
:10DCE00042F400423A60376806682D682C4A24687E
:10DCF0000C303E44006812682A4F35442C442044BE
:10DD00000244C2F34E02284E2848294D294C42F4C1
:10DD100000423A60376806682D68274A24680C304C
:10DD20003E4400681268254F35442C442044024488
:10DD3000C2F34E02224E2348234D244C42F40042AB
:10DD40003A60376806682D68214A24680C303E44E2
:10DD50000068126835442C4420440244C2F34E0249
:10DD60001C4842F4004202600B7062B6F0BC70477F
:10DD700062B6704724B0034024B00B405AA0FF1F86
:10DD800038B003403CB0034040B003402CB00340E7
:10DD900058B003405CB0034060B0034064B003403F
:10DDA0006CB0034030B0034038B00B403CB00B4087
:10DDB00040B00B4044B00B404CB00B402CB00B407B
:10DDC00058B00B405CB00B4060B00B4064B00B40EF
:10DDD0006CB00B4030B00B4030B42948294A2A4B74
:10DDE0002A4D6024E121047011701B78284C082B07
:10DDF00030D00A2B2748284937D00C2B0CBF3522AE
:10DE00003D2212232A60236002600B60234B2449C9
:10DE10001B78244ABBB101230B601360224B2349BA
:10DE20001B78234A012B26D9042B0FD9082B1ED986
:10DE3000102B94BF862387230B6013601D4B012298
:10DE40001A7030BC70470B601360E7E784230B60E7
:10DE50001360F3E700F58E200F49083001221323E9
:10DE60002A60236002600B60D0E73922F7E7852340
:10DE70000B601360E2E780230B601360DEE700BFF6
:10DE800000400740014007404892FF1F08B0034090
:10DE90000CB0034008B00B400CB00B405DA0FF1F5E
:10DEA00020B0034020B00B404992FF1F24B0034034
:10DEB00024B00B405AA0FF1F0C2830B417D91023F0
:10DEC000984228BF18461C46104A114D1178181A5E
:10DED0008C42287018D00F4913700B7823B10E496B
:10DEE0000E4A00230B60136030BCFFF775BF0A2891
:10DEF00002D90C231C46E7E7082802D90A231C464E
:10DF0000E2E708231C46DFE730BC70474892FF1F5A
:10DF100059A0FF1F5AA0FF1F24B0034024B00B409C
:10DF200028282FD8334B2DE9F0411E5CFF2E2BD033
:10DF3000314B1B78002B2AD132062CD472B62F4DD0
:10DF40002F4C2F46012326602B7062B672B62368D1
:10DF50001B060CD43B781BB9F4E72B78002BF1D0CF
:10DF600062B603F0A1F872B623681806F5D5254B02
:10DF70001B6800222A7062B6234A107843FA00F028
:10DF8000BDE8F081002070470020BDE8F081FFF778
:10DF900081FE3206D2D572B61C4DDFF87C801C4C57
:10DFA00006F04007FFB206F03F06D8F80030DFB1B8
:10DFB00023F01003C8F8003001232660134A2B70A9
:10DFC00062B672B6236819060CD413781BB9ECE755
:10DFD0002B78002BE9D062B603F066F872B623689E
:10DFE0001B06F5D50B4BC3E743F01003C8F8003010
:10DFF000E2E700BF786101005AA0FF1F5CA0FF1F8D
:10E0000000B0034010B0034059A0FF1F5BA0FF1FEA
:10E0100000B00B4010B00B400CB00B400A4A0B494B
:10E02000136843F4805313600B7843B9084BC02244
:10E030001A70084B80F30C0000B218807047044B34
:10E0400080221A70F5E700BF2C8004405DA0FF1FFE
:10E0500021C00C4000C00C40F0B51B4B1B4E596852
:10E0600018689A68DB6885B06C460FC433789907E6
:10E070001DD5174A174C1378174913F0700318BFB2
:10E080001370164A164B8027177000263320032280
:10E0900026706D4608701A7072B6043C45F0010592
:10E0A0002046A84762B6237813F0700309D10D4BC0
:10E0B000064901E0013B02D00A78D207FAD505B043
:10E0C000F0BD237005B0F0BDA46101000100024065
:10E0D00000000240040002400B0002400700024022
:10E0E0000A000240410D0300B0F5006F0AD210B5DE
:10E0F000094B1B78DB07044606D504F1A0500078D5
:10E10000C0B210BD00207047FFF7A6FF04F1A05079
:10E110000078C0B210BD00BF01000240B0F5006F32
:10E1200017D238B50F4B1B78DA070D46044611D5C8
:10E1300004F1A0500378AB420AD00B4A137813F0D5
:10E14000700318BF1370074A05701378DB07FCD5FE
:10E1500038BD7047FFF780FF04F1A0500378AB4251
:10E16000EBD1F5E7010002400000024008B5104C79
:10E1700008E0236859050DD423681A050FD42368D5
:10E18000DB0411D423685803F3D501F087FB23681F
:10E190005905F1D500F00EF823681A05EFD500F007
:10E1A0002DFF2368DB04EDD501F0EAF9EAE700BFB3
:10E1B0003480044008B5FFF7D9FF00BF014B10229F
:10E1C0001A80704700200540704700BF094908B514
:10E1D0000B6830B16A461844A2F58052904202D2D0
:10E1E0000860184608BD04F041FA0C2303604FF0A4
:10E1F000FF3008BD4C92FF1FFEE700BFEFF3138016
:10E2000070B9EFF310836BB9EFF305825AB94FF48D
:10E210008070EFF311832BB1984228BF18467047E6
:10E220004FF0FF3070470F2A01D81846F1E7014B35
:10E23000D05CEEE7F0E300E0704700BF10B40F4B96
:10E2400053F8302092F880422CB1012369B182F852
:10E25000803010BC704703EBC0035B681A6841B99B
:10E2600022F002021A6010BC704782F8003110BC24
:10E27000704742F003021A6010BC7047B46101009D
:10E280001C4A02EBC00301295B6811D004291BD092
:10E2900052F83000002280F8802229B1022920D0D3
:10E2A000032922D01A6070474FF480721A607047B9
:10E2B00052F830004FF4A27280F880121A601A6887
:10E2C00022F020021A60704752F830104FF4A27208
:10E2D000012081F880021A601A6842F020021A6058
:10E2E000704740F203121A6070474FF481721A604F
:10E2F000704700BFB4610100212848D8F8B5042A4E
:10E3000044D8DFE802F0484B4E0345004FF4102696
:10E310002B4B03EBC0030D465C68216811F4E061F0
:10E3200048D0284B284A2949C3F89C2104F140428F
:10E330002748C3F8A411A2F59221264FC3F8A001E3
:10E340007C292548C3F8A871C3F8AC012CD9A2F5E3
:10E3500094237C2B2AD9A2F596237C2B28D9A2F5CD
:10E3600098237C2B29D9A2F59A227C2A27D81B48EE
:10E3700072B6236823F4702343F08072C4F38401DF
:10E380001643236040F82150266062B6F8BD7047FE
:10E390004FF43026BCE74FF40026B9E74FF440268F
:10E3A000B6E74FF42026B3E70D48E1E70D48DFE775
:10E3B0000D48DDE7FFF764FFB3E70C48D8E7F8BD89
:10E3C000B46101000082FF1FF188FF1F9988FF1FC1
:10E3D000C588FF1F6D88FF1F4188FF1F2893FF1FFF
:10E3E0005092FF1F8892FF1FD892FF1F0893FF1FB4
:10E3F0001A4B03EBC00010B4426802F14043A3F58E
:10E4000092217C2923D9A3F594217C290DD9A3F548
:10E4100096217C291FD9A3F598217C2919D9A3F528
:10E420009A237C2B11D80E4C00E00E4C72B6136868
:10E430000D4823F08773C2F3840123F4803343F043
:10E440008073136044F8210062B610BC7047074C1B
:10E45000ECE7074CEAE7074CE8E700BFB4610100CE
:10E460002893FF1F8892FF1F39E200005092FF1F80
:10E470000893FF1FD892FF1F30B4054B054D064C83
:10E48000002210211A602A602060196030BC704799
:10E4900014D0034004D0034000D00340282838B5EE
:10E4A0002ED0002904464FDD5F4B1B78012505FA6D
:10E4B00003F28A4202D8212837D938BD0338C2B2C4
:10E4C000012A3AD9202C4AD0192C48D0574A126830
:10E4D00002FB011222FA03F31D2800F29B80DFE801
:10E4E00000F0928B847D9999766F99999999999971
:10E4F00099999968615A53994C999999999999451B
:10E50000494B1B780B2B08D90C2B1CBF0C3B19411A
:10E510000846BDE83840FFF781BDC3F10C039940C0
:10E520000846BDE83840FFF779BD2946FFF786FE6B
:10E530002946BDE83840FFF7A3BE3D4A126802FBFA
:10E54000011222FA03F3C7E72128B6D80021FFF70A
:10E5500075FE20460121BDE83840FFF791BE354ADF
:10E56000126802FB011222FA03F3B5E73249334A7B
:10E570000B604FF45173136038BD3149314A0B6061
:10E580004FF45173136038BD2F49304A0B6040F28D
:10E590004443136038BD2E492E4A0B6040F2444379
:10E5A000136038BD2C492D4A0B6040F24443136080
:10E5B00038BD2B492B4A0B6040F24443136038BDF1
:10E5C00029492A4A0B6040F24443136038BD284968
:10E5D000284A0B6040F24443136038BD2649274A5D
:10E5E0000B6040F24443136038BD2549254A0B6057
:10E5F00040F24443136038BD2349244A0B604FF472
:10E600005173136038BD2249224A0B604FF4517395
:10E61000136038BD212C3FF650AF7F29D4BF0021B5
:10E620000121204693E700BF3093FF1F088003407D
:10E630000890034008800B4010800B4048A0044025
:10E6400018800B404CA004401880034008B00440E0
:10E650001080034004B004404080034018C00440D0
:10E660003880034014C004402880034010B00440A8
:10E67000208003400CB004403080034010C00440B0
:10E68000488003401CC0044018900340349004406C
:10E69000109003403090044038B1102828BF10205B
:10E6A000044AC3B2107813707047024A01231078ED
:10E6B000137070473093FF1F2DE9F8430E468046D4
:10E6C0003249334D304603F05DFF47F612230028F0
:10E6D0001ABF1D464FF002094FF00109002425FA28
:10E6E00004F003F059FD4FF05E51074603F0ACFD16
:10E6F0000146304603F05AFF30B90134072CEED101
:10E70000E80903F049FD07463146384603F050FE5C
:10E710004FF07C5103F08EFC03F082FF4FF6FF7246
:10E720009042A8F1030328BF1046012B29D9B8F164
:10E73000170F17D8174B23FA08F303F0010383F0E0
:10E74000010223B9B8F1190F0FD0BDE8F883124BBD
:10E75000124D13491A6044EAC9042A6008601C601B
:10E76000BDE8F883B8F1200FECD10E4B0E4D0F49E8
:10E77000002244EAC9041A602A6008601C60BDE8EF
:10E78000F8830B4B0B4D0C49F2E700BF001BB74061
:10E79000006CDC026006F00000800340048003404F
:10E7A0000880034000800B4004800B4008800B4031
:10E7B000009003400490034008900340212801D8B2
:10E7C000FFF73CBD704700BF212806D8044B53F823
:10E7D000303093F80002C0B270470020704700BF8D
:10E7E000B4610100212801D8FFF74ABD704700BF7E
:10E7F00072B60C490C4B0D4A1B680868126862B669
:10E80000520102D5322B88BF01300949C3F5BB3311
:10E810004FF47A72FF33A1FB031302FB00F000EB0D
:10E820009310704760A0FF1F18E000E004ED00E0C7
:10E83000ABAAAAAA2DE9F843054672B6204F214B90
:10E84000214A1B683C68126862B6520102D5322B1D
:10E8500088BF013495B3C3F5BB331C4EDFF8649019
:10E86000DFF86480FF334FF47A72A6FB031302FBD8
:10E8700004F404EB931472B6D9F800103A68D8F88F
:10E8800000E062B6C1F5BB33FF33A6FB03031EF005
:10E89000806FC4EB93134FF47A7002D0322988BF93
:10E8A000013200FB0233B3F57A7F04D3013D05D07A
:10E8B00004F57A74DFE702F0F7FBDCE7BDE8F883E4
:10E8C00060A0FF1F18E000E004ED00E0ABAAAAAAD8
:10E8D000F8B52D4B2D49DFF8D0E0DFF8D0C02C4E35
:10E8E0002C4D2D4C2D4A2E4F4FF4000018604FF048
:10E8F000807018604FF0007018604FF080601860F2
:10E900004FF0006018600020086028234BF6FF716C
:10E91000CCF80010CEF80030336013602B60236019
:10E920003B60B3629362092245F8242CC4F8D80FE7
:10E9300005F57F65C7F8D41F07F5FF2707F5FA67C8
:10E94000C6F8F83F2B6006F5FF26C4F8D42F05F56E
:10E95000FD2504F5FF24386006F2F4761148316095
:10E9600005F5FF6504F5FD642B6023600260FFF789
:10E9700033FA1920FFF75EFF01F0F6FC40F21310A6
:10E98000BDE8F840FFF756BF08E100E0048003400F
:10E9900014800340248003402C8003401C800340EB
:10E9A0003480034000800B400C800340088003400B
:10E9B0002B4A2C491368F0B543F4006313600A78BE
:10E9C000294F2A4E2A4D2B4C2B490023092A3B70F4
:10E9D00033702B7023700B703DD01A2A21D0274B37
:10E9E0001B780A2B25D01F2B30D01F2827D80020BA
:10E9F00002460125224B234C1A7023495D700422E4
:10EA00004FF0020E88273C26402598729A704FF4EA
:10EA1000004083F813E05A751F74DE70257008609B
:10EA2000F0BD1A4B40F213321A60144B1B780A2BBC
:10EA3000D9D1174B4FF451721F281A60D7D9C0F3A0
:10EA40004432C0F3471500F01F00D3E7114B4FF4D9
:10EA500051721A60C9E7104B40F213321A60BEE7D8
:10EA6000348004403193FF1FD4A0FF1F69A0FF1F13
:10EA7000DCA0FF1FD5A0FF1F68A0FF1F3293FF1F60
:10EA800000B006402FE400E004E100E004D00440C0
:10EA900010B0044000D004400CB00440144B1449A2
:10EAA0009B7803F0EC0200F003031343420700F0ED
:10EAB0000F0248BF43F01003042A8B7013D00C4B95
:10EAC0000B4A5B79C10603F0EF0348BF43F0100324
:10EAD00053719379820603F0EF03054A48BF43F070
:10EAE0001003937170478B7943F040038B71E6E715
:10EAF00000B00640234B1B681B0542D510B5224CC5
:10EB0000237823B102F0D0FA2378002BFAD11F48E2
:10EB10001F4A204B4FF4004400210460D1701B7841
:10EB2000092B1FD01A2B03D11B4B40F203121A6082
:10EB30001A4B1B7803F07F030A2B1DD01F2B03D128
:10EB4000174B40F203121A60164A114B1648174928
:10EB500012681C79DB79002303700B700AB1012362
:10EB6000137010BD124B40F203121A600B4B1B784E
:10EB700003F07F030A2BE1D10E4B40F203121A601F
:10EB8000E2E770473480044068A0FF1F84E100E0A2
:10EB900000B006403193FF1F04D004403293FF1FA2
:10EBA00000D0044064A0FF1FD4A0FF1F69A0FF1F76
:10EBB0000CB0044010B004400A4A38B5054613783A
:10EBC00003F0FF04002BFAD101212846FFF70AFECB
:10EBD00021462846FFF7F2FD034A044B52F8352040
:10EBE0001A6038BD68A0FF1FB4610100D8A0FF1FE4
:10EBF00009B140F08000174A1378984216D010B43B
:10EC0000154C246824050FD503F07F030A2B1CD074
:10EC10001F2B11D0002900F07F0114BF6023442373
:10EC20000A290DD01F2902D0107010BC70470B4963
:10EC300043F440730B60F7E7084B00241C60E9E7DE
:10EC4000074943F440730B60EEE7054B00241C605A
:10EC5000E0E700BF3293FF1F3480044000D004403F
:10EC600010B00440124B1A7882420CD01149096846
:10EC7000090507D5092A16D01A2A0AD009280DD065
:10EC80001A2801D0187070470B4A40F213311160F6
:10EC9000F8E7094A002109281160F1D1074A40F23A
:10ECA00013311160EEE7054A00211160E6E700BF6D
:10ECB0003193FF1F3480044004D004400CB0044062
:10ECC0000D4B1B6813F4006305D0212805D90B4BAD
:10ECD00000201860704718467047094B10B5074C64
:10ECE00053F8303023600121FFF77CFD23680022B8
:10ECF0001A70012010BD00BF3480044064A0FF1FC3
:10ED0000B46101000C4B1B6813F4006306D0172894
:10ED100006D00A4A537B03F0FE035373002070476A
:10ED2000074B064A40F202311960537B43F001035E
:10ED300053730120704700BF3480044000B0064088
:10ED400008B004402DE9F84F234B1B681A053BD54A
:10ED5000224B1B680BB101221A70DFF89090204DF6
:10ED600099F80040DFF888801E4E0134272C8ABFB6
:10ED70004FF0000A5FFA84FA54460746AB462B78F8
:10ED80009C4216D1FFF73AFA40281FDC33791B0664
:10ED9000F5D59BF800300133272B86BF00221346A0
:10EDA000DAB218F80330DBB2F3712A702B789C4288
:10EDB000E8D00D490B4BFFB20120BC2208F80470CB
:10EDC000087089F800A0DA70BDE8F88FFF28D6DD5A
:10EDD00002F06AF9D3E700BF34800440D8A0FF1FD7
:10EDE000D5A0FF1F00B0064068A0FF1FDCA0FF1FDA
:10EDF0006CA0FF1F2DE9F84F294B1B681A0548D559
:10EE0000284B1B6805460BB101221A7005EB010A5D
:10EE1000554540D2DFF89C80234CDFF89C90234F6F
:10EE20000AE015F8012B09F80B20214A0123AA4515
:10EE3000137088F800602ED098F80030227803F123
:10EE4000010BBBF1270F86BF0026B3465FFA8BF696
:10EE50009345E6D1BC22FA7005E03A7913060BD44B
:10EE600022789345DDD1FFF7C9F94028F5DDFF2869
:10EE7000F6DD02F019F9F3E722780132272A86BF7E
:10EE800000210A46D1B219F80220D2B2FA712170DB
:10EE9000E6E7BDE8F88F054BBC22DA70BDE8F88FD5
:10EEA00034800440D8A0FF1FD5A0FF1F00B006404B
:10EEB00068A0FF1FDCA0FF1F6CA0FF1F10B5044C53
:10EEC000237823B102F0F0F82378002BFAD110BD9B
:10EED00068A0FF1F064A074B1B781078DBB2C0B250
:10EEE00083422CBF273000F1FF30C01A704700BFAB
:10EEF000D5A0FF1FDCA0FF1F054A064B10781B782A
:10EF0000C0B2DBB2984238BF4030C01A704700BF71
:10EF1000D4A0FF1F69A0FF1F30B4154B154C1A7801
:10EF20002378D2B2DBB29A421ED001333F2B0ED9E6
:10EF30001149124B087819680023C0B2237021B11F
:10EF4000D31A1A2B01DC00230B7030BC70470A481F
:10EF50000A49C05C0968DDB2C0B225700029F4D04E
:10EF60009A4238BF4032EBE74FF0FF30EDE700BF89
:10EF7000D4A0FF1F69A0FF1F94A0FF1F64A0FF1F64
:10EF8000084A094B12781B78DBB29A4207D001334A
:10EF9000402B28BF0023054AD05CC0B270474FF019
:10EFA000FF307047D4A0FF1F69A0FF1F94A0FF1F70
:10EFB0000D4B1B681B0516D530B40C4B0C4CDA7886
:10EFC0000C480D4902F0CB024025DA705D74DA7806
:10EFD00042F03402DA7023780268DBB20B700AB1B7
:10EFE0000023137030BC70473480044000B00640EA
:10EFF00069A0FF1F64A0FF1FD4A0FF1FF0B4384B0F
:10F000001A7912F0300F2CD072B6997D01F0FF0200
:10F0100000293DD062B6334F334938780D78334EEE
:10F020001C46C0B2EDB2431C402BE17928BF00233F
:10F03000AB4202F1FF32C9B21CBFF154184612F0C4
:10F04000FF02F0D12A4B1B68C2B23A704BB1A84202
:10F0500036BFC5F14005401B40192728C4BF012217
:10F060001A701F49CA78D2B2150616D452060DD5A9
:10F070001B4B1B795B0609D51E4B1F491B680022E1
:10F080000A7003B11A70164B3C22DA70F0BC70475C
:10F090004022D9795A7462B6E3E70B791C06E5D5AC
:10F0A000164B174E1C783378E4B2DBB29C420ED07C
:10F0B000144D01E0A3420AD00133282B28BF0023BE
:10F0C0000879E85CC0B2C871087D0728F2D9DBB2C4
:10F0D000034933700B79180644BF7C23CB70C5E716
:10F0E00000B00640D4A0FF1F69A0FF1F94A0FF1F1F
:10F0F00064A0FF1FD8A0FF1F68A0FF1FDCA0FF1F98
:10F10000D5A0FF1F6CA0FF1F2DE9F84F214B1B68F6
:10F1100007460BB101221A70DFF888901E4D99F84E
:10F120000040DFF884801D4E0134272C8ABF4FF049
:10F13000000A5FFA84FA5446AB462B78A34216D1F4
:10F14000FFF75CF840281FDC33791B06F5D59BF8E8
:10F1500000300133272B86BF00221346DAB218F89D
:10F160000330DBB2F3712A702B78A342E8D00C494C
:10F170000A4BFFB208F804700120AC22087089F82D
:10F1800000A0DA70BDE8F88FFF28D6DD01F08CFF13
:10F19000D3E700BF54A1FF1F51A1FF1F00C00640CD
:10F1A00050A1FF1F58A1FF1FE8A0FF1F1C4BDFF855
:10F1B00094C01A681B49F0B542F480521A4D1A6087
:10F1C000DFF884E0194F1A4E1A4C00238CF80030F7
:10F1D0004FF451722B701F2840F213358EF8003017
:10F1E0003B70337025600A6012D819460124124A18
:10F1F000124D11701248547000212C274026937232
:10F200004FF4003491701174D7702E700460F0BD0B
:10F21000C0F34431C0F3471400F01F03E7E700BF19
:10F22000348004400CC00440E5A0FF1F51A1FF1F23
:10F2300050A1FF1F08C0044000C0064031E400E0B8
:10F2400004E100E0E4A0FF1F58A1FF1F144B144984
:10F250009B7803F0EC0200F003031343420700F035
:10F260000F0248BF43F01003042A8B7013D00C4BDD
:10F270000B4A5B79C10603F0EF0348BF43F010036C
:10F2800053719379820603F0EF03054A48BF43F0B8
:10F290001003937170478B7943F040038B71E6E75D
:10F2A00000C00640F8B5134B1B68DB041FD5124C99
:10F2B000237823B101F0F8FE2378002BFAD10F4B0D
:10F2C0000F4A104D104F114E114C12484FF400319F
:10F2D00019600023D37040F203113960316029684E
:10F2E0001579D2792370037011B101230B70F8BD29
:10F2F000F8BD00BF3480044050A1FF1F84E100E04E
:10F3000000C00640E0A0FF1F08C004400CC004403D
:10F31000E4A0FF1FE5A0FF1F0A4A38B50546137891
:10F3200003F0FF04002BFAD101212846FFF75AFA17
:10F3300021462846FFF742FA034A044B52F835208B
:10F340001A6038BD50A1FF1FB461010054A1FF1F16
:10F3500009B140F080000F4A1378984219D010B4D8
:10F360000D4C2468E40412D503F07F03082B02D16E
:10F370000A4B00241C60002900F07F0314BF6021A9
:10F380004421082B03D1054B41F4407119601070E2
:10F3900010BC70473393FF1F348004400CC00440FE
:10F3A000704700BF0D4B1B6813F4805305D0212814
:10F3B00005D90B4B00201860704718467047094B61
:10F3C00010B5074C53F8303023600121FFF70AFADB
:10F3D000236800221A70012010BD00BF3480044051
:10F3E000E0A0FF1FB46101000C4B1B6813F48053B5
:10F3F00006D00E2806D00A4A537B03F0FE0353734F
:10F4000000207047074B064A40F202311960537BD7
:10F4100043F0010353730120704700BF3480044060
:10F4200000C0064004C00440034B1B68DB0401D548
:10F43000FFF76ABE704700BF3480044070B5094EC4
:10F4400004464518AC4204F101040AD03368DB04D9
:10F45000F8D514F8010CFFF757FEAC4204F1010493
:10F46000F4D170BD3480044010B5044C237823B12E
:10F4700001F01AFE2378002BFAD110BD50A1FF1F16
:10F48000064A074B1B781078DBB2C0B283422CBF10
:10F49000273000F1FF30C01A704700BF51A1FF1F95
:10F4A00058A1FF1F054A064B10781B78C0B2DBB28B
:10F4B000984238BF4030C01A704700BFE4A0FF1F19
:10F4C000E5A0FF1F30B4154B154C1A782378D2B243
:10F4D000DBB29A421ED001333F2B0ED91149124B99
:10F4E000087819680023C0B2237021B1D31A1A2BEF
:10F4F00001DC00230B7030BC70470A480A49C05C2D
:10F500000968DDB2C0B225700029F4D09A4238BF34
:10F510004032EBE74FF0FF30EDE700BFE4A0FF1F04
:10F52000E5A0FF1F10A1FF1FE0A0FF1F084A094B25
:10F5300012781B78DBB29A4207D00133402B28BFE8
:10F540000023054AD05CC0B270474FF0FF307047CF
:10F55000E4A0FF1FE5A0FF1F10A1FF1F054B064AF7
:10F560001B7806491268DBB20B700AB100231370D6
:10F57000704700BFE5A0FF1FE0A0FF1FE4A0FF1F32
:10F5800030B42B4B1A7994061FD52A48DA790378C0
:10F59000294901333F2B0978C8BF00238B42D2B2DF
:10F5A00003D0264CD9B2E2540170254A116861B1EA
:10F5B000244A1278D2B2934236BFC2F140029B1A5B
:10F5C0009B18272BC4BF01230B70194AD378DBB2D9
:10F5D000180611D45A060DD5154B1B795B0609D5B3
:10F5E000194B1A491B6800220A7003B11A70104B9C
:10F5F0002C22DA7030BC704711790906EAD514491B
:10F6000010480C780178C9B28C420DD04A1C272AC8
:10F6100084BF00210A460F4D054C98BFD1B2AA5CA9
:10F62000D2B2E2710170D5E76C21D170D2E700BF90
:10F6300000C00640E4A0FF1FE5A0FF1F10A1FF1FB0
:10F64000E0A0FF1F51A1FF1F54A1FF1F50A1FF1FEA
:10F6500058A1FF1FE8A0FF1F21282FD8184B195CC5
:10F66000FF292BD0174B184ADFF870C003EBC000FE
:10F67000F0B54368DFF868E0144F154D154E0024CF
:10F680001C60DEF80030012043F020038840CEF8F3
:10F69000003014604FF4A07338602E60C2F800C0D0
:10F6A000013BFDD113689B05FCD42023013BFDD118
:10F6B000094B09B233F8110080B2F0BD0020704749
:10F6C000C4620100B46101000050044008500440CD
:10F6D00004500440000002030051044080014A002D
:10F6E00038800440431E032B14D872B60A4951F8DF
:10F6F000230068B170B4094C058834F813204668BB
:10F7000041F82360521B24F8132062B670BC704786
:10F7100062B6704700207047B4A1FF1F0CA3FF1F03
:10F72000013803280BD872B6074B53F8203043B189
:10F7300000205B680130002BFBD162B670470020CF
:10F7400070471846F9E700BF08A2FF1F30B472B631
:10F750002B4A13781D0706D52A4B196A002936D083
:10F76000996A002941D053781C0706D5254B196C9E
:10F7700000293ED0996C002939D09378190705D516
:10F78000204B196E002936D0996E89B1D3781B07AA
:10F7900007D51C4BD3F880207AB3D3F888201121E9
:10F7A0003AB162B6184B00221A7030BC00F058BE55
:10F7B0000D21154C154D227843F8315003EBC10350
:10F7C0000830013A5860227062B630BC704704229B
:10F7D0000D4C0F4D217843F8325003EBC203083033
:10F7E0004A1E5860227062B6EFE70521E1E7092161
:10F7F000DFE70822ECE70C22EAE71022E8E700BF87
:10F80000AC6301000080FF1F31A2FF1FC800400051
:10F8100088004000431E032B1DD81B4A400140F0C6
:10F82000100030B4104472B6184CE25C032A1BD8A6
:10F83000DFE802F00212151703220D88E25410F0DF
:10F84000080F14BFC823882343EA05430831036027
:10F85000416062B630BC704708300222EDE70522F5
:10F86000EBE708300422E8E7094A52F8230038B1F0
:10F87000084A52F82300416042F8231062B6E9E7D3
:10F8800042F82310034AF7E70080FF1F40A2FF1F42
:10F8900008A2FF1F18A2FF1F00BE00BF2DE9F04FF6
:10F8A000DFF820B3DFF820A387B044E0AF4F4FEA82
:10F8B000930807EBC809013ED9F8042003F00803B8
:10F8C000F6B2A2F1080003F0FF04002B40F00B8118
:10F8D00057F838301B0C99B222F8081C002B00F0A6
:10F8E000F980A34B22F8064C42F8044C53F826202A
:10F8F000002A00F075819F4D55F8263058609E4CC7
:10F9000045F8260034F81630194424F8161000F093
:10F9100087FD002800F05D81984A994B19F0080F87
:10F9200000F1080018BF1346C9F8040047F8383042
:10F9300008238BF800309BF80040E4B265071DD522
:10F94000904B1B78BBB190490A7802F0FF032AB1B3
:10F95000013BDBB20B70002B00F001858B490A786C
:10F9600002F0FF032AB1013BDBB20B70002B00F069
:10F970002D8100F073FE04238BF8003004F008039F
:10F9800003F0FF02002B00F0DA809AF80030DBB2BF
:10F990001E098BD19A08DFF8D49159F8321009EB7F
:10F9A000C200C1F38301013940680C297DD8DFE82A
:10F9B00001F080807C7C7C7C7C7C467C7C7C0700AD
:10F9C000D0F800E0724C4168724F734E6160C4F829
:10F9D00000E01FFA8EF140F2816E0025674B49F876
:10F9E0003230012071453D60C9F81050C9F81850F7
:10F9F00030705E4A00F20881B1F5D06F80F08283EA
:10FA0000B1F5817F00F0668300F28F82802900F0DB
:10FA10007483822940F0A782A18801F07F01042924
:10FA200000F2A1825D4B5E4A89000B44157055704F
:10FA300019788D0740F1808310700220F2E2554F53
:10FA40003A6842B3574B544E5749188834780D786A
:10FA50004028864645F0020828BF4FF0400E002C93
:10FA600084F001043470CEEB00000CBF8824C8245D
:10FA700009EBC80680B285F0010544EA0E447260C5
:10FA8000188049F8384072440D7018B9BEF1400F23
:10FA900018BF00223A603E4B1A88B2F5A06F04D11D
:10FAA00000219A785970414B1A70414A0123137012
:10FAB0003EE7374C258842F221018D4200F05A8200
:10FAC00024683C49324D8C4200F000822B4949F8B1
:10FAD0003210EAE7294A2A4B19F0080F18BF1346DB
:10FAE00047F8383024E700F0BBFC334A334952F87A
:10FAF0002630002B78D058688C5D42F8260003F140
:10FB00000802C9F80420032C05D8DFE804F0120F1E
:10FB1000150204228A551A8819F0080F0CBF882391
:10FB2000C82343EA024347F8383001E702228A55E6
:10FB3000F1E703228A55EEE705228A55EBE7E00755
:10FB400000F13082210600F15F82A20706D51C4A2F
:10FB50001C4913780220DBB213700870E30602D54B
:10FB6000184B10221A7007B0BDE8F08F0080FF1FFD
:10FB7000B4A1FF1F60A1FF1F0CA3FF1FC80040001E
:10FB8000880040003CA2FF1FC5A1FF1FB0A2FF1FBD
:10FB900028A2FF1F5CA1FF1FC4A1FF1FC0200740B8
:10FBA00034A2FF1F70A1FF1F30A2FF1F9820074043
:10FBB000942007402109000308A2FF1F40A2FF1F55
:10FBC00088200740802007409020074000F0ACFFCD
:10FBD000CFE6AC4A47F83800137801331370A7E634
:10FBE00043F82600A84D8AE68B5D032B00F26B825A
:10FBF00001A252F823F000BF31F9000031F90000F2
:10FC0000F9FF0000F3FF000040F62115A94200F0C3
:10FC1000358100F29F81B1F5086F00F0FF81B1F5E9
:10FC2000106F40F0A0819948116AA47804700C0606
:10FC300000F19382D9F828209549100600F18882B6
:10FC4000D9F830209249120600F17D82D9F8382087
:10FC50008F49130600F17282D9F840208C491506AD
:10FC600000F12E83D9F848208949140600F1238336
:10FC7000D9F850208649100600F11883D9F8582089
:10FC80008349120600F10D83D9F8602080491306DC
:10FC900000F12083D9F868207D49150600F115830D
:10FCA000D9F870207A49140600F1DE82D9F878205C
:10FCB0007749100600F1D382D9F8802074491206E2
:10FCC00000F1E982D9F888207149130600F1DD823C
:10FCD000D9F890206E49150600F1D182D9F8982004
:10FCE0006B49140600F1C5826A486B4A6B49019062
:10FCF0006B486C4C644D0294002304970596804633
:10FD00001C4617460E460395386828B1456800F032
:10FD1000A7FB2846002DF9D100233B60039B3068E8
:10FD20001A46002342F8243028B1456800F098FBB9
:10FD30002846002DF9D100223260019A98F800304F
:10FD40001146002241F8042B029A0191023B4FF028
:10FD5000000122F81410032B09D8DFE813F050013A
:10FD60000400500104004FF0010388F80030013412
:10FD7000042C07F1040706F1040608F10108C3D1B9
:10FD8000494C404D2278494B049F059E00211007A5
:10FD900029701A7000F14E82454962780A7000217C
:10FDA000C9F83010C9F838101107DFF8E48000F105
:10FDB0002C82A2783F49DFF8D8800A700021120710
:10FDC000C9F85010C9F8581000F10882E2783A4991
:10FDD0002F4C0A7013074FF00001C9F87010C9F8D2
:10FDE000781000F1BF8133780293002283F001057F
:10FDF000C9F89020C9F898200020019080468646D6
:10FE000002462E490C7844F0020C09EBCC03039314
:10FE1000029B002B039B5A600CBF8822C82242EA37
:10FE2000080384F0010249F83C3035700A70DFF8AD
:10FE300060C0234BDFF88480002840F01681BEF1BB
:10FE4000400F1BD142F0020C09EBCC03019ADFF802
:10FE500040E05A60002D40F01E81050445F0880501
:10FE60009DF808304EF83C50024433700C70134635
:10FE7000402803D10020134A3B601080124A01231E
:10FE8000137012E631A2FF1F60A1FF1F3CA2FF1FEB
:10FE90000080FF1F18A2FF1FB4A1FF1F08A2FF1FB1
:10FEA00040A2FF1F0CA3FF1FAC630100C42007404A
:10FEB000C8200740CC200740D020074030A2FF1FB9
:10FEC000C4A1FF1F70A1FF1F942007406C68B149B7
:10FED0008C427FF4FBAD0178A9297FF4F7AD41781E
:10FEE00045297FF4F3AD8178C2297FF4EFADC17865
:10FEF0006B297FF4EBADA849A84E0878347880F0E0
:10FF00000105002C40F002000D700CBF8821C821B3
:10FF100084F0010449F8301009EBC000A0493470A6
:10FF20000025052445600C70D0E540F20232914274
:10FF300040F09480A28802F07F02042A13D86588DA
:10FF40008DB998490290920011440A7842F0020259
:10FF50000A7051E740F62122914200F0828042F27D
:10FF6000212291427DD08F4A0F2313708E4A0123A4
:10FF700013709AE58849894E0D78377885F0010E1F
:10FF8000002F45F0020581F800E00CBF8821C82150
:10FF900049F8351009EBC50587F0010700213770D6
:10FFA00069608DE5814B80487B491A614FF0020EF4
:10FFB00080F800E07B4F0A707D49196099607D4EA2
:10FFC0007D4D7E4C9A610D213970FF213170DFF833
:10FFD00008E2297022707A4D7A4A8EF800109F2725
:10FFE000012406F8047C5D600470DA6007B0BDE8A7
:10FFF000F08F01238B559BE400238B5598E44FF041
:020000021000EC
:10000000000388F80030B2E666496B4B80220D2071
:1000100008701A70A2077FF5A1AD98E56A496B4A8E
:1000200009781170E588854280F089815A490C78F9
:10003000402DAE4644F0020C28BF4FF0400E02EBBC
:100040000E0309EBCC000193012342604FEA0E48F6
:10005000CEEB050002930025C822E0E6B1F5A06FC3
:1000600081D1012300250293C6E640287FF6EAAE3F
:1000700042F002020CEBC201019E4E60BDB19DF840
:10008000085053491D703346403888F800404033CB
:100090004CF83210EFE69DF8083033700504019BF0
:1000A0000C7045F0C80503444EF83C50E0E69DF85E
:1000B00008501D70019B3E4988F80040403840338D
:1000C0004CF83210D7E619F0080F0CBF02230323B7
:1000D0008B552DE4A28802F07F02042A3FF643AF3D
:1000E0006588002D7FF43FAF2E49029092001144A5
:1000F0000A7822F002020A707EE6344A0220157065
:1001000055708FE733494A68002A3FF42CAF658861
:10011000B4F804E004E00C314A68002A3FF423AF4D
:100120000B88AB42F7D14B887345F4D12D0A032DD0
:100130000CBF1078088975E7022073E7C86B083890
:1001400000F08EF988E5486B083800F089F97DE504
:10015000C86A083800F084F972E5506A083800F07F
:100160007FF967E500F05CF9002800F0D6800830E0
:100170000F4AC4F88400C4F8802000F051F9002828
:1001800000F0C5800830124AC9F88C00C9F88820F0
:1001900029E600BF0100040030A2FF1FC4A1FF1F19
:1001A000C5A1FF1FC0200740942007400080FF1F0B
:1001B00088004000882007408020074098200740A2
:1001C00074A1FF1FC8A1FF1F3CA2FF1F34A2FF1F85
:1001D000C8004000B06301008C20074000F020F907
:1001E000002800F0A68008305D4AC8F86400C8F80E
:1001F000602000F015F9002800F095800830594A79
:10020000C9F86C00C9F86820E0E500F009F9002899
:1002100077D00830524AC8F84400C8F8402000F0AF
:10022000FFF8002867D008304E4AC9F84C00C9F8DA
:100230004820BEE500F0F4F8002856D00830484ABF
:10024000C9F82400C9F8202000F0EAF8002846D0B8
:100250000830444AC9F82C00C9F828209CE5C86F2A
:10026000083800F0FDF827E5486F083800F0F8F886
:100270001CE5D1F89C00083800F0F2F834E5D1F81C
:100280009400083800F0ECF828E5D1F88C00083824
:1002900000F0E6F81CE5D1F88400083800F0E0F83A
:1002A00010E5C86D083800F0DBF8EDE4486D08385B
:1002B00000F0D6F8E2E4C86C083800F0D1F8D7E4D2
:1002C000486C083800F0CCF8CCE4C86E083800F070
:1002D000C7F8E5E4486E083800F0C2F8DAE42A7896
:1002E000C9F8280001322A7056E52A78C9F820009A
:1002F00001322A70A8E72A78C9F8480001322A702A
:1003000057E52A78C8F8400001322A7087E72A7832
:10031000C9F8880001322A7065E52A78C4F880009F
:1003200001322A7029E72A78C9F8680001322A7058
:100330004CE52A78C8F8600001322A7059E7402855
:10034000864628BF4FF0400E02EB0E0301930123B7
:10035000CEEB00004FEA0E480025029351E500BEA7
:1003600088004000C80040002DE9F843204C00F010
:1003700037FF002204F1A00023461A605A600833B8
:1003800083424FF00001F8D11A4A1B4F13681B4DEE
:100390001B481C4EDFF87880DFF878C0DFF87890D3
:1003A000DFF878E043F480231360C4F307233B7045
:1003B000C4F307432B70240EFF2302F52832047088
:1003C000114D88F8003011488CF80030D432337069
:1003D000012389F8003070268EF800104FF4007465
:1003E000102107F8183C2E7004601170BDE8F883E6
:1003F0000080FF1F348004409C200740B02007404D
:10040000B42007401020074049E400E008E100E084
:1004100080200740882007409420074000210740A3
:1004200072B60D480268B2FA82F30F2B10DC4FF05F
:100430000041D94022EA0102026062B6074803EB9C
:10044000C303DB00C2180021C15010465160704741
:1004500062B60020704700BF3493FF1FBC83FF1FAC
:100460000D4B0E4AC31AA2FB03231B090F2B0CD8FA
:100470000B4A127852B972B60A484FF0004102682E
:1004800021FA03F31A43026062B67047064A1278F3
:10049000002AF0D0FFF75AB9BC83FF1F398EE3382A
:1004A00031A2FF1F3493FF1F3CA2FF1F38B50E4B34
:1004B0000E4C1B68218805468BB1B1F5917F05D2A2
:1004C0000B4A4B1C55549BB2238038BD0022084870
:1004D00098470021064A55540123238038BDB1F5C1
:1004E000917FEDD338BD00BF68A2FF1F16A3FF1F89
:1004F0001CA3FF1F2DE9F843214E224F3168012331
:1005000080463B70B1B1204D4B8801EB8302013333
:1005100000240F2BC2F808802C7004D84B800023D5
:100520003B70BDE8F88340230B800320FFF772F98E
:100530003460F4E7DFF8549099F80030002BF0D0E5
:10054000114D45F6215408E0013C12D02B7883B9B7
:1005500000F0AAFD99F800307BB10320FFF7E0F826
:100560000528F1D8FFF75CFF014630600028EBD08A
:10057000CAE701232B70BDE8F883BDE8F88300BF0C
:1005800084A2FF1F58A2FF1F88A2FF1F3CA2FF1FCB
:100590001201F8B5D5B2A1B3012943D0437804467E
:1005A00000781B0643EA004040F4704045F0040622
:1005B0008F1E3043FFF79EFF022F04F1020314D970
:1005C000053414F8023C14F8032C14F8010C1B0435
:1005D00043EA0223334343EA0060033FFFF78AFF05
:1005E000022F234604F10304EBD8022F23D0012F5E
:1005F0000DD045F4774040F00500BDE8F840FFF726
:1006000079BF14482843BDE8F840FFF773BF187856
:1006100045F4770545F0060545EA0020BDE8F840B9
:10062000FFF768BF03780C4845EA03452843BDE857
:10063000F840FFF75FBF1A78587845F0774545F0E6
:10064000070545EA022545EA0040BDE8F840FFF706
:1006500051BF00BF06F0F70007F000F738B5084BB0
:100660001C7824B9074D296809B14B8803B938BDF6
:100670009B000B800320FFF7CDF82C6038BD00BF36
:1006800058A2FF1F84A2FF1F2DE9F041AD4E336831
:100690000746002B00F092801D885A88910803EBD2
:1006A00081010432AA428C6842D25A8004F00F06BB
:1006B0004FEA1428A449A6F1080208F00F00C4F379
:1006C0000313062A00F101050B701AD9B31E012B82
:1006D0005FFA88F04ED9052E48D0042E00F0A48190
:1006E000731F022B7FD90F2E0ED1F72842D8F02886
:1006F00002D0964B1B883BB1FFF7D8FE0020BDE827
:10070000F08127B1BD4202D00020BDE8F081082E63
:10071000C4F3033300F08780092E11D00A2E40F075
:1007200094800A2BF0D18A4B8A4A1B68A02181E071
:100730001846FFF795FE0420FEF7D4FF3060B5E7BA
:10074000092BE1D1270E00F07B81834B814A1B6886
:100750009021C4F307461170EDB2FCB2002B00F0FB
:100760009D80224631462846984797E0F02843D995
:10077000F72841D0F1380E28C6D801A353F820F04D
:10078000370901001B0901000909010009070100DF
:1007900009070100FB08010009070100DB0901004E
:1007A00009070100A5090100BF090100E3080100D4
:1007B00009070100CB080100AF080100674B1B7857
:1007C000002BA1D00420FEF78DFF034630600028E7
:1007D0009AD00588002D7FF460AFFFF741FE3560A9
:1007E0002846BDE8F081FFF761FEC4F30740FFF73C
:1007F0005DFE072E02D1200EFFF758FE534B584ADC
:10080000198858481468584D524A017000270E0A3A
:10081000F0201F802E7010700CB301225348A047A7
:100820000120BDE8F081082B7FF46EAF504B494AA0
:100830001B688021C4F307461170EDB2240E6BB320
:10084000284622463146984728E00B2E11D10B2B23
:100850007FF45AAF474B3F4A1B68B021EAE7464B4B
:100860001B68002B00F0FB80404898470120BDE842
:10087000F0810C2E40F000810C2B7FF445AF3F4BF4
:10088000344A1B68C0211170EDB2C4F30746002B37
:1008900000F0C88028463146240E98473849314A2E
:1008A000314B0D7016701C700120BDE8F081354B86
:1008B0001B68002B00F0D6809847C4F30746254BF1
:1008C000EDB2240E83F80080E8E72F4B1B68002B65
:1008D000F2D12E4B1B68A3B1FE209847C4F3074604
:1008E000EDE72B4B1B68002BE6D1284B1B6843B16F
:1008F000FC209847C4F30746E1E7264B1B68002B12
:10090000DAD1C4F30746DAE7234B1B68C4F3074682
:10091000002BD4D030469847D1E7204B1A68002AE4
:10092000EFD0260C630C06F07F0003F47E531843CF
:10093000F6B29047C3E71A4B1B68C4F30746002B77
:10094000E8D1BCE790A2FF1F1AA3FF1F16A3FF1F49
:100950006CA2FF1F14A3FF1FA0A2FF1F3CA2FF1F3A
:1009600068A2FF1F18A3FF1F19A3FF1F1CA3FF1FCF
:1009700098A2FF1F9CA2FF1F80A2FF1F5CA2FF1F67
:100980001BA3FF1F48A2FF1F4CA2FF1F50A2FF1F67
:100990008CA2FF1F7CA2FF1F94A2FF1F64A2FF1F57
:1009A00078A2FF1F3F4B1B68002B85D13E4B1B6875
:1009B000002BA6D0FA209847C4F307467FE73B4BAD
:1009C0001B68002B7FF478AF374B1B68002B98D047
:1009D000FB209847C4F3074671E7354B1B68002B93
:1009E0007FF46AAF304B1B68002B8AD0F820984701
:1009F000C4F3074663E70E2B7FF486AE2D4A2E4BD9
:100A00001268E0211970002A47D0260C610C06F00C
:100A10007F0301F47E511943EDB2A1F50051284640
:100A20009047F6B2240E39E7FFF740FDC4F30740C4
:100A3000FFF73CFD200EFFF739FD0020BDE8F081F7
:100A40001E4B1D4A1B6880211170EDB2C4F307468E
:100A500083B1314628463A4698473C461EE7012076
:100A6000BDE8F081104B1B68002B3FF44AAFFF201C
:100A7000984746E71C4611E70D2EBCD10D2B7FF49D
:100A800043AE0F4B0C4A1B68D0211170EDB2C4F37A
:100A90000746002B7FF4FEAEC4E7C4F30746EDB271
:100AA000240EFBE674A2FF1F50A2FF1F54A2FF1FDB
:100AB00044A2FF1F60A2FF1F14A3FF1F98A2FF1FE5
:100AC00070A2FF1F38B5164D2868E0B10188448830
:100AD000A14213DD03191B7A83B104F10803C21884
:100AE0000C1B002302E012F8011F21B10133A342C5
:100AF000F9D1204638BD1C46204638BDFFF7B0FC72
:100B00000020286038BD074B1B780BB9002038BD8A
:100B10000220FEF7E7FD28600028D7D1F6E700BFE6
:100B2000ACA2FF1F3CA2FF1F0D4B1B78BBB910B539
:100B30000C4C216803F0FF024B883F2B07DC073386
:100B40000B4401F1470003F8012F8342FBD14023FE
:100B50000B800120FEF75EFE0023236010BD70476E
:100B6000A4A2FF1FA8A2FF1F70B5EFF3108272B6F8
:100B70000C4C206880B10C4E00254369236073B192
:100B80009D6102B962B6457783689847EFF310829A
:100B900072B620680028F0D102B962B670BD336029
:100BA000EFE700BFB4A2FF1FB8A2FF1FFFF7DCBF33
:100BB000024A136801331360704700BF60A0FF1F33
:100BC0004B0803F1376303F5D83310B50446B3FB84
:100BD000F1F0FDF7EDFE044B1B7803B110BD20468C
:100BE000BDE8104000F03EBB7093FF1F08B50846FB
:100BF000FEF7A8F8012008BD08B50846FEF7A2F8E0
:100C0000012008BD38B508460D4602F0F9FA044641
:100C100001462846FEF7EEF8204638BD10B50846D6
:100C200014461146FEF7E6F8204610BDFEF7C0B99F
:100C300008B50846FEF766F8003018BF012008BD69
:100C400008B50846FEF73CF8003018BF012008BD83
:100C500008461146FDF7CCBF0846FEF703B800BFB3
:100C60000846FDF7A9BF00BFFDF744BF10B54B080C
:100C700003F13760144600F5D830B0FBF1F0FDF712
:100C800097FE2046BDE81040FDF708BFFEF778B993
:100C9000FEF742B9FEF730B9FEF710B9FEF71AB900
:100CA0000368064A1B68934205D110B5C8B2FEF727
:100CB00049F8012010BDC9B2184700BFF90B010067
:100CC0000368064A1B68934205D110B5C8B2FEF707
:100CD00039F8012010BDC9B2184700BFF90B010057
:100CE0000368064A1B68934205D110B5C8B2FEF7E7
:100CF00029F8012010BDC9B2184700BFF90B010047
:100D00000368064A1B68934205D110B5C8B2FEF7C6
:100D100019F8012010BDC9B2184700BFF90B010036
:100D20004B0803F1B76303F5584310B50446B3FB12
:100D3000F1F0FEF73BFA044B1B7803B110BD2046DF
:100D4000BDE8104000F08EBA7193FF1F08B5084649
:100D5000FEF76AFB012008BD08B50846FEF764FBF4
:100D6000012008BD38B508460D4602F049FA044690
:100D700001462846FEF762FB204638BD10B50846FE
:100D800014461146FEF75AFB204610BDFEF7E6BB9F
:100D900008B50846FEF728FB003018BF012008BD43
:100DA00008B50846FEF7FEFA003018BF012008BD5E
:100DB00008461146FEF7CCBA0846FEF7F1BA00BF66
:100DC0000846FEF7A9BA00BFFEF76CBA10B54B088B
:100DD00003F1B760144600F55840B0FBF1F0FEF7A0
:100DE000E5F92046BDE81040FEF730BAFEF79EBB9D
:100DF000FEF768BBFEF756BBFEF736BBFEF740BBFF
:100E00000368064A1B68934205D110B5C8B2FEF7C5
:100E10000BFB012010BDC9B2184700BF590D0100DE
:100E20000368064A1B68934205D110B5C8B2FEF7A5
:100E3000FBFA012010BDC9B2184700BF590D0100CF
:100E40000368064A1B68934205D110B5C8B2FEF785
:100E5000EBFA012010BDC9B2184700BF590D0100BF
:100E60000368064A1B68934205D110B5C8B2FEF765
:100E7000DBFA012010BDC9B2184700BF590D0100AF
:100E8000704700BF0368F0B4FBB1002501249D60EA
:100E9000DC601B4C1A601C44241104F144056A11E7
:100EA000032692009E60174F0679174B47F82410CF
:100EB00002F1604202F5614205F01F05012000FACF
:100EC00005F5E6541560F0BC7047104C236843F4F8
:100ED0000003236000BF0E4B0E4DA4F58734A4F52C
:100EE0009E7401261E60234604609C68002CD0D0AE
:100EF0001033AB420360F8D1002303601846E2E7E9
:100F0000008FFCBF6093FF1F44E400E03C8004407E
:100F100000700340407103400168A9B10B4BF0B46D
:100F20000B441B110A4E0B4F0B4D46F8237003F177
:100F3000440202F01F0401235211A340002445F88B
:100F400022308C600460F0BC704700BF008FFCBF93
:100F50006093FF1F810E010080E100E0024A034B15
:100F6000012111601B6818470C7103406093FF1F3B
:100F7000024A034B012111605B6818471C71034052
:100F80006093FF1F024A034B012111609B681847C1
:100F90002C7103406093FF1F024A034B0121116033
:100FA000DB6818473C7103406093FF1FF8B50E469D
:100FB00071B17AB10746144600253B6816F8011B4B
:100FC0001B6838469847013C0544F6D12846F8BDD1
:100FD0000846F8BD1046F8BD00B5064A03681288F9
:100FE0005B6883B001A9ADF804200222984703B0E2
:100FF0005DF804FBA8630100F0B507468BB0002A3A
:1010000033D0012A08BF0A2251B3212400E0F4B2F0
:10101000B1FBF2F502FB1511C8B2092900F130014C
:1010200098BFC8B20AA988BF3730214488BFC0B270
:1010300001F8240C661E2946002DE8D133B1013C8D
:10104000E4B20AAB23442D2203F8242C3B6801AA06
:1010500011195B683846C4F1220298470BB0F0BD05
:1010600030228DF825202124E8E70368C9B21B68E7
:1010700098470BB0F0BD00BF0029BABF49422D23ED
:1010800000230A22FFF7B8BF08B5F0F757FEF1F7C3
:101090002BFB00F009F8FAE701F016BB01F01CBBCE
:1010A000704700BF704700BF2DE9F843314E3378D9
:1010B00093B1314F3A787AB90122D9073A7036D4D0
:1010C0009A0719D400225B073A7005D52B4B1A6892
:1010D00012B1EFF305820AB1BDE8F883EFF3108196
:1010E00072B6186818B1264C2278002A2ED0002932
:1010F000F2D162B6BDE8F883DFF8908098F800205E
:10110000002ADFD0DFF88890002405E0013498F849
:101110000030E4B2A34212D959F824502B68284673
:101120001B6998470028F1D02B699847EEE7FFF735
:10113000C9FCC8B9134B1B781BB93378C0E73378A7
:10114000C0E7337803F0FE033370B9E745691D60EB
:10115000012323705DB1AA6101B962B6002545770C
:10116000836898472570B7E700F092F8E2E7064BEE
:101170001D60F1E77293FF1FC5A2FF1FC0A2FF1FF2
:10118000C4A2FF1F5294FF1FBCA2FF1FD4A2FF1FC7
:10119000C8A2FF1FF0B44D1E2E46002400E001340B
:1011A000B0FBF2F302FB1300092800F130078ABFFD
:1011B0003730F8B2C0B206F8010F1846002BEED156
:1011C0000A1953704CB1107815F8016F287001336B
:1011D000E01A834202F80169F5DB0846F0BC70476B
:1011E00070B584B072B6194B194D1A487022412659
:1011F0000F2480211A702E701A460470197013780B
:101200001B06FCD5144B186862B6144B144C98425C
:1012100098BF00EB800001A998BF40000A22FFF7A9
:10122000B9FF01A92046002311F8012B01333AB17F
:101230000A2B20F8022FF7D11623237004B070BDBB
:101240005B00DBB2237004B070BD00BF0000024041
:101250000700024006000240080002407F96980006
:101260003C94FF1F30B40749074C0A782378074D98
:1012700042F0020245F823000A700133237030BCAB
:10128000704700BF7293FF1FD4A2FF1FC8A2FF1FA9
:10129000704700BFFFFFFFFF2DE9F043DFF8EC8050
:1012A0008BB006460F4600F073F898F90030013312
:1012B00004460D4637D03046394600F0DFF90028A5
:1012C00031D02BA3D3E900233046394600F02CFE61
:1012D000814668BB28A3D3E900233046394600F095
:1012E00005FE00B398F90030254ACDF8209004247B
:1012F00000200021022BCDE90467CDE902670094AC
:101300000192CDE906012CD0684600F0BDF940B34A
:10131000089B1BB101F0AAF9089B0360DDE90601F7
:101320000BB0BDE8F083204629460BB0BDE8F08342
:10133000134A98F90030019203210022CDE9046795
:10134000CDE90267009108922BB90E4B4FF0604235
:10135000CDE90623D8E70C490020022BCDE9060190
:10136000D2D101F083F922230360D1E7AFF30080EB
:10137000EF39FAFE422E864051302DD5104987C0F4
:101380001C640100FFFFEF470000F07F5394FF1F34
:101390002DE9F04FB04F21F00042BA4283B00C4625
:1013A0004FEAD17605460DD9AC4FBA4225D9C1F3E3
:1013B0001303034340F0EF800EB10020014603B059
:1013C000BDE8F08FA64B9A4200F2CC80A54B9A4222
:1013D00000F2DE808AA3D3E9002300F063F9002243
:1013E000A14B00F0A1FD002800F005812846214610
:1013F00000229D4B00F056F9E1E783A3D3E90023D7
:1014000000F092FD002840F0CB802846214680A3C2
:10141000D3E9002300F06AFD0028CED1934B284683
:1014200003EBC60821467CA3D3E9002300F0ECFAC5
:10143000D8E9002300F036F900F080FD804600F086
:101440007DFA77A3D3E9002306460F4600F0DCFAC5
:1014500002460B462846214600F022F972A3D3E942
:101460000023CDE900013046394600F0CDFA82462E
:101470008B4652465B46DDE9000100F011F9054656
:101480000C462A4623462846214600F0BDFA68A3AA
:10149000D3E9002306460F4600F0B6FA66A3D3E967
:1014A000002300F0FDF832463B4600F0ADFA64A39D
:1014B000D3E9002300F0F6F832463B4600F0A4FAE8
:1014C00061A3D3E9002300F0EBF832463B4600F07D
:1014D0009BFA5FA3D3E9002300F0E4F832463B46D1
:1014E00000F092FA02460B462846214600F0D8F852
:1014F00006460F462846214632463B46B8F1000FC5
:1015000056D000F081FA324604460D463B46002094
:101510004FF0804100F0C4F802460B4620462946B1
:1015200000F09CFB02460B465046594600F0B8F8C6
:10153000DDE9002300F0B4F80B4602464A490020DA
:1015400000F0AEF86FF47F7398454FDA08F57A78BB
:1015500001EB085100224FF0B87300F055FA03B0C8
:10156000BDE8F08F424B9A423FF658AF414BF40032
:101570002344D3E9002300F093F83F4BC6F1010860
:101580001C44CDE90001D4E900ABC6EB080870E7C4
:101590004FF0000875E702460B4600F083F80EE7AF
:1015A00017A3D3E900231046194600F02DFA06E7E9
:1015B00000F02AFA0022804689464FF080433046E8
:1015C000394600F06DF802460B464046494600F0A9
:1015D00045FB2A46234600F063F802460B460020EE
:1015E000214900F05DF803B0BDE8F08F01EB085130
:1015F00003B0BDE8F08F804643E700BFAFF3008043
:101600009C7500883CE4377EEF39FAFE422E864016
:1016100051302DD5104987C0FE822B654715F73F05
:101620000000E0FE422EE63F763C7935EF39EA3D98
:10163000D0A4BE726937663EF16BD2C541BDBB3ED8
:101640002CDE25AF6A56113F93BDBE166CC1663FB6
:101650003E5555555555C53F412E8640FFFFEF7FFE
:10166000422ED63FFFFF2F3E0000F03F20640100D6
:10167000B1A2F03F406401003064010041F000413C
:1016800001F58010C00F7047002070470B460146DF
:10169000184600F0E5BF00BF81F0004102E000BF46
:1016A00083F0004330B54FEA41044FEA430594EA22
:1016B000050F08BF90EA020F1FBF54EA000C55EA5D
:1016C000020C7FEA645C7FEA655C00F0E2804FEA2E
:1016D0005454D4EB5555B8BF6D420CDD2C4480EA10
:1016E000020281EA030382EA000083EA010180EA40
:1016F000020281EA0303362D88BF30BD11F0004F8E
:101700004FEA01314FF4801C4CEA113102D04042C3
:1017100061EB410113F0004F4FEA03334CEA1333FE
:1017200002D0524263EB430394EA050F00F0A78016
:10173000A4F10104D5F1200E0DDB02FA0EFC22FA11
:1017400005F2801841F1000103FA0EF2801843FA05
:1017500005F359410EE0A5F120050EF1200E012AF6
:1017600003FA0EFC28BF4CF0020C43FA05F3C01834
:1017700051EBE37101F0004507D54FF0000EDCF1AD
:10178000000C7EEB00006EEB0101B1F5801F1BD356
:10179000B1F5001F0CD349085FEA30004FEA3C0C5A
:1017A00004F101044FEA445212F5800F80F09A8050
:1017B000BCF1004F08BF5FEA500C50F1000041EB54
:1017C000045141EA050130BD5FEA4C0C404141EB58
:1017D000010111F4801FA4F10104E9D191F0000F7F
:1017E00004BF01460020B1FA81F308BF2033A3F102
:1017F0000B03B3F120020CDA0C3208DD02F1140CF9
:10180000C2F10C0201FA0CF021FA02F10CE002F133
:101810001402D8BFC2F1200C01FA02F120FA0CFC2C
:10182000DCBF41EA0C019040E41AA2BF01EB045175
:10183000294330BD6FEA04041F3C1CDA0C340EDC73
:1018400004F11404C4F1200220FA04F001FA02F3B6
:1018500040EA030021FA04F345EA030130BDC4F174
:101860000C04C4F1200220FA02F001FA04F340EA69
:101870000300294630BD21FA04F0294630BD94F01A
:10188000000F83F4801306BF81F480110134013D01
:101890004EE77FEA645C18BF7FEA655C29D094EA72
:1018A000050F08BF90EA020F05D054EA000C04BFF0
:1018B0001946104630BD91EA030F1EBF00210020DB
:1018C00030BD5FEA545C05D14000494128BF41F07A
:1018D000004130BD14F580043CBF01F5801130BDDE
:1018E00001F0004545F0FE4141F470014FF0000069
:1018F00030BD7FEA645C1ABF194610467FEA655C1A
:101900001CBF0B46024650EA013406BF52EA0335BB
:1019100091EA030F41F4002130BD00BF90F0000FA9
:1019200004BF0021704730B54FF4806404F13204E5
:101930004FF000054FF0000150E700BF90F0000F9E
:1019400004BF0021704730B54FF4806404F13204C5
:1019500010F0004548BF40424FF000013EE700BF95
:1019600042004FEAE2014FEA31014FEA02701FBF25
:1019700012F07F4393F07F4F81F06051704792F0F7
:10198000000F14BF93F07F4F704730B54FF4607471
:1019900001F0004521F0004120E700BF50EA0102BC
:1019A00008BF704730B54FF000050AE050EA010269
:1019B00008BF704730B511F0004502D5404261EBD9
:1019C00041014FF4806404F132045FEA915C3FF41A
:1019D000DCAE4FF003025FEADC0C18BF03325FEAB3
:1019E000DC0C18BF033202EBDC02C2F1200300FA68
:1019F00003FC20FA02F001FA03FE40EA0E0021FA8D
:101A000002F11444C1E600BF70B54FF0FF0C4CF476
:101A1000E06C1CEA11541DBF1CEA135594EA0C0F2C
:101A200095EA0C0F00F0DEF82C4481EA030621EA67
:101A30004C5123EA4C5350EA013518BF52EA0335A2
:101A400041F4801143F4801338D0A0FB02CE4FF054
:101A50000005E1FB02E506F00042E0FB03E54FF084
:101A60000006E1FB03569CF0000F18BF4EF0010E7C
:101A7000A4F1FF04B6F5007F64F5407404D25FEA78
:101A80004E0E6D4146EB060642EAC62141EA55512B
:101A90004FEAC52040EA5E504FEACE2EB4F1FD0C6D
:101AA00088BFBCF5E06F1ED8BEF1004F08BF5FEAEB
:101AB000500E50F1000041EB045170BD06F000469D
:101AC00046EA010140EA020081EA0301B4EB5C044A
:101AD000C2BFD4EB0C0541EA045170BD41F4801142
:101AE0004FF0000E013C00F3AB8014F1360FDEBF67
:101AF000002001F0004170BDC4F10004203C35DA43
:101B00000C341BDC04F11404C4F1200500FA05F3C5
:101B100020FA04F001FA05F240EA020001F0004266
:101B200021F0004110EBD37021FA04F642EB0601DC
:101B30005EEA430E08BF20EAD37070BDC4F10C0406
:101B4000C4F1200500FA04F320FA05F001FA04F2CA
:101B500040EA020001F0004110EBD37041F10001B6
:101B60005EEA430E08BF20EAD37070BDC4F12005C1
:101B700000FA05F24EEA020E20FA04F301FA05F229
:101B800043EA020321FA04F001F0004121FA04F2D1
:101B900020EA020000EBD3705EEA430E08BF20EAA1
:101BA000D37070BD94F0000F0FD101F000464000DB
:101BB00041EB010111F4801F08BF013CF7D041EA5D
:101BC000060195F0000F18BF704703F00046520061
:101BD00043EB030313F4801F08BF013DF7D043EA32
:101BE0000603704794EA0C0F0CEA135518BF95EAE8
:101BF0000C0F0CD050EA410618BF52EA4306D1D16F
:101C000081EA030101F000414FF0000070BD50EA8D
